:020000040800F2
:10000000007E0324BD020008D9A10008EF580008B3
:10001000DD98000843040008C7EF00080000000056
:1000200000000000000000000000000031C40008D3
:10003000650400080000000011A3000835C5000891
:10004000D7020008D7020008D7020008D70200082C
:10005000D7020008D7020008D7020008D70200081C
:10006000D7020008D7020008D7020008D70200080C
:10007000D7020008D7020008D7020008D7020008FC
:10008000D7020008D7020008D7020008D7020008EC
:10009000D7020008D7020008D7020008D7020008DC
:1000A000D7020008D7020008D7020008D7020008CC
:1000B000D7020008D7020008D1C50008D7020008FF
:1000C000D7020008D7020008D7020008D7020008AC
:1000D000D702000811D40008D7020008D702000890
:1000E000D7020008D702000800000000D70200086D
:1000F000D7020008D7020008D7020008D70200087C
:10010000D7020008D7020008D7020008D70200086B
:10011000D7020008D7020008D7020008D70200085B
:10012000D7020008D7020008D7020008D70200084B
:10013000D7020008D7020008D7020008D70200083B
:1001400000000000000000000000000000000000AF
:10015000D7020008D7020008D7020008D70200081B
:10016000D7020008D7020008D7020008D70200080B
:10017000D7020008D7020008D7020008D7020008FB
:10018000D7020008D7020008D7020008D7020008EB
:10019000D7020008D7020008D7020008D7020008DB
:1001A000D7020008D7020008D7020008D7020008CB
:1001B000D7020008D7020008D7020008D7020008BB
:1001C000D7020008D7020008D7020008D7020008AB
:1001D000D7020008DDA10008D7020008D7020008F6
:1001E000D7020008D7020008D7020008D70200088B
:1001F000D7020008D7020008D7020008D70200087B
:10020000D7020008D7020008D7020008D70200086A
:10021000D7020008D7020008D7020008D70200085A
:10022000D7020008D7020008D7020008000000002B
:10023000D7020008D702000800000000D70200081B
:10024000D7020008D7020008D7020008D70200082A
:10025000D7020008D7020008D7020008D70200081A
:10026000D7020008D7020008D7020008D70200080A
:10027000D7020008D7020008D702000800000000DB
:10028000D702000800000000D702000800000000AC
:1002900000000000D7020008DFF80CD000F094F84E
:1002A00000480047F1F80008007E032430BF72B612
:1002B000704762B6704780F30888704706488047E9
:1002C00006480047FEE7FEE7FEE7FEE7FEE7FEE73B
:1002D000FEE7FEE7FEE7FEE73DC5000899020008DD
:1002E0002DE9F05F0546002092469B46884606466B
:1002F000814640241BE0284641464746224600F0FE
:1003000053F853465A46C01A914110D31146184625
:10031000224600F03AF82D1A67EB01084F462246B4
:100320000120002100F031F817EB00094E41201E9A
:10033000A4F10104DFDC484631462A464346BDE8C5
:10034000F09F40EA01039B0703D009E008C9121F90
:1003500008C0042AFAD203E011F8013B00F8013B7F
:10036000521EF9D27047D2B201E000F8012B491EAB
:10037000FBD270470022F6E710B513460A46044642
:100380001946FFF7F0FF204610BD202A04DB203A73
:1003900000FA02F1002070479140C2F1200320FAD8
:1003A00003F3194390407047202A04DB203A21FAD6
:1003B00002F00021704721FA02F3D040C2F120027E
:1003C0009140084319467047064C074D06E0E06827
:1003D00040F0010394E8070098471034AC42F6D38C
:1003E000FFF75EFF345901085459010870B58C18A5
:1003F00010F8015B15F0070301D110F8013B2A1139
:1004000006D110F8012B03E010F8016B01F8016B25
:100410005B1EF9D12B0705D40023521E0DD401F821
:10042000013BFAE710F8013BCB1A921C03E013F8EA
:10043000015B01F8015B521EF9D5A142D8D300201F
:1004400070BD00BFFEE7000010B50AF01FF90AF00A
:10045000CFF80348006840F004000149086010BD6F
:100460009CEF00E0704730B5034614460022DA687E
:100470000022D1E9000540EA05200D8940EA054047
:100480000D7B40EA05600243DA60002030BD30B5E4
:100490000346144600229A680022D1E9000540EA8A
:1004A00005200D8940EA05400D7B40EA05600243C6
:1004B0009A60002030BD000010B50246002313688A
:1004C00009480340D1E901042043CC6820430C696A
:1004D00020434C6940EA44208C6940EA443003439D
:1004E0001360002010BD00008901F0FF70B50446C4
:1004F0001D460023B5F5804F13D154F822300C4827
:100500000340D1E9000640EA06108E6840EA062062
:100510008E8940EA06408E693043034344F8223016
:1005200003E06FF0704044F82200002070BD00002E
:100530000000F0CF10B502460023086852F82030C2
:100540001B480340D1E901042043CC6820430C69D7
:1005500020434C6920438C692043CC6920430C6ABA
:1005600020434C6A20438C6A2043CC6A20430C6BA6
:1005700020438C6B20434C6B20430343886808283E
:1005800001D143F04003086842F82030086BB0F511
:10059000801F05D1086818B110680C6B20431060EB
:1005A000086818B110684C6B20431060002010BD23
:1005B0008004C0FF30B5034614460022601C53F887
:1005C000202002F04042D1E9000540EA05108D6884
:1005D00040EA05208D8940EA0545088A401E45EA23
:1005E0000055087D801E45EA00608D69284302435E
:1005F000601C43F82020186800F4801038B1586857
:1006000020F47002088A401E42EA00525A6000201C
:1006100030BD30B50246002300240868012816D0FA
:1006200013686FF30E03D1E901052843CD68284311
:100630000D6928434D6928438D692843CD692843B6
:100640000D6A28434D6A28430343136019E0136879
:1006500023F4F843D1E9070528434D6A28430343AF
:1006600054686FF30E04D1E901052843CD6828438F
:100670000D6928434D6928438D692843044313605D
:100680005460002030BD0246506940EA410050618C
:100690000020704718B5034600200090D1E90004FF
:1006A00020438C68641E40EA4410CC6840EA442031
:1006B000009000981861002018BD000070B5034636
:1006C000154600220024012D1FD09A6802F07042C6
:1006D0000868401E4E68761E40EA06168868401E6E
:1006E00046EA0026C868401E46EA0036088A401ED0
:1006F00046EA0046888A401E46EA0056087E401EAA
:1007000046EA006002439A6022E09A68114802407B
:10071000C868401E0603888A401E46EA005002430D
:10072000DC6804F070440868401E4E68761E40EA9B
:1007300006168868401E46EA0026088A401E46EAD9
:100740000046087E401E46EA006004439A60DC6072
:10075000002070BDFF0F0FFF38B504464FF0AA30E0
:1007600000900949897901FB04F004236A460021BD
:1007700009F012FD044989796143481C04236A4643
:10078000002109F009FD38BDCC0B002438B5044622
:10079000002000900F49897901FB04F001236A468B
:1007A000002109F0A7FB9DF80000FF2810D109499E
:1007B00089796143481C01236A46002109F09AFBAC
:1007C0009DF80000FF2801D1002038BD0120FCE782
:1007D0000220FAE7CC0B0024F8B5054600260024D9
:1007E00006E04FF6FF703049496921F81400641C97
:1007F0002D484089A042F4D800202B49888100244C
:1008000033E02949897901FB04F004236A46002179
:1008100009F070FB9DF80000FF2809D145B122497D
:1008200089796143481C01236A46002109F062FB73
:100830009DF80000FF2813D19DF802009DF80310D9
:1008400000EB012618484089B04203D9164949698E
:1008500021F8164014488089401C1349888103E020
:10086000214612A00EF08EFD641C0F484089A04264
:10087000C7D800240BE00C48406930F814000A493E
:100880004989884202DB0849CC8104E0641C06489F
:100890004089A042EFD800BF0348C089642801DA2C
:1008A0000220F8BD0020FCE7CC0B0024626164202C
:1008B000626C6F636B20696E6465783A25640D0A1B
:1008C00000000000F8B5002600202D498881002492
:1008D00017E02046FFF75AFF05468DB9204609F07C
:1008E00089F805463DB1214626A00EF04BFD204675
:1008F000FFF732FF04E022488089401C20498881AC
:10090000641C1F484089A042E3D81D48818921A06A
:100910000EF038FD1A488089642801DA0120F8BDFC
:1009200017488089C0EB401000EB4000642190FB29
:10093000F1F600200090002415E02046FFF726FF86
:1009400005467DB90E49897901FB04F002236A4608
:10095000194609F021FC0098401C00900098B04214
:1009600000D104E0641C06484089A042E5D800BFDD
:100970000120FFF731FF08B10220D0E70020CEE7C9
:10098000CC0B002442616420626C6F636B3A256477
:100990000D0A0000676F6F645F626C6F636B6E754A
:1009A0006D3A25640D0A000010B509F053F808B13E
:1009B000012010BD1F48406920B11E484169002038
:1009C0000FF08AFA1B484089410000200FF096FA88
:1009D000184948610A4652895100164A5069FFF782
:1009E000C9FC1448406908B90120E2E70120FFF77B
:1009F000F3FE044664B110A00EF0C4FCFFF762FFE2
:100A00000446002C13D012A00EF0BCFC0220D0E74C
:100A10000848418913A00EF0B5FC0648818917A04B
:100A20000EF0B0FC0348C18919A00EF0ABFC002009
:100A3000BFE70000CC0B0024666F726D6174206EFE
:100A4000616E6420666C6173682E2E2E0D0A0000A4
:100A5000666F726D6174206661696C6564210D0A50
:100A600000000000746F74616C20626C6F636B2017
:100A70006E756D3A25640D0A00000000676F6F64A3
:100A800020626C6F636B206E756D3A25640D0A00F1
:100A900076616C696420626C6F636B206E756D3A71
:100AA00025640D0A0000000070B509480468456817
:100AB0008668344454B108220649204605F06AF895
:100AC000042204491031284605F064F870BD000086
:100AD0000010005C5202002410B504460CB901203D
:100AE00010BD94F83500022803D0802060650120F5
:100AF000F6E734492068884205D3334920688842A4
:100B000001D8012000E00020C0B1042084F83500A5
:100B10002C49206888420AD32B492068884206D88D
:100B20002068006820F001002168086048E0206823
:100B3000006820F001002168086041E0206800683A
:100B400020F00E00216808601E49206888420AD300
:100B50001D492068884206D82068006820F00100FE
:100B60002168086005E02068006820F00100216825
:100B70000860206E006820F48070216E086094F890
:100B80005C100120884011490860D4E919104860C0
:100B9000E06E40B1E06E006820F48070E16E0860A5
:100BA000D4E91C10486000BF002084F8340000BF66
:100BB000012084F83500206D10B12046216D884752
:100BC00000208DE710000240B8040240045402588F
:100BD00070B5044600F052F906462546681C10B16F
:100BE00004480078054400BF00F048F9801BA84283
:100BF000FAD370BD1C0000240348006840F00100D7
:100C0000014908607047000020040058F8B502460A
:100C10000B460021002600240020824D00BFFCE08E
:100C2000012707FA01F61F6807EA0604B4427CD1DF
:100C30005F68022F02D05F68122F1AD14FEAD10CE1
:100C400002F1200757F82C004F074FEAD76C0F2707
:100C500007FA0CF7B8434FEA417C4FEADC6C1F6996
:100C600007FA0CF738434FEAD10C02F1200747F896
:100C70002C0010684FEA410C032707FA0CF7B84321
:100C80001F7907F003074FEA410C07FA0CF73843C6
:100C900010605F68012F08D05F68022F05D05F6881
:100CA000112F02D05F68122F17D190684FEA410CC4
:100CB000032707FA0CF7B8434FEA410CDF6807FA3D
:100CC0000CF738439060506801278F40B8431F7974
:100CD000C7F300178F4038435060D0684FEA410C8B
:100CE000032707FA0CF7B8434FEA410C9F6807FA4D
:100CF0000CF73843D0605F6807F08057B7F1805F2A
:100D000095D100BF484F3F6847F00207DFF818C190
:100D1000CCF8007067463F6807F00207009700BFF5
:100D200000BF424F4FEA910C00E075E057F82C00ED
:100D30008F074FEA177C0F2707FA0CF7B8433C4F91
:100D4000BA4201D100272DE03A4FBA4201D1012722
:100D500028E0394FBA4201D1022723E0374FBA4287
:100D600001D103271EE0364FBA4201D1042719E012
:100D7000344FBA4201D1052714E0334FBA4201D1B2
:100D800006270FE0314FBA4201D107270AE0304F62
:100D9000BA4201D1082705E02E4FBA4201D10927F6
:100DA00000E00A274FEA817C4FEA1C7C07FA0CF727
:100DB00038431E4F4FEA910C47F82C002868A04397
:100DC0005F6807F48037B7F5803F00D12043286083
:100DD0006868A0435F6807F40037B7F5003F00D1AB
:100DE000204368604FF0B0473868A0435F6807F45D
:100DF0008017B7F5801F00D120434FF0B04738600F
:100E00007868A0435F6807F40017B7F5001F00D1AA
:100E100020434FF0B0477860491C1029FFF400AF21
:100E2000F8BD000080000058F4440258080400583F
:100E3000000002580004025800080258000C025832
:100E4000001002580014025800180258001C0258E2
:100E50000020025800240258024613690B400BB1CF
:100E6000012000E00020704742694A40426170471B
:100E70000AB1018300E04183704700000148006827
:100E800070470000140000240348006803490978F3
:100E90000844014908607047140000241C00002425
:100EA00010B5032000F02EFB002000F007F808B179
:100EB000012010BD00F034FA0020FAE770B50446B6
:100EC0000E4800784FF47A71B1FBF0F00C490968D4
:100ED000B1FBF0F5284604F09FFA08B1012070BD7F
:100EE000102C07D200222146501E00F0CDFA0548F2
:100EF000046001E00120F2E70020F0E71C0000247C
:100F0000000000241800002470B504460E46154663
:100F100000BF94F8A000012801D1022070BD01207B
:100F200084F8A00000BF022084F8A10005EB850131
:100F300001EBC50204F1380101EB82003422314695
:100F4000FFF7FFF92A463146204608F0F1F9012063
:100F50002168486284F8A10000BF002084F8A00046
:100F600000BF00BFDAE7000070B504460025002688
:100F70000CB9012070BD94F8A10028B9002084F8B4
:100F8000A000204600F07EF8022084F8A10020682E
:100F9000806920F0704021688861D4E9010108432C
:100FA000E168084321690843216889690843216889
:100FB0008861206880683249084021688860A08A7A
:100FC000050420688068A169294308432168886076
:100FD0002068C0682A4908402168C860A08B0504C1
:100FE0002068C068216A294308432168C8602068D6
:100FF00000692349084021680861A08C0504206825
:101000000069A16A29430843216808612068406992
:101010001B49084021684861A08D0504206840698B
:10102000216B294308432168486194F83500050283
:1010300094F8360006042068C06A00F07F402168FA
:10104000C86246EA050094F8341008432168C96A6A
:1010500008432168C8622068406B40F006002168A0
:1010600048632068806940F00100216888610020A1
:10107000C4F8A400012084F8A10000207AE7000051
:1010800000F800F010B586B0044600BF374800688D
:1010900040F00800354908600846006800F0080084
:1010A000009000BF00BF00BF30481038006840F01B
:1010B00010002E49103908600846006800F0100042
:1010C000009000BF00BF00BF2848001F006840F428
:1010D00080702649091F08600846006800F4807087
:1010E000009000BF00BF00BF0846006840F40070D9
:1010F00008600846006800F40070009000BF00BF60
:1011000000BF0846006840F4806008600846006838
:1011100000F48060009000BF00BF202001900120FB
:10112000029003900320049001A91148FFF76EFD7F
:101130004FF4E04001900220029000200390032031
:1011400004900E20059001A90A48FFF75FFD48F6BC
:101150007C60019001A90848FFF758FDFF2001902D
:1011600001A90648FFF752FD06B010BDE44402583D
:101170000004025800200258002402580028025897
:101180002DE9F04104460E461746984600BF94F8F4
:10119000A000012802D10220BDE8F081012084F8DE
:1011A000A00000BF022084F8A10008EB880000EB3B
:1011B000C80104F1380000EB81052E60A86A3044B4
:1011C0006860AF60E86A3844E860424629462046D5
:1011D00008F0AEF801202168486284F8A10000BF41
:1011E000002084F8A00000BF00BFD5E72DE9F04142
:1011F00004460E461746984600BF94F8A000012802
:1012000002D10220BDE8F081012084F8A00000BFD7
:10121000022084F8A10008EB880000EBC80104F16B
:10122000380000EB8105286830446860A8683844BD
:10123000E860AE62EF6242462946204608F078F840
:1012400001202168486284F8A10000BF002084F8D2
:10125000A00000BF00BFD5E74178154A11600178B2
:10126000F9B1121D41681160017B0907C27A41EA98
:101270000261827A41EAC241427B41EA8241827B39
:1012800041EA4241C27B41EA0241427A41EA0221FB
:10129000027A41EA420102781143054A083211609C
:1012A00005E00021024A121D1160121D11607047F5
:1012B00098ED00E000BF00BF00BFBFF35F8F00BF2D
:1012C00000BF00BF0548006820F480300349086073
:1012D00000200249703108607047000024ED00E0F2
:1012E00040F001010D4A11600C497039096841F460
:1012F00080310A4A703A116000BF00BF00BFBFF3DF
:101300004F8F00BF00BF00BF00BF00BF00BFBFF3D3
:101310006F8F00BF00BF00BF7047000094ED00E07A
:101320007047000070B504460E4615460CB9012002
:1013300070BD94F8210028B9002084F820002046D0
:1013400000F022F8211D2068FFF7B6F83146D4E9F5
:101350000002FFF79CF82946D4E90002FFF783F862
:101360002068006840F004002168086005480068B3
:1013700040F0004003490860012084F8210000206B
:10138000D6E700000040005210B586B0044600BF0A
:101390003148006840F480502F49086008460068D2
:1013A00000F48050009000BF00BF00BF2A480C30FE
:1013B000006840F0080028490C31086008460068C1
:1013C00000F00800009000BF00BF00BF08460068A2
:1013D00040F0100008600846006800F0100000901F
:1013E00000BF00BF00BF0846006840F04000086032
:1013F0000846006800F04000009000BF00BF402099
:10140000019000200290012003900320049001A984
:101410001248FFF7FBFB4FF400700190022002908E
:1014200000200390032004900C20059001A90C4893
:10143000FFF7ECFB4DF6330001900020039001A96B
:101440000648FFF7E3FB4FF4F060019001A905485F
:10145000FFF7DCFB06B010BDD4440258000C025864
:10146000001802580010025801460846002809DBFF
:1014700000F01F0301229A4043099B0003F1E0237F
:10148000C3F8002100BF70472DE9F05F80460D468C
:1014900016460DF087FF074639462A46334601F0C7
:1014A0000700C0F1070ABAF1040F02D94FF0040A8D
:1014B00001E0C0F1070AD14600F1040ABAF1070FB2
:1014C00002D24FF0000A01E0A0F1030AD4464FF027
:1014D000010A0AFA09FAAAF1010A0AEA020A0AFA50
:1014E0000CFA4FF0010B0BFA0CFBABF1010B0BEA02
:1014F000030B4AEA0B04214640460DF05BFFBDE8B2
:10150000F09F000000BF00F00702064B19684FF67D
:10151000FF031940044B0B4343EA0221014B1960BE
:1015200000BF70470CED00E00000FA0502461168AC
:101530000120C2F8F803886B40F400308863886BA0
:1015400040F48020886300207047000001460A684C
:101550000120C1F8F403002081F8EC03906940F009
:1015600000609061506D024B184350650020704739
:101570000300001070470246106841620020704767
:10158000F0B503461446002500221868426A21B9C6
:1015900042EA04401E68B06219E01868806A02EBF3
:1015A0001042002508E0186800F5827050F8250008
:1015B00002EB1042681CC5B2481EA842F3DC42EAA6
:1015C0000447186800F582704E1E40F8267000200F
:1015D000F0BD000010B50446012003490870D4F89E
:1015E000FC030CF0D3F910BD1B02002470B50446B7
:1015F0000D46C5EBC50304F1380101EB8301CA6850
:101600002946D4F8FC030CF011F970BD70B50446FE
:101610000D46C5EBC50304F5FC7101EB8301CA68F7
:101620002946D4F8FC030CF06EF970BD10B50446E1
:1016300000200549087005A00DF0A4FED4F8FC03B5
:101640000CF0A7F910BD00001B02002455534220E6
:1016500044657669636520446973636F6E6E656384
:101660007465642E0D0A000070B504460D46002610
:1016700005F08000802808D105F07F00C0EBC00194
:1016800004F1380000EB810607E005F07F00C0EBB5
:10169000C00104F5FC7000EB810605F07F0030709E
:1016A00005F08000C009707000BF94F8B8030128ED
:1016B00001D1022070BD012084F8B80300BF31467B
:1016C00020680CF04BFF00BF002084F8B80300BF77
:1016D00000BFEFE770B504460D46002605F0800018
:1016E000802808D105F07F00C0EBC00104F138006C
:1016F00000EB810605E0C5EBC50104F5FC7000EBCD
:1017000081060020B07005F07F003070C5F3C01076
:10171000707000BF94F8B803012801D1022070BD99
:10172000012084F8B80300BF314620680DF060F94D
:1017300000BF002084F8B80300BF00BFEFE770B51A
:1017400004460D4600BF94F8B803012801D10220D9
:1017500070BD012084F8B80300BF05F08000802828
:1017600005D105F07F0120680DF052FB02E02068F2
:101770000DF038FB00BF002084F8B80300BF00BFA5
:10178000E6E7024601F00F00C0EBC00302F5FC7073
:1017900000EB8300008B80B270472DE9F0470546CF
:1017A0000E4690461F464FF00009002406F08000C8
:1017B000802808D106F07F00C0EBC00105F1380099
:1017C00000EB810407E006F07F00C0EBC00105F5E7
:1017D000FC7000EB810406F07F00207006F08000B2
:1017E000C0096070C4F80880E770607808B120789C
:1017F000E080022F01D10020207100BF95F8B803CE
:10180000012802D10220BDE8F087012085F8B80345
:1018100000BF214628680CF0BFFD00BF002085F8FE
:10182000B80300BF4846EEE72DE9F04104460E46F6
:1018300017469846002506F07F00C0EBC00104F56E
:10184000FC7000EB8105EF60C5F814800020A861F2
:10185000687006F07F0028702069012800D12F6190
:1018600006F07F0028B9227C294620680CF0C6FFCC
:1018700004E0227C294620680DF044F90020BDE8F0
:10188000F08170B504460D46002605F080008028E2
:1018900008D105F07F00C0EBC00104F1380000EB77
:1018A000810605E0C5EBC50104F5FC7000EB81067F
:1018B0000120B07005F07F003070C5F3C01070706B
:1018C00000BF94F8B803012801D1022070BD0120A7
:1018D00084F8B80300BF314620680DF0CDF805F05C
:1018E0007F0028B9217C04F56F7220680DF05EF846
:1018F00000BF002084F8B80300BF00BFE6E72DE971
:10190000F04104460E4617469846002506F07F0033
:10191000C0EBC00104F1380000EB8105EF60C5F8B1
:1019200014800020A8610120687006F07F002870F4
:101930002069012800D12F6106F07F0028B9227CA0
:10194000294620680CF05AFF04E0227C29462068D2
:101950000DF0D8F80020BDE8F08100002DE9FC5F13
:10196000044626684FF0000B0020019080460025B9
:10197000009081468246FE4F20680DF083FA0028D1
:101980007DD120680DF0B6FA08B9BDE8FC9F20684B
:101990000DF0B0FA00F00200022801D12168486180
:1019A00020680DF0A7FA00F40020B0F5002F67D1F1
:1019B000002520680DF074FA0190A8E0019800F06D
:1019C000010000287ED0E9B220680DF088FA804638
:1019D00008F00100002860D0012106F5306000EB1E
:1019E00045108160306CE34988420ED3206901289C
:1019F0000BD1D6F8080B00F4004030B14FF4004191
:101A000006F5306000EB45108160206901282BD17C
:101A1000C5EBC50104F5FC7000EB8100816806F59B
:101A2000306000EB45100069C0F31200091AC5EBE5
:101A3000C50204F5FC7000EB82008161C5EBC501B5
:101A400004F5FC7000EB8100C5EBC502C16804F52C
:101A5000FC7000EB820080680144C5EBC50204F510
:101A6000FC7000EB8200C160E9B22046FFF7CEFDBA
:101A70002069012811D185B9C5EBC50101E0EEE26D
:101A800049E004F5FC7000EB8100406928B904F5D9
:101A90006F72012120680CF089FF08F00800082807
:101AA0001DD1306CB349884210D3206901280DD173
:101AB000D6F8080B00F4004040B14FF4004106F5A1
:101AC000306000E01FE000EB45108160204600F030
:101AD00071FC082106F5306000EB4510816008F0CC
:101AE0001000102805D1102106F5306000EB4510DC
:101AF000816008F02000202805D1202106F5306003
:101B000000EB451081606D1C019840080190019820
:101B100000287FF453AF20680DF0ECF900F480202A
:101B2000B0F5802F7DD120680DF0B1F9019000252E
:101B300085E0019800F0010000287CD0E9B220681F
:101B40000DF0B7F9804608F00100E8B30120A84085
:101B5000009040F6340080590099884340F63401E3
:101B60008851012106F5106000EB45108160206965
:101B7000012815D1C5EBC50104F1380000EB810047
:101B8000C5EBC502C16804F1380000EB8200806833
:101B90000144C5EBC50204F1380000EB8200C160CE
:101BA000E9B22046FFF722FD2069012810D15DB976
:101BB000C5EBC50104F1380000EB8100406918B99C
:101BC00004F56F72012100E002E020680CF0EEFEE7
:101BD00008F00800082805D1082106F5106000EB80
:101BE0004510816008F01000102805D1102106F57D
:101BF000106000EB4510816008F04000402805D1DE
:101C0000402106F5106000EB4510816008F00200ED
:101C1000022805D1022106F5106000EB4510816015
:101C200001E010E007E008F08000802803D1294699
:101C3000204608F0DBFA6D1C0198400801900198DD
:101C400000287FF476AF20680DF054F900F00040D2
:101C5000B0F1004F1AD140F60400805920F0010184
:101C600040F60400815194F8EC03012807D10020CC
:101C700084F8EC0300212046FFF77CFC02E02046BC
:101C800000F064FB4FF000402168486120680DF0CF
:101C900031F900F40060B0F5006F0CD140F6080097
:101CA000805900F0010010B1204600F097FB4FF47E
:101CB00000602168486120680DF01CF900F00060A8
:101CC000B0F1006F17D14FF000602168486194F8BF
:101CD000EC0368B9012084F8EC032068406DC0F380
:101CE0008300C4F8F00301212046FFF743FC02E023
:101CF000204600F073FB20680DF0FCF800F48050E3
:101D0000B0F5805F60D140F60400805920F00101F9
:101D100040F604008151102120680DF079F84FF051
:101D2000000B0CE0FF2106F5106000EB4B1081600A
:101D300006F5306000EB4B1081600BF1010B606821
:101D40005845EFD84FF0FF3140F618008151001D83
:101D5000805940F0011140F61C008151206BA0B168
:101D6000D6F8840840F00B01C6F8841804E000009F
:101D70000084D7170A31544F40F64400805940F090
:101D80000B0140F6440081510EE040F614008059EA
:101D900040F00B0140F614008151001F805940F0C3
:101DA0000B014FF401608151D6F8000820F4FE6069
:101DB000C6F80008217C04F56F7220680CF0F6FD6F
:101DC0004FF480502168486120680DF093F800F4CA
:101DD0000050B0F5005F7AD120680CF03FFB20681E
:101DE000C06820F470502168C86020680DF028F8A1
:101DF00058B90021E1604FF4007161612068C0684A
:101E000040F410502168C86082E00321E160402165
:101E1000616101F02DFC07469248874209D3924840
:101E2000874206D22068C06840F470502168C860BC
:101E30006EE08D48874209D38C48874206D22068DD
:101E4000C06840F460502168C86061E087488742FC
:101E500009D38748874206D22068C06840F45050B2
:101E60002168C86054E08248874209D3814887428C
:101E700006D22068C06840F440502168C86047E03E
:101E80007C48874209D37C48874206D22068C068D4
:101E900040F430502168C8603AE07748874209D35F
:101EA0007648874206D22068C06840F420502168F6
:101EB000C8602DE0714887420AD37148874207D233
:101EC0002068C06840F410502168C86020E026E017
:101ED0006B48874209D36B48874206D22068C068A6
:101EE00040F400502168C86012E06648874209D378
:101EF0006548874206D22068C06840F4E0502168F7
:101F0000C86005E02068C06840F4C0502168C8601F
:101F1000204600F0CFF94FF4005021684861206856
:101F20000CF0E8FF00F01000102845D1206880690F
:101F300020F0100021688861D6F8209009F00F0089
:101F4000C0EBC00104F5FC7000EB810AC9F343400B
:101F500002281AD147F6F07009EA000030B3C9F33D
:101F60000A123046DAF80C100CF0CAFFC9F30A1155
:101F7000DAF80C000844CAF80C00C9F30A11DAF8C0
:101F800018000844CAF8180010E0C9F343400628B6
:101F90000CD1082204F56F7130460CF0B1FFC9F383
:101FA0000A11DAF818000844CAF818002068806995
:101FB00040F010002168886120680CF09BFF00F061
:101FC0000800082805D1204600F0D4F9082021682F
:101FD000486120680CF08EFF00F48010B0F5801F7F
:101FE00007D1E9B2204600F051F84FF48010216883
:101FF000486120680CF07EFF00F40010B0F5001F6F
:1020000007D1E9B2204600F04AF84FF400102168E9
:10201000486120680CF06EFF00F08040B0F1804F06
:1020200006D12046FFF7D6FA4FF08040216848617C
:1020300020680CF05FFF00F0040004280FD1206836
:10204000D0F8049009F00400042802D12046FFF7DC
:10205000EDFA2068406840EA09002168486000BF46
:1020600093E40000C0ACD800C0E1E4000024F40018
:1020700080730601A0491A01002D310140A44C01D2
:1020800000366E0120ABA6010048E80170B5044699
:102090000D462946D4F8FC030BF0EAFC70BD70B580
:1020A00004460D462946D4F8FC030BF0E4FC70BD51
:1020B00030B58BB00446002514B901200BB030BDFB
:1020C000032084F8B903204600F0A0F820680CF043
:1020D0008DFB282204F110016846FEF732F994E8DE
:1020E0000F000CF0DDF9002120680CF01DFF002529
:1020F00030E00121C5EBC50204F1380000EB82009D
:102100004170C5EBC50204F1380000F82250C5EB60
:10211000C50200EB8200C5800021C5EBC50204F1B9
:10212000380000EB8200C170C5EBC50204F1380035
:1021300000EB82008160C5EBC50204F1380000EBC2
:102140008200C160C5EBC50204F1380000EB8200DB
:1021500041616D1C0F2DCCD3002536E00021C5EB6D
:10216000C50204F5FC7000EB82004170C5EBC502AE
:1021700004F5FC7000F82250C5EBC50204F13800EC
:1021800000EB8200C580C5EBC50204F5FC7000EBD6
:102190008200C170C5EBC50204F5FC7000EB820043
:1021A0008160C5EBC50204F5FC7000EB8200C160E4
:1021B000C5EBC50204F5FC7000EB820041612068AC
:1021C00000F5827040F825106D1C0F2DC6D3282213
:1021D00004F110016846FEF7B4F894E80F000CF023
:1021E0002FFA012084F8B903A06A012802D1204601
:1021F000FFF7ACF9606A012802D12046FFF796F993
:1022000020680CF00EFA002058E7000010B5B6B0B8
:1022100004464FF4802002904FF44010239002A80F
:1022200000F062FB20492068884239D100BF1F4876
:10223000006840F001001D4908600846006800F091
:102240000100019000BF00BF4FF4C0503190022048
:10225000329000203390032034900A20359031A929
:102260001348FEF7D3FC0121032008F02AF800BF31
:102270000E480838006840F000600C4908390860D2
:102280000846006800F00060019000BF00BF002217
:1022900001216520FFF7F8F86520FFF7E5F800E079
:1022A00000BF36B010BD000000000840E0440258F6
:1022B0000000025870B504460125E06810B10228FC
:1022C0000AD104E00CA00DF05DF8002509E011A092
:1022D0000DF058F8012504E015A00DF053F8012584
:1022E00000BF00BFD4F8FC030BF0E8FB2946D4F88C
:1022F000FC030BF01DFC70BD55534220446576690C
:102300006365204C69627261727920205B48535D7D
:102310000D0A000055534220446576696365204CE0
:1023200069627261727920205B46535D0D0A00007C
:1023300055534220446576696365204C6962726139
:10234000727920205B46533F5D0D0A0010B50446AC
:1023500003A00DF017F8D4F8FC030BF0D1FB10BD6F
:1023600044657669636520526573756D65640D0A11
:102370000000000010B50446D4F8FC030BF0C7FBC6
:1023800010BD70B504460D4600BF94F8B80301288F
:1023900001D1022070BD012084F8B80300BF294696
:1023A00020680CF0D9FD00BF002084F8B80300BFFE
:1023B00000BFEFE710B5044604F56F71D4F8FC03D5
:1023C0000BF0CAFB10BD10B5044620680CF01AF9DA
:1023D00020680CF0FFFC002010BD000010B5044682
:1023E00000200549087005A00CF0CCFFD4F8FC03D0
:1023F0000BF0FBFB10BD00001B0200244465766956
:10240000636520496E2073757370656E64206D6F0F
:1024100064652E0D0A0000000348006840F08070DB
:1024200001490860704700000C48025810B501F0DF
:1024300067F90949096801F470614FF4807292FAF2
:10244000A2F2B2FA82F2D140044A515CC840044977
:1024500008600846006810BD18440258E4100108DE
:102460000000002410B501F003F90749096801F0E4
:102470007001102292FAA2F2B2FA82F2D140034A1B
:10248000515CC84010BD000020440258E41001080F
:1024900070B5014600220120002300249FED811A1F
:1024A000B0EE410A9FED7F1AF0EE410A7E4D2D6895
:1024B00005F003027C4D2D68C5F305307A4D2D1DC6
:1024C0002D6805F01003784D14352D68C5F3CC0543
:1024D00015FB03F501EE105AB8EE411AB0EE410AB1
:1024E00022B1012A4DD0022A7DD169E06E4D283DEE
:1024F0002D68C5F340152DB36B4D283D2D68C5F3F0
:10250000C1066A4D25FA06F4B4FBF0F501EE105A47
:10251000F8EE411A9FED661A80EE012A624D1035E1
:102520002D68C5F3080501EE105AB8EE411A32EED7
:10253000011AB7EE002A31EE021A21EE811AF0EEEE
:10254000410A1DE0594DB5FBF0F501EE105AF8EEC9
:10255000411A9FED571A80EE012A534D10352D6810
:10256000C5F3080501EE105AB8EE411A32EE011A11
:10257000B7EE002A31EE021A21EE811AF0EE410A7E
:102580005EE04C4DB5FBF0F501EE105AB8EE412A75
:102590009FED471AC0EE011A434D10352D68C5F363
:1025A000080501EE105AB8EE411A31EE811AF7EE25
:1025B000001A31EE211A22EE011AF0EE410A3FE034
:1025C0003D4DB5FBF0F501EE105AF8EE411A9FEDC6
:1025D000381A80EE012A344D10352D68C5F30805F0
:1025E00001EE105A00E00CE0B8EE411A32EE011A8A
:1025F000B7EE002A31EE021A21EE811AF0EE410AFE
:102600001EE02C4DB5FBF0F501EE105AB8EE412A54
:102610009FED271AC0EE011A234D10352D68C5F322
:10262000080501EE105AB8EE411A31EE811AF7EEA4
:10263000001A31EE211A22EE011AF0EE410A00BF13
:1026400000BF194D10352D68C5F346256D1C01EEF0
:10265000105AB8EE411AC0EE811ABCEEE11A81EDB3
:10266000001A114D10352D68C5F306456D1C01EE9D
:10267000105AB8EE411AC0EE811ABCEEE11A81ED93
:10268000011A094D10352D68C5F306656D1C01EE64
:10269000105AB8EE411AC0EE811ABCEEE11A81ED73
:1026A000021A70BD00000000284402580090D003B8
:1026B0000000004600093D0040787D0170B50146EC
:1026C00000220120002300249FED811AB0EE410A70
:1026D0009FED7F1AF0EE410A7E4D2D6805F0030252
:1026E0007C4D2D68C5F305507A4D2D1D2D6805F4E0
:1026F0008073784D1C352D68C5F3CC0515FB03F5AB
:1027000001EE105AB8EE411AB0EE410A22B1012A88
:102710004DD0022A7DD169E06E4D283D2D68C5F36C
:1027200040152DB36B4D283D2D68C5F3C1066A4D8C
:1027300025FA06F4B4FBF0F501EE105AF8EE411A52
:102740009FED661A80EE012A624D18352D68C5F39B
:10275000080501EE105AB8EE411A32EE011AB7EE32
:10276000002A31EE021A21EE811AF0EE410A1DE034
:10277000594DB5FBF0F501EE105AF8EE411A9FEDF8
:10278000571A80EE012A534D18352D68C5F30805F8
:1027900001EE105AB8EE411A32EE011AB7EE002AD5
:1027A00031EE021A21EE811AF0EE410A5EE04C4D44
:1027B000B5FBF0F501EE105AB8EE412A9FED471A2D
:1027C000C0EE011A434D18352D68C5F3080501EE1A
:1027D000105AB8EE411A31EE811AF7EE001A31EEB6
:1027E000211A22EE011AF0EE410A3FE03D4DB5FB01
:1027F000F0F501EE105AF8EE411A9FED381A80EE0E
:10280000012A344D18352D68C5F3080501EE105A1C
:1028100000E00CE0B8EE411A32EE011AB7EE002AE1
:1028200031EE021A21EE811AF0EE410A1EE02C4D23
:10283000B5FBF0F501EE105AB8EE412A9FED271ACC
:10284000C0EE011A234D18352D68C5F3080501EEB9
:10285000105AB8EE411A31EE811AF7EE001A31EE35
:10286000211A22EE011AF0EE410A00BF00BF194DF5
:1028700018352D68C5F346256D1C01EE105AB8EECB
:10288000411AC0EE811ABCEEE11A81ED001A114D19
:1028900018352D68C5F306456D1C01EE105AB8EECB
:1028A000411AC0EE811ABCEEE11A81ED011A094D00
:1028B00018352D68C5F306656D1C01EE105AB8EE8B
:1028C000411AC0EE811ABCEEE11A81ED021A70BD08
:1028D00000000000284402580090D0030000004689
:1028E00000093D0040787D012DE9F04104460025B6
:1028F0000026206800F00060B0F1006F30D1606EFB
:1029000048B1B0F5801F0DD0B0F5001F10D0B0F564
:10291000401F15D113E0F948006840F40030F74932
:1029200008600FE00221201D07F0F4FC054609E0D5
:10293000022104F1240007F085FD054602E001E0D4
:10294000012500BF00BF55B9EC482430006820F4D1
:102950004010616E0843E9492431086000E02E43CD
:10296000208800F48070B0F5807F2DD1606D05283F
:102970001AD2DFE800F0030A10171800DF480068D9
:1029800040F40030DD49086010E00021201D07F010
:10299000C1FC05460AE0002104F1240007F052FDC5
:1029A000054603E002E001E0012500BF00BF55B984
:1029B000D2482430006820F00700616D0843CF49F9
:1029C0002431086000E02E43208800F40070B0F548
:1029D000007F33D1A06D802817D003DC40B14028A0
:1029E0001CD10CE0C02817D0B0F5807F16D114E0C0
:1029F000C248006840F40030C049086010E000217F
:102A0000201D07F087FC05460AE0002104F12400A0
:102A100007F018FD054603E002E001E0012500BFD4
:102A200000BF55B9B5482430006820F4E070A16DAE
:102A30000843B2492431086000E02E43208800F4A6
:102A40008060B0F5806F38D1D4F8A400B0F5800F65
:102A500019D004DC50B1B0F5001F1DD10DE0B0F568
:102A6000C00F17D0B0F5000F16D114E0A3480068CE
:102A700040F40030A149086010E00021201D07F05B
:102A800049FC05460AE0002104F1240007F0DAFCC5
:102A9000054603E002E001E0012500BF00BF5DB98B
:102AA00096482C30006820F46000D4F8A410084345
:102AB00092492C31086000E02E43208800F4006029
:102AC000B0F5006F38D1D4F8A800B0F1007F19D06C
:102AD00004DC50B1B0F1807F1DD10DE0B0F1407F3A
:102AE00017D0B0F1806F16D114E08448006840F42C
:102AF00000308249086010E00021201D07F00AFC28
:102B000005460AE0002104F1240007F09BFC05467D
:102B100003E002E001E0012500BF00BF5DB9774896
:102B20002C30006820F0E060D4F8A8100843734906
:102B30002C31086000E02E43206800F00070B0F1F6
:102B4000007F27D1A06CA0B1102804D0202809D084
:102B500030280FD10CE06948006840F40030674924
:102B6000086009E00221201D07F0D4FB054603E0C0
:102B700002E001E0012500BF00BF55B95F482030E9
:102B8000006820F03000A16C08435C4920310860E7
:102B900000E02E43208800F48050B0F5805F36D1ED
:102BA000E06DB0F5005F19D004DC50B1B0F5805F86
:102BB0001DD10DE0B0F5405F17D0B0F5804F16D1B4
:102BC00014E04E48006840F400304C49086010E0C2
:102BD0000021201D07F09EFB05460AE0002104F1BC
:102BE000240007F02FFC054603E002E001E0012588
:102BF00000BF00BF55B941482430006820F4E040D0
:102C0000E16D08433D492431086000E02E432088EF
:102C100000F40050B0F5005F34D1206EB0F5403FB5
:102C20001DD007DC68B1B0F5803F0BD0B0F5003F98
:102C300018D10DE0B0F5802F12D0B0F5A02F11D132
:102C40000FE011E00121201D07F064FB05460BE0B9
:102C5000012104F1240007F0F5FB054604E003E040
:102C600002E001E0012500BF00BF55B92348243030
:102C7000006820F4E020216E0843204924310860D8
:102C800000E02E43208800F48040B0F5804F38D11A
:102C9000D4F8AC00B0F1405F1DD007DC68B1B0F1F2
:102CA000805F0BD0B0F1005F18D10DE0B0F1804F24
:102CB00012D0B0F1A04F11D10FE011E00121201D81
:102CC00007F028FB05460BE0012104F1240007F082
:102CD000B9FB054604E003E002E001E0012500BF86
:102CE00000BF6DB905482C30006820F0E040D4F8F2
:102CF000AC10084301492C31086002E02C44025812
:102D00002E43208800F40040B0F5004F26D1E06E3D
:102D100098B1B0F1805F03D0B0F1005F0ED106E052
:102D2000FA48006840F40030F849086008E00121E2
:102D3000201D07F0EFFA054602E001E0012500BF83
:102D400000BF55B9F1482430006820F04050E16ED2
:102D50000843EE492431086000E02E43206800F06B
:102D60008070B0F1807F27D1606CA0B1012804D0C1
:102D7000022809D003280FD10CE0E448006840F491
:102D80000030E249086009E00221201D07F0C2FA84
:102D9000054603E002E001E0012500BF00BF55B990
:102DA000DA482030006820F00300616C0843D749FE
:102DB0002031086000E02E43206800F48000B0F568
:102DC000800F7DD1D248006840F48070D0490860FF
:102DD000FEF754F8074606E0FEF750F8C01B6428DB
:102DE00001D9032505E0CA48006800F48070002876
:102DF000F2D000BF8DBBC5484430006800F440707D
:102E0000B4F8B01001F44071884214D0BF48443087
:102E1000006820F44078BD484430006840F48030B9
:102E2000BA49443108600846006820F480300860E0
:102E30000846C0F80080D4F8B000B0F5807F15D106
:102E4000FEF71CF8074609E0FEF718F8C01B41F230
:102E50008831884202D9032507E038E0AB48443086
:102E60000068C0F340000028EED000BF4DBB00BF9B
:102E7000B4F8B00000F44070B0F5407F0ED1A34824
:102E80001C38006820F47C51A24AD4F8B0001040ED
:102E900041EA10109D491C39086007E09B481C3826
:102EA000006820F47C5099491C39086097484430E8
:102EB0000068B4F8B010C1F30B010843934901E076
:102EC00006E002E04431086002E02E4300E02E43B9
:102ED000207800F0010068B3A06F182819D005DC35
:102EE00048B1082808D0102816D10BE0202811D0AE
:102EF000282811D10FE011E00121201D07F00AFA66
:102F000005460BE0012104F1240007F09BFA054679
:102F100004E003E002E001E0012500BF00BF55B975
:102F20007A482830006820F03800A16F08437749BC
:102F30002831086000E02E43207800F002000228CB
:102F400028D1606F062815D2DFE800F003040A11CB
:102F5000121311E00121201D07F0DCF905460BE0FA
:102F6000012104F1240007F06DFA054604E003E0B6
:102F700002E001E0012500BF00BF55B963482830D9
:102F8000006820F00700616F08436049283108603D
:102F900000E02E43207800F0040004282AD1D4F861
:102FA0009000062815D2DFE800F003040A1112137E
:102FB00011E00121201D07F0ADF905460BE00121CC
:102FC00004F1240007F03EFA054604E003E002E0C5
:102FD00001E0012500BF00BF5DB94C482C300068FE
:102FE00020F00700D4F89010084348492C310860BD
:102FF00000E02E43207800F02000202836D1D4F8BD
:103000008C00B0F1405F1DD007DC68B1B0F1805F8B
:103010000BD0B0F1005F18D10DE0B0F1804F12D0AD
:10302000B0F1A04F11D10FE011E00021201D07F0F9
:1030300071F905460BE0022104F1240007F002FAC1
:10304000054604E003E002E001E0012500BF00BF07
:103050005DB92E482830006820F0E040D4F88C108C
:1030600008432A492831086000E02E43207800F008
:103070004000402836D1D4F89800B0F5406F1DD0FC
:1030800007DC68B1B0F5806F0BD0B0F5006F18D1D8
:103090000DE0B0F5805F12D0B0F5A05F11D10FE068
:1030A00011E00021201D07F035F905460BE0022153
:1030B00004F1240007F0C6F9054604E003E002E04D
:1030C00001E0012500BF00BF5DB910482C30006849
:1030D00020F4E050D4F8981008430C492C310860D3
:1030E00000E02E43207800F0800080283BD1D4F807
:1030F0009C00B0F5C04F24D00EDCA0B1B0F5005F4D
:1031000012D0B0F5804F1FD114E000002C440258BB
:1031100000480258FFFCFF0FB0F5004F12D0B0F589
:10312000204F11D10FE011E00021201D07F0F2F82F
:1031300005460BE0022104F1240007F083F905465F
:1031400004E003E002E001E0012500BF00BF4DB94B
:10315000B248006820F46040D4F89C100843AF499E
:10316000086000E02E43207800F00800082816D1FF
:10317000D4F88000B0F5805F06D1022104F124006C
:1031800007F060F906430AE0A448001F006820F435
:103190004050D4F880100843A049091F08602078E7
:1031A00000F01000102814D1D4F89400B0F5807FFE
:1031B00006D1022104F1240007F044F9064308E097
:1031C0009648006820F44070D4F89410084393495E
:1031D0000860206800F40020B0F5002F26D1D4F854
:1031E000A00030B1B0F5803F09D0B0F5003F0ED15E
:1031F0000CE00021201D07F08DF8054609E00221B2
:1032000004F1240007F01EF9054602E001E0012563
:1032100000BF00BF4DB98148006820F44030D4F8A9
:10322000A01008437D49086000E02E43206800F4A8
:103230008020B0F5802F2DD1D4F88400B0F5801F08
:1032400006D0B0F5001F0CD0B0F5401F11D10FE033
:1032500072482C38006840F4003070492C390860FE
:1032600009E0012104F1240007F0ECF8054602E032
:1032700001E0012500BF00BF5DB96848001F00687C
:1032800020F44010D4F8841008436449091F0860F2
:1032900000E02E43206800F48030B0F5803F24D158
:1032A000E06C18B1B0F5803F0FD108E05B482C38D6
:1032B000006840F4003059492C39086007E00221C9
:1032C000201D07F027F8054601E0012500BF00BFDB
:1032D00055B952480C38006820F48030E16C08433E
:1032E0004E490C39086000E02E43206800F0005081
:1032F000B0F1005F05D1022104F1240007F0A2F82B
:103300000643206800F40030B0F5003F27D1E06F9D
:10331000A0B1B0F5807F06D0B0F5007F0CD0B0F53D
:10332000407F0CD109E03D482C38006840F4003063
:103330003A492C39086004E003E002E001E001258D
:1033400000BF00BF55B93548001F006820F4407029
:10335000E16F08433149091F086000E02E432068EF
:1033600000F48010B0F5801F09D12C48083800689F
:1033700020F00040216F0843284908390860206880
:1033800000F08050B0F1805F0AD1244848380068CE
:1033900020F48040D4F8B41008432049483908602C
:1033A000206800F40010B0F5001F09D11B48083850
:1033B000006820F08070A16E084318490839086041
:1033C000206800F08040B0F1804F11D100BF134859
:1033D0004838006820F40040104948390860084621
:1033E0000068D4F8B81008430C494839086000BF99
:1033F000206800F00040B0F1004F09D107480C38B8
:10340000006820F04050216D084304490C390860E1
:1034100016B90020BDE8F0810120FBE758440258AE
:1034200070B504460D4600268D48006800F0070080
:10343000A8420ED28A48006820F007002843884935
:1034400008600846006800F00700A84201D001208B
:1034500070BD207800F00200022807D18148006882
:1034600020F00F00E16808437E490860207800F0F2
:103470000100002851D07B48006820F47060A168EA
:103480000843784908606068022807D175481838F1
:103490000068C0F34040F8B90120D9E7606803280C
:1034A00007D1704818380068C0F34060A0B9012007
:1034B000CEE76068012807D16A4818380068C0F371
:1034C000002048B90120C3E7664818380068C0F3F7
:1034D000800008B90120BBE762480838006820F086
:1034E0000700616808435F4908390860FDF7C6FCBA
:1034F00006466068022811D108E0FDF7BFFC801B7A
:1035000041F28831884201D90320A1E755480838A3
:10351000006800F038001028EFD13AE06068032816
:1035200011D108E0FDF7AAFC801B41F288318842E6
:1035300001D903208CE74B480838006800F03800B8
:103540001828EFD125E06068012811D108E0FDF7C7
:1035500095FC801B41F28831884201D9032077E72E
:1035600040480838006800F038000828EFD110E023
:1035700008E0FDF783FC801B41F28831884201D9C5
:10358000032065E737480838006800F03800002855
:10359000EFD13348006800F00700A8420ED9304848
:1035A000006820F0070028432D490860084600689D
:1035B00000F00700A84201D0012049E7207800F080
:1035C0000400042807D12748006820F07000216912
:1035D000084324490860207800F00800082809D131
:1035E0002048001D006820F07000616908431D49F3
:1035F000091D0860207800F01000102809D1194832
:10360000001D006820F4E060A16908431549091D08
:103610000860207800F02000202809D111480830E7
:10362000006820F07000E16908430E490831086025
:1036300000F066F80B49096801F470614FF480727C
:1036400092FAA2F2B2FA82F2D140074A515CC84023
:10365000064908600020FDF731FC0020F8E6000074
:103660000020005218440258E41001080000002411
:1036700010B5FEF7DBFE0949096801F00F010122D0
:1036800092FAA2F2B2FA82F2D140054A515CC840E5
:10369000044908600846006810BD0000184402583C
:1036A000E41001080400002410B5FFF7E1FF07490A
:1036B000096801F07001102292FAA2F2B2FA82F2C5
:1036C000D140034A515CC84010BD00001C44025860
:1036D000E410010810B5FFF7CBFF0749096801F4B2
:1036E000E0614FF4807292FAA2F2B2FA82F2D14013
:1036F000024A515CC84010BD1C440258E410010845
:1037000070B5012500EE905A00220121002300240B
:10371000DFED861AB0EE610ADFED841AB0EE611AB1
:103720000020834D2D6805F0380535B1082D15D0E2
:10373000102D15D0182D7CD114E07D4D103D2D6835
:10374000C5F3401545B17A4D103D2D68C5F3C1064E
:10375000784D25FA06F000E07648E5E07648E3E0AB
:103760007648E1E0724D18352D6805F00302704D82
:1037700018352D68C5F305116D4D1C352D6805F004
:1037800001036B4D24352D68C5F3CC0515FB03F5FE
:1037900001EE905AF8EE611AB0EE610A22B1012AE8
:1037A0004FD0022A7DD16BE0614D103D2D68C5F3ED
:1037B00040152DB35E4D103D2D68C5F3C1065D4D1E
:1037C00025FA06F4B4FBF1F501EE905AB8EE612A41
:1037D000DFED5B1AC0EE212A554D20352D68C5F36B
:1037E000080501EE905AF8EE611A72EEA11AF7EE92
:1037F000002A71EEA21A62EE211AB0EE611A1FE0E1
:103800004C4DB5FBF1F501EE905AB8EE612ADFEDB3
:103810004C1AC0EE212A464D20352D68C5F3080507
:1038200001EE905AF8EE611A72EEA11AF7EE002A34
:1038300000E077E071EEA21A62EE211AB0EE611A92
:103840005EE03D4DB5FBF1F501EE905AB8EE612A10
:10385000DFED3B1AC0EE212A354D20352D68C5F32A
:10386000080501EE905AF8EE611A72EEA11AF7EE11
:10387000002A71EEA21A62EE211AB0EE611A3FE040
:103880002E4DB5FBF1F501EE905AB8EE612ADFED51
:103890002C1AC0EE212A264D20352D68C5F30805C7
:1038A00000E00EE001EE905AF8EE611A72EEA11AF5
:1038B000F7EE002A71EEA21A62EE211AB0EE611A3A
:1038C0001EE01D4DB5FBF1F501EE905AF8EE612AB0
:1038D000DFED1B1A80EE212A154D20352D68C5F32A
:1038E000080501EE905AF8EE611A72EE211AB7EE51
:1038F000002A71EE821A62EEA11AB0EE611A00BFC0
:1039000000BF0B4D20352D68C5F346256D1C00EE1C
:10391000905AF8EE601A81EE212AFCEEC21A11EEDE
:10392000900A01E0044800BF00BF70BD0000000025
:10393000104402580090D00300093D0040787D01FA
:103940000000004670B504460025207800F0010014
:10395000002872D0F948006800F0380010280CD018
:10396000F648006800F03800182812D1F3481830E3
:10397000006800F0030002280BD1F04810380068FE
:10398000C0F3404000286DD0606800286AD1012053
:1039900070BD00BF6068B0F5803F08D1E7481038BF
:1039A000006840F48030E549103908602EE0606816
:1039B00068B9E2481038006820F48030DF491039D7
:1039C00008600846006820F4802008601EE06068F7
:1039D000B0F5A02F0DD1D9481038006840F48020F0
:1039E000D649103908600846006840F48030086005
:1039F0000CE0D2481038006820F48030CF491039EC
:103A000008600846006820F48020086000BF6068F5
:103A1000A0B1FDF733FA054608E0FDF72FFA401B89
:103A200041F28831884201D90320B1E7C3481038F8
:103A30000068C0F340400028EFD013E0FDF71EFA05
:103A4000054608E0FDF71AFA401B41F2883188422A
:103A500001D903209CE7B94810380068C0F3404002
:103A60000028EFD1207800F00200022847D1B348A7
:103A7000006800F0380058B1B048006800F0380025
:103A800018283ED1AD481830006800F00300B8BBDC
:103A9000AA4810380068C0F3800018B1E06808B97F
:103AA000012075E7A5481038006820F01900E1688A
:103AB0000843A24910390860FDF7E0F9054606E021
:103AC000FDF7DCF9401B022801D9032060E79B4881
:103AD00010380068C0F380000028F1D097480C38F7
:103AE000006820F47C304FF47C3292FAA2F2B2FAF1
:103AF00082F221699140084390490C3908604AE0FC
:103B0000FFE7E06868B38D481038006820F01900BE
:103B1000E1680843894910390860FDF7AFF90546A7
:103B200006E0FDF7ABF9401B022801D903202FE77F
:103B3000824810380068C0F380000028F1D07F4828
:103B40000C38006820F47C304FF47C3292FAA2F2F8
:103B5000B2FA82F221699140084378490C39086031
:103B600019E076481038006820F0010073491039D8
:103B70000860FDF783F9054606E0FDF77FF9401B75
:103B8000022801D9032003E76C4810380068C0F30D
:103B900080000028F1D1207800F01000102877D1A3
:103BA0006648006800F0380008280CD063480068B8
:103BB00000F03800182823D160481830006800F061
:103BC000030001281CD15D4810380068C0F30020B4
:103BD00020B1E069802801D00120D9E657480C388F
:103BE000006820F0F8404FF0F84292FAA2F2B2FAE0
:103BF00082F2216A9140084350490C39086047E03D
:103C0000E06958B34D481038006840F080004B49D7
:103C100010390860FDF732F9054606E0FDF72EF988
:103C2000401B022801D90320B2E64448103800683E
:103C3000C0F300200028F1D040480C38006820F084
:103C4000F8404FF0F84292FAA2F2B2FA82F2216AF8
:103C50009140084339490C39086019E03748103859
:103C6000006820F08000354910390860FDF706F93A
:103C7000054606E0FDF702F9401B022801D90320A2
:103C800086E62E4810380068C0F300200028F1D1E5
:103C9000207800F00800082836D16069D0B12748A4
:103CA0006430006840F00100244964310860FDF789
:103CB000E5F8054606E0FDF7E1F8401B022801D9CA
:103CC000032065E61D4864300068C0F3400000280A
:103CD000F1D019E019486430006820F0010017495C
:103CE00064310860FDF7CAF8054606E0FDF7C6F83E
:103CF000401B022801D903204AE6104864300068BE
:103D0000C0F340000028F1D1207800F020002028E6
:103D100034D1A069D8B109481038006840F4805007
:103D2000064910390860FDF7A9F8054608E0FDF7D7
:103D3000A5F8401B022803D9032029E610440258A5
:103D4000AF480068C0F340300028F0D016E0AC481F
:103D5000006820F48050AA490860FDF78FF80546F6
:103D600006E0FDF78BF8401B022801D903200FE67F
:103D7000A3480068C0F340300028F2D1207800F05A
:103D8000040004287DD19F48006840F480709D495C
:103D90000860FDF773F8054606E0FDF76FF8401B75
:103DA000642801D90320F3E59648006800F4807088
:103DB0000028F2D000BFA068012808D190487030D8
:103DC000006840F001008E49703108602DE0A06865
:103DD00068B98B487030006820F001008849703164
:103DE00008600846006820F0040008601DE0A06834
:103DF00005280DD182487030006840F004008049E9
:103E0000703108600846006840F0010008600CE06E
:103E10007B487030006820F00100794970310860FB
:103E20000846006820F00400086000BFA068A0B148
:103E3000FDF724F8054608E0FDF720F8401B41F2A5
:103E40008831884201D90320A2E56D4870300068AE
:103E5000C0F340000028EFD013E0FDF70FF805464F
:103E600008E0FDF70BF8401B41F28831884201D988
:103E700003208DE5624870300068C0F340000028E0
:103E8000EFD1606A00287CD05D481030006800F0F7
:103E90003800182876D0606A022874D15848006823
:103EA00020F0807056490860FCF7E8FF054606E000
:103EB000FCF7E4FF401B022801D9032068E55048C5
:103EC0000068C0F340600028F2D100BFD4E90A10B6
:103ED00041EA00104A492831096840F2F33291431F
:103EE0000843474928310860208E401EC0F308006F
:103EF000616B491E4FF47E4202EA41210843218F43
:103F0000491ED20102EA014108433C21095D491ED4
:103F1000120202EA0161084339493031086000BFEA
:103F2000081D00684FF6F87188434FF6F87292FA50
:103F3000A2F2B2FA82F2A16C9140084330493431C6
:103F400008602F482C30006820F00C00216C0843DA
:103F50002B492C3108600846006820F00200616C93
:103F6000084327492C3108600846006840F4803037
:103F700008600846006840F40030086008460068A1
:103F800002E03BE038E01FE040F480200860084693
:103F9000006840F0010008601948006840F0807037
:103FA00017490860FCF76AFF054606E0FCF766FF64
:103FB000401B022801D90320EAE411480068C0F33D
:103FC00040600028F2D019E00D48006820F08070B1
:103FD0000B490860FCF752FF054606E0FCF74EFF70
:103FE000401B022801D90320D2E405480068C0F331
:103FF00040600028F2D101E00120C9E40020C7E4BC
:10400000004402580048025870B504460D460CB9E9
:10401000012070BD94F82C0028B9002084F82D00F0
:10402000204600F019F8022084F82C00211D206899
:10403000FCF7EFFA2946D4E90002FCF73FFB0548FC
:10404000006840F0004003490860012084F82C001B
:104050000020DEE70040005210B586B0044600BFE5
:104060005A48006840F00200584908600846006855
:1040700000F00200009000BF00BF00BF534820388E
:10408000006840F4805051492039086008460068B3
:1040900000F48050009000BF00BF00BF4B481438B0
:1040A000006840F004004949143908600846006877
:1040B00000F00400009000BF00BF00BF0846006889
:1040C00040F0080008600846006800F00800009012
:1040D00000BF00BF00BF0846006840F01000086045
:1040E0000846006800F01000009000BF00BF00BF4D
:1040F0000846006840F0200008600846006800F0AC
:104100002000009000BF00BF00BF0846006840F0DC
:10411000400008600846006800F04000009000BFC2
:1041200000BF00BF0846006840F0800008600846F5
:10413000006800F08000009000BF00BF00BF08468C
:10414000006840F4807008600846006800F48070E1
:10415000009000BF00BF0D200190022002900120BE
:104160000390032004900C20059001A91848FCF747
:104170004DFD4CF20370019001A91648FCF746FD75
:104180004FF68370019001A91348FCF73FFD4FF6ED
:104190003F00019001A91148FCF738FD48F23710A3
:1041A000019001A90E48FCF731FD4FF47F400190CA
:1041B00001A90C48FCF72AFD40F2FF60019001A91B
:1041C0000948FCF723FD06B010BD0000F444025876
:1041D00000080258000C025800100258001402583F
:1041E00000180258001C02580020025870B50446FE
:1041F0000D4694F82C00022800D170BD022084F8EE
:104200002C0029462068FCF73EFA012084F82C0097
:104210000020F2E770B504460D46164694F82C00CF
:10422000022800D170BD022084F82C0032462946B5
:104230002068FCF72FFA2868022803D1052084F8AB
:104240002C0002E0012084F82C000020EAE70000A6
:1042500070B588B004460D46032084F83000A06B8A
:10426000032820D0B5F5004F04D1606B40F080509A
:1042700060631CE0B5F5804F07D1204607F0AEFE25
:104280000646606B3043606311E03DB9204607F09D
:1042900071FE0646606B3043606308E0606B40F07F
:1042A0000060606303E0606B40F080506063606BAF
:1042B00038B1194821688863012084F8300008B0BB
:1042C00070BD60680390A068049005952069069011
:1042D0006069042802D3606907900FE0A06DB0F513
:1042E000007F02D16069079008E0A06DB0F5807F83
:1042F00002D10220079001E004200790DDE90601C9
:10430000CDE90001206803A90EC907F053FA012086
:1043100084F830000020D2E7FF0FE01F10B50246FE
:10432000D06D800F0870D06DC0F383604870D06D81
:10433000C0F301608870D06D000CC870B2F85C00EA
:10434000000A087192F85C004871106E000DC88078
:10435000106EC0F3034008726020805AC0F3C03072
:1043600048726020805AC0F3803088726020805A82
:10437000C0F34030C8726020805AC0F30030087328
:1043800000204873906B002836D16020805A800549
:10439000030D506E43EA90700861506EC0F3C26026
:1043A0000875506EC0F302604875506EC0F34250FD
:1043B0008875506EC0F38240C875506EC0F3C2302D
:1043C00008760869401C90640B7E906C03F007032C
:1043D0009B1C01249C4060439064087A00F00F030A
:1043E00001209840D064D2E912035B0A584310655B
:1043F0004FF40073536521E0906B012813D16020C6
:10440000805C8006830A506E43EA104008610869A8
:10441000401C83029364936C13654FF40073D36460
:10442000D36C53650AE02E4813689863506B40F0D4
:1044300080505063012082F8300010BD6420805A03
:10444000C0F3803001F8190F6420805AC0F3C61001
:1044500048706420805C00F07F008870906EC00F10
:10446000C870906EC0F341700871906EC0F38260A6
:104470004871906EC0F383508871906EC0F34050C5
:10448000C87100200872906EC0F300404872682026
:10449000805AC0F3C03088726820805AC0F38030E0
:1044A000C8726820805AC0F3403008736820805A70
:1044B000C0F3003048736820805AC0F381208873AD
:1044C0006820805AC0F30120C8736820805CC0F364
:1044D000460008740120487419390020ADE7000037
:1044E000FF0FE01F0246906B0860D06B4860106CB5
:1044F0008860506CC860906C0861D06C4861106D29
:104500008861506DC86100207047F8B505460020ED
:1045100000906946284607F015FD064616B1686BFF
:10452000304368630098C0F343242046F8BD000080
:1045300070B590B005460C466946284607F068FC01
:10454000064656B1284829688863686B304368631B
:10455000012085F8300010B070BD0098C0F38110C4
:1045600020700098C0F340106070009800F47F0045
:10457000000A009940EA11606080019800060199E4
:1045800001F47F4140EA0120019901F47F0140EAF2
:104590001120019940EA116060600298207202982F
:1045A000000A60720298C0F30350A0720398C0B270
:1045B000029901F07F4140EA1140A0810398C0F3C5
:1045C0008520A0730398C0F30120E0730398C0F323
:1045D00003102074039800F00F0060740498000E1C
:1045E000A0740020B7E70000FF0FE01FF0B585B012
:1045F000044614B9012005B0F0BD94F8300020B98C
:1046000000202076204600F097F8032084F8300040
:10461000204600F055F808B10120ECE76946204635
:10462000FFF786FF08B10120E5E79DF810609DF8CF
:104630001170A06B012805D106B91FB14FF40071AC
:10464000A16507E0A06B012802D10102A16501E08C
:104650000021A1652046E168FFF7FAFD08B10120BD
:10466000C9E7A06DB0F5007F06D0A06DB0F5807FE2
:1046700002D0A06B012805D1204607F00FFA08B13F
:104680000120B8E7FCF7FAFB05460CE0FCF7F6FB67
:10469000401B401C38B94FF000406063012084F893
:1046A00030000320A7E72046FFF72FFF0428EDD1B5
:1046B00000206063E062012084F8300000209AE767
:1046C00070B588B0044600200390049005900690D1
:1046D000FA200790DDE90601CDE90001206803A971
:1046E0000EC907F067F8064616B1012008B070BD84
:1046F000206807F079F806460EB10120F6E720465B
:1047000007F000FB05463DB1012084F83000606BE6
:10471000284360630120E9E7204607F07DFA05465B
:104720003DB1012084F83000606B284360630120B4
:10473000DCE70020DAE7000010B586B0044600BFD1
:104740002048006840F480301E4908600846006830
:1047500000F48030009000BF00BF00BF19480C304B
:10476000006840F0040017490C31086008460068F2
:1047700000F00400009000BF00BF00BF08460068C2
:1047800040F0080008600846006800F0080000904B
:1047900000BF00BF4FF4F8500190022002900120AA
:1047A0000390032004900C20059001A90648FCF713
:1047B0002DFA0420019001A90448FCF727FA06B05D
:1047C00010BD0000D444025800080258000C0258E2
:1047D0002DE9F04F89B00446894693469846FCF788
:1047E0004DFB0290DA464D46B9F1000F07D1606BE0
:1047F00040F000606063012009B0BDE8F08F94F8DC
:10480000300001287ED1002060630AEB0801206D92
:10481000814205D9606B40F0007060630120EBE7D6
:10482000032084F8300000202168C862A06B0128B2
:1048300001D04FEA4A2A4FF40071206806F0CFFBFE
:1048400006464EB16B4821688863606B30436063F5
:10485000012084F83000CFE74FF0FF3003904FEA9B
:104860004820049090200590022006900020079098
:10487000089003A9206806F09CFD2068C06840F0FD
:1048800040002168C860B8F1010F07D90220E0623A
:104890005146206806F00CFC064606E00120E06266
:1048A0005146206806F021FC06464EB15148216869
:1048B0008863606B30436063012084F830009BE7BD
:1048C00033E02068406B00F40040B8B10020019054
:1048D00011E0206806F093FF07462F706D1C380A20
:1048E00028706D1C380C28706D1C380E28706D1CDB
:1048F0000198401C019001980828EAD3FCF7BEFA01
:10490000029900E06FE0411A1298814201D2129898
:1049100058B9384821688863606B40F00040606394
:10492000012084F83000032066E72068406B00F423
:1049300095700028C5D02068C06820F0400021682C
:10494000C8602068406B00F48070A0B1B8F1010F1E
:1049500011D9A06B03280ED0206806F0A9FC0646EA
:104960004EB1244821688863606B30436063012046
:1049700084F8300040E72068406B00F0080050B138
:104980001C4821688863606B40F008006063012068
:1049900084F8300030E72068406B00F0020050B12E
:1049A000144821688863606B40F002006063012056
:1049B00084F8300020E72068406B00F0200050B100
:1049C0000C4821688863606B40F020006063012020
:1049D00084F8300010E7084821688863012084F8D3
:1049E0003000002008E7606B40F000506063012059
:1049F00002E70000FF0FE01F3A0F00182DE9F04F0B
:104A000089B00446884692461F46DDF848B0FCF758
:104A100035FA0290D1464646B8F1000F07D1606BD7
:104A200040F000606063012009B0BDE8F08F94F8A9
:104A3000300001287ED10020606309EB0701206D62
:104A4000814205D9606B40F0007060630120EBE7A4
:104A5000032084F8300000202168C862A06B012880
:104A600001D04FEA49294FF40071206806F0B7FAE7
:104A700005464DB16D4821688863606B28436063CB
:104A8000012084F83000CFE74FF0FF300390780228
:104A9000049090200590002006900790089003A9AC
:104AA000206806F086FC2068C06840F0400021685D
:104AB000C860012F07D92020E0624946206806F02F
:104AC0003EFC054606E01020E0624946206806F0FC
:104AD00053FC05464DB1554821688863606B2843F7
:104AE0006063012084F830009EE73CE02068406B62
:104AF00000F4804018B3002001901DE03078009051
:104B0000761C3078009941EA00200090761C3078BD
:104B1000009941EA00400090761C3078009941EA03
:104B200000600090761C6946206806F083FE0198BC
:104B3000401C00E074E0019001980828DED3FCF7E7
:104B40009DF90299401A584502D2BBF1000F0AD1D3
:104B5000364821688863606B28436063012084F8CD
:104B60003000032060E72068406B00F48D7000285F
:104B7000BCD02068C06820F040002168C860206870
:104B8000406B00F4807098B1012F11D9A06B0328FD
:104B90000ED0206806F08CFB05464DB123482168F5
:104BA0008863606B28436063012084F830003BE732
:104BB0002068406B00F0080050B11C4821688863F1
:104BC000606B40F008006063012084F830002BE740
:104BD0002068406B00F0020050B1144821688863DF
:104BE000606B40F002006063012084F830001BE736
:104BF0002068406B00F0100050B10C4821688863B9
:104C0000606B40F010006063012084F830000BE717
:104C1000074821688863012084F83000002003E7FA
:104C2000606B40F0005060630120FDE6FF0FE01F65
:104C30003A0F001870B50446002500260CB9012073
:104C400070BD606A00B900BFA06AB0F5800F00D1E6
:104C500000BF8E49206888420CD08D492068884268
:104C600008D08C492068884204D0E0680F2801D918
:104C70000120E5E7204607F0F5FA0646834920685B
:104C8000884209D082492068884205D0814920683D
:104C9000884201D0082E0DD87C492068884207D070
:104CA0007B492068884203D07A492068884203D132
:104CB000102E01D90120C3E7A06AB0F5800F1DD1E5
:104CC0007249206888420DD071492068884209D015
:104CD00070492068884205D0206BB0F5702F01D94B
:104CE0000120ADE7206B10B9A089050400E0256B19
:104CF000E068B0EB154F01D90120A1E794F88100DD
:104D000028B9002084F88000204600F0C5F8022071
:104D100084F881002068006820F0010021680860A4
:104D2000A069B0F1806F0BD16068B0F5800F07D13A
:104D3000A06B28B92068006840F4805021680860A2
:104D4000A16AE06908432843E16B0843E16808432E
:104D500021688860616A606B0843A16B0843A169A0
:104D600008432169084361690843216A084361686F
:104D70000843E16C0843A1680843A16C0843A16D96
:104D800008432168C860A06AB0F5800F4DD1206C3F
:104D9000012806D12068006840F4004021680860BE
:104DA00005E02068006820F4004021680860606C1D
:104DB000012806D12068006840F48040216808601E
:104DC00005E02068006820F48040216808602F49D1
:104DD000206888420AD02E492068884206D02D4992
:104DE0002068884202D0B5F5702F0ED02749206880
:104DF000884207D026492068884203D02549206888
:104E0000884209D1B5F5F81F06D12068006840F442
:104E100000502168086005E02068006820F4005018
:104E2000216808602168E06A0864606888B9A06A3F
:104E300038B92068806820F4C05040F400602168D0
:104E400088602068806820F4C06040F48060216839
:104E500088602068006D20F00100216808656068A6
:104E600000F48000B0F5800F07D12068C06820F002
:104E70000040616D08432168C8600020C4F88400C8
:104E8000012084F881000020DAE6000000300140B3
:104E900000380040003C004010B5B6B0044600BFEA
:104EA0001A48006840F00200184908600846006887
:104EB00000F00200019000BF00BF00BF134808309F
:104EC000006840F4804011490831086008460068D5
:104ED00000F48040019000BF00BF4FF4805002906A
:104EE0000020199002A8FDF7FFFC4FF460403190BC
:104EF0000220329001203390032034900520359019
:104F000031A90348FBF782FE36B010BDE0440258D9
:104F1000000402582DE9F84F0446884691461D4684
:104F20000A9E0027BA4600BF94F88000012802D1EB
:104F30000220BDE8F88F012084F8800000BFFBF755
:104F40009DFF074694F88100012812D06068B0F5F3
:104F5000800F05D1A06818B994F88100042808D002
:104F60004FF0020A00BF002084F8800000BF5046C6
:104F7000DFE7B8F1000F03D0B9F1000F00D045B959
:104F80004FF0010A00BF002084F8800000BF5046A7
:104F9000CFE794F88100042802D0052084F881002E
:104FA0000020C4F88400C4F86490A4F86A50A4F8FF
:104FB0006850C4F85C80A4F86250A4F86050206780
:104FC0006067206840686FF30F00284321684860DD
:104FD0002068006840F00100216808606068B0F552
:104FE000800F05D12068006840F4007021680860D7
:104FF000E0680F284CD942E0B4F8620088B120681C
:10500000406900F0020002280BD1E06D00682168C1
:105010000862E06D001DE065B4F86200401EA4F86F
:105020006200B4F86A0088B12068406948F208015B
:10503000084058B12068006B616E0860606E001D0A
:105040006066B4F86A00401EA4F86A00701CB0B133
:10505000FBF714FFC01BB04211D3204607F084F8C1
:1050600000BF002084F8800000BFD4F8840040F422
:105070008070C4F88400012084F8810059E7B4F8F6
:1050800062000028B8D1B4F86A000028B4D10FE15A
:10509000E068072871D966E0B4F8620020B32068A0
:1050A000406900F0020002281ED1B4F86200012815
:1050B0000ED9E06B60B1E06D006821680862E06DB8
:1050C000001DE065B4F86200801EA4F862000BE0E9
:1050D000E06D008821680884E06D801CE065B4F80C
:1050E0006200401EA4F86200B4F86A0010B32068A1
:1050F000406900F46040E8B12068406900F4004075
:1051000060B12068006B616E0860606E001D6066B3
:10511000B4F86A00801EA4F86A000BE02068008ED4
:10512000616E0880606E801C6066B4F86A00401E84
:10513000A4F86A00701CB0B1FBF7A0FEC01BB0421F
:1051400011D3204607F010F800BF002084F880003B
:1051500000BFD4F8840040F48070C4F884000120BB
:1051600084F88100E5E6B4F86200002894D1B4F830
:105170006A00002890D19BE0FFE790E0B4F862005D
:1051800058B32068406900F00200022833D1B4F817
:10519000620003280FD9E06B40280CD9E06D00684D
:1051A00021680862E06D001DE065B4F86200001F30
:1051B000A4F862001FE0B4F8620001280ED9E06B89
:1051C00060B1E06D008821680884E06D801CE065B6
:1051D000B4F86200801EA4F862000CE0E06D007874
:1051E000216881F82000E06D401CE065B4F86200A1
:1051F000401EA4F86200B4F86A0048B32068406911
:1052000000F4604020B32068406900F4004060B1C1
:105210002068006B616E0860606E001D6066B4F807
:105220006A00001FA4F86A0020E02068406900F4CA
:10523000C040B0F5005F0CD92068008E616E088018
:10524000606E801C6066B4F86A00801EA4F86A0074
:105250000CE0206890F83000616E0870606E401CB1
:105260006066B4F86A00401EA4F86A00701CB0B111
:10527000FBF704FEC01BB04211D3204606F074FFBA
:1052800000BF002084F8800000BFD4F8840040F400
:105290008070C4F88400012084F8810049E6B4F8E5
:1052A000620000287FF46AAFB4F86A000028F9D1E0
:1052B0003B46002208212046009606F0E0FF28B178
:1052C000D4F8840040F02000C4F88400204606F0A2
:1052D0004BFF00BF002084F8800000BF012084F84D
:1052E0008100D4F8840008B1012022E6002020E6E5
:1052F00070B504460E4615460CB9012070BD94F8F1
:10530000450028B9002084F84400204600F024F825
:1053100004F108012068FBF70DF93146A268206806
:10532000FBF748F92946E36AD4E90102FBF7DEF806
:10533000A168206850F8210040F00100A2682168AF
:1053400041F822000348006840F00040014908602D
:105350000020D3E70040005210B586B0044600BFDD
:105360002048006840F480501E49086008460068E4
:1053700000F48050009000BF00BF00BF19480C30FF
:10538000006840F0080017490C31086008460068C2
:1053900000F00800009000BF00BF00BF0846006892
:1053A00040F0100008600846006800F0100000900F
:1053B00000BF00BF4EF2B3700190022002900120A6
:1053C0000390032004900C20059001A90648FBF7E8
:1053D0001DFC4FF68070019001A90448FBF716FCF4
:1053E00006B010BDD4440258000C025800100258F8
:1053F000042808D14FF0E021096941F004014FF081
:10540000E022116107E04FF0E021096921F0040179
:105410004FF0E0221161704770B504462546681EC2
:10542000B0F1807F01D301200FE0681E4FF0E02132
:1054300048610F214FF0FF3009F0BCFF00204FF012
:10544000E021886107200861002070BD10B5044686
:105450000CB9012010BD94F83D0028B9002084F853
:105460003C00204600F00CF8022084F83D00211D8D
:10547000206807F0CFF8012084F83D000020E9E71C
:10548000704701460868C06840F001000A68D060B3
:105490000868008840F001000A681080002070470A
:1054A0007047704701460022002391F8792091F857
:1054B0007A3042EA030070472DE9F0410446206843
:1054C000C569206807682068866805F00F08B8F18C
:1054D000000F0DD105F0200050B107F0200010B9E9
:1054E00006F0805020B1204607F003FABDE8F081B5
:1054F000B8F1000F72D05D48304018B907F49070D1
:1055000000287AD005F0010048B107F4807030B16E
:10551000012021680862E06F40F00100E06705F0BB
:10552000020048B106F0010030B102202168086293
:10553000E06F40F00400E06705F0040048B106F0B9
:10554000010030B1042021680862E06F40F00200E1
:10555000E06705F0080078B107F0200028B906F0F0
:10556000805010B906F0010030B1082021680862AF
:10557000E06F40F00800E067E06F70B305F02000D6
:1055800040B107F0200010B906F0805010B120465D
:1055900007F0AFF9E06F00F0080020B920688068DC
:1055A00000F0400018B3204607F083F920688068B7
:1055B00000F04000B8B12068806820F04000216809
:1055C0008860606F58B12A48616F0865606FFBF7AB
:1055D00083FA10B1606F016D88470DE00DE0204641
:1055E000FFF75FFF08E02046FFF75BFF04E020467F
:1055F000FFF757FF0020E06778E705F4801078B1E7
:1056000006F4800060B14FF4801021680862202009
:1056100084F8790084F87A002046FFF741FF65E7B7
:1056200005F0800048B107F0800010B906F40000D2
:1056300018B1204607F074FE58E705F0400030B17D
:1056400007F0400018B1204607F043F94EE705F493
:10565000000040B107F0804028B12068006820F0C9
:1056600080402168086000BF40E700000100001092
:105670009BC8000810B504460CB9012010BDA069F4
:1056800000B100E000BF94F8790028B9002084F848
:105690007800204600F02AF8242084F87900206859
:1056A000006820F0010021680860204607F066F9D4
:1056B000012800D1E2E7606B10B1204607F03EF808
:1056C0002068406820F49040216848602068806825
:1056D00020F02A00216888602068006840F00100FE
:1056E00021680860204607F09EF8C7E710B586B02D
:1056F00004462149206888423BD100BF1F4800680A
:1057000040F001001D4908600846006800F00100F3
:10571000009000BF00BF00BF18481030006840F084
:1057200010001649103108600846006800F01000AB
:10573000009000BF00BF4FF4007001900220029063
:1057400001200390022004900720059001A90C4835
:10575000FBF75CFA4FF48060019001A90848FBF761
:1057600055FA2520FBF780FE032211462520FBF782
:105770008BFE06B010BD000000100140E04402584E
:105780000000025810B5034693F87A00202867D12C
:1057900001B10AB9012010BD00BF93F878000128BB
:1057A00001D10220F7E7012083F8780000BF596695
:1057B000A3F86820A3F86A2000BF9868B0F5805F5E
:1057C0000AD1186920B940F2FF10A3F86C001CE060
:1057D000FF20A3F86C0018E0986848B9186918B958
:1057E000FF20A3F86C0010E07F20A3F86C000CE011
:1057F0009868B0F1805F08D1186918B97F20A3F8C4
:105800006C0002E03F20A3F86C0000BF0020D867C6
:10581000222083F87A0000BF002083F8780000BFC0
:105820001868806840F001001C68A0601868006873
:1058300000F0005060B11868006840F480701C6887
:1058400020601868806840F080501C68A06005E007
:105850001868006840F490701C68206000209AE787
:10586000022098E71D4A0168914236D11C490988F7
:1058700001F4004189BB1A49098801F4804171B1E2
:10588000184909780A2903D00021154A118024E01B
:105890001349098841F40041114A11801DE0114962
:1058A00009780D2906D10E49098841F480410C4A36
:1058B000118012E00B490978094A1288C2F30D02DF
:1058C000094B995406490988491C054A118011461B
:1058D0000988C72901DD00211180704700100140AF
:1058E0001000002412000024FC040024704700BFB4
:1058F000FEE7000010B5002210211248FBF7B8FAAD
:105900001048006820F440600E49086008460068AE
:1059100040F480600860002220210A48FBF7A8FAC2
:10592000022009F0B3FF012210210648FBF7A0FA7C
:10593000022009F0ABFF002210210248FBF798FA81
:1059400010BD0000001C025810B5002210211248A2
:10595000FBF78EFA1048006820F440600E4908609A
:105960000846006840F480600860012220210A484F
:10597000FBF77EFA022009F089FF01221021064878
:10598000FBF776FA022009F081FF0022102102487D
:10599000FBF76EFA10BD0000001C025870B50546FA
:1059A00000241848006820F4406016490860084642
:1059B0000068086000261AE0002210211148FBF759
:1059C00057FA022009F062FF012210210D48FBF76F
:1059D0004FFA6006040E20210A48FBF73DFA08B191
:1059E000601CC4B2012009F051FF701CC6B2082E21
:1059F000E2DB15B9FFF7A8FF01E0FFF77BFF2046C8
:105A000070BD0000001C025870B504461C480068B8
:105A100020F440601A4908600846006840F480603D
:105A20000860002210211648FBF722FA002523E027
:105A3000E00928B1012220211148FBF719FA04E0FE
:105A4000002220210E48FBF713FA6006040E022004
:105A500009F01CFF012210210948FBF709FA022076
:105A600009F014FF002210210548FBF701FA02207B
:105A700009F00CFF681CC5B2082DD9DB70BD000011
:105A8000001C025810B51348006820F4406011490A
:105A900008600846006840F4806008600122202108
:105AA0000C48FBF7E5F9012210210A48FBF7E0F961
:105AB000042009F0EBFE002220210648FBF7D8F96C
:105AC000042009F0E3FE002210210248FBF7D0F980
:105AD00010BD0000001C025810B51348006820F4E7
:105AE0004060114908600846006840F48060086022
:105AF000002210210C48FBF7BBF9002220210A48A4
:105B0000FBF7B6F9042009F0C1FE01221021064876
:105B1000FBF7AEF9012220210348FBF7A9F9042085
:105B200009F0B4FE10BD0000001C025810B500249E
:105B30001748006820F4406015490860084600686E
:105B40000860012220211248FBF792F9012009F098
:105B50009DFE012210210E48FBF78AF9012009F071
:105B600095FE07E0601CC4B2FA2C03DDFFF7B4FF1A
:105B7000012010BD20210648FBF76EF90028F1D165
:105B8000002210210248FBF773F90020F1E7000022
:105B9000001C025830B50B46002100BF16E00A2455
:105BA000B4EB107F05D9302404EB107403F81140D6
:105BB00005E0412404EB10740A3C03F81140000195
:105BC00000254C00641C1D554C1CE1B29142E6DBE3
:105BD00030BD000000B587B000BF2448006840F029
:105BE0000100224908600846006800F001000190A9
:105BF00000BF00BF00BF0846006840F00400086016
:105C00000846006800F00400019000BF00BF00BF1C
:105C10000846006840F0800008600846006800F010
:105C20008000019000BF00BF01200290002003907F
:105C3000022004900320059002A90D48FAF7E6FF20
:105C40004FF40050029000200390012004900320A4
:105C5000059002A90748FAF7D9FF0C20029002A983
:105C60000548FAF7D3FF07B000BD0000E044025832
:105C70000000025800080258001C025870B5044683
:105C800000260D4805880D48006818B1204602F02E
:105C900081FF0FE00848408845430021084602F094
:105CA0006BFD02F039FF002602E005490C80761CEE
:105CB000AE42FAD370BD0000C4060024DC07002405
:105CC0000000086010B504465C4884715C480068B8
:105CD00050B1204602F088FF5948C08A57490880D1
:105CE0005748008B488010BD002C51D1F0205349FB
:105CF00008804FF4A07048800846808849F24131FE
:105D0000884205D04D48808845F21031884214D130
:105D10002C204A4908812A2048812B208881084666
:105D2000808845F21031884206D14FF4A070434973
:105D300008804FF4F07048807BE04048808845F24E
:105D40001051884210D14FF430503C4908814FF433
:105D5000285048814FF42C5088814FF4F07008800F
:105D60004FF44870488064E03448808841F66311FD
:105D700088425ED12C20314908812B2048812A207D
:105D800088814FF4F07008804FF44870488050E0EC
:105D90004FF4A07029490880F02048800846808888
:105DA00049F24131884205D02448808845F21031BB
:105DB000884207D12C20214908812A2048812B20A4
:105DC000888129E01D48808845F21051884210D111
:105DD0004FF43050194908814FF4285048814FF44E
:105DE0002C5088814FF4487008804FF4F070488040
:105DF00012E01248808841F6631188420CD12C20B1
:105E00000E4908812A2048812B2088814FF4487050
:105E100008804FF4F07048800848808845F21031BF
:105E2000884206D14FF4F070044908804FF4A07006
:105E30004880002002F066FB00BF54E7C40600243F
:105E4000DC07002470B504460D461646434800683A
:105E500028B132462946204602F0DCFE70BD40489B
:105E6000808849F24131884205D03D48808845F21A
:105E70001031884214D13A49488902F041FE20127B
:105E800002F032FEE0B202F02FFE3549888902F0BE
:105E900037FE281202F028FEE8B202F025FE54E098
:105EA0002F48808845F21051884220D12C494889DA
:105EB00002F026FE201202F017FE29494989491CEA
:105EC00088B202F01DFEE0B202F00EFE244988897D
:105ED00002F016FE281202F007FE21498989491CAA
:105EE00088B202F00DFEE8B202F0FEFD2DE01C4883
:105EF000808841F66311884227D11948807920B9FA
:105F000017480088401E001B84B21549488902F0DA
:105F1000F7FD201202F0E8FDE0B202F0E5FD2012EC
:105F200002F0E2FDE0B202F0DFFD0D49888902F0E7
:105F3000E7FD281202F0D8FDE8B202F0D5FD2812E4
:105F400002F0D2FDE8B202F0CFFD05480089054914
:105F50000880891C0E8000BF80E70000DC07002459
:105F6000C4060024FEFF07602DE9F84F05460E46E3
:105F700017469846DDF828904FF0000B144800684B
:105F800040B143463A4631462846CDF8009002F0EB
:105F900069FE1BE0781B401C1FFA80FB344613E0AF
:105FA0002146284602F0E8FB02F0B6FD4FF0000A59
:105FB00006E00849A1F800900AF101001FFA80FAF2
:105FC000DA45F6DB601C84B24445E9DDBDE8F88FB4
:105FD000DC0700240000086000B595B003F03AF932
:105FE000FE4988800846808818B102F0DFFE02F082
:105FF000E4B900BFFA48006840F00200F8490860C0
:106000000846006800F00200019000BF00BF202099
:1060100010900120119012900320139010A9F148C4
:10602000FAF7F4FD02F00AFAEF48F0490860F04888
:106030004860002088600021EC48C16001611021A7
:10604000416100218161C16101624FF4805141626F
:10605000002181624FF48041C162002101634163EC
:106060004FF4801181631120099000200A9055207F
:106070000B9000200F901520029000200390152017
:1060800004900020089002AA09A9D848FFF730F927
:10609000322009F0EFFBD32002F032FD02F000FACB
:1060A000CE49888002F0FCF9CC49888002F0F8F9EA
:1060B000CA498880084680884FF6FF7101EA0020AF
:1060C000C649888002F0ECF9C44989880843C3496D
:1060D00088800846808849F24131884278D0D420AF
:1060E00002F00EFD02F0DCF9BC49888002F0D8F91C
:1060F000BA49888002F0D4F9B84988800846808877
:106100004FF6FF7101EA0020B449888002F0C8F917
:10611000B24989880843B14988800846808845F299
:106120001031884254D04FF45A4002F0E9FC02F09A
:10613000B7F9AA4988804FF45B4002F0E1FC02F015
:10614000AFF9A6498880084680884FF6FF7101EABA
:106150000020A24988804FF45C4002F0D1FC02F09C
:106160009FF99E49898808439C4988800846808811
:10617000B0F5004F02D145F21050888097488088D2
:1061800045F21051884223D0A12002F0B9FC02F060
:1061900087F99249888002F083F9904988800846FF
:1061A00080884FF6FF7101EA00208C49888002F058
:1061B00077F98A4989880843884988800846808811
:1061C00045F26171884203D141F6631083498880AA
:1061D0008248808849F2413188427CD1CF2002F048
:1061E0008FFC002002F080FCC12002F07DFC3020FA
:1061F00002F07AFCED2002F083FC642002F074FCD3
:10620000032002F071FC122002F06EFC812002F0EB
:106210006BFCE82002F074FC852002F065FC102085
:1062200002F062FC7A2002F05FFCCB2002F068FCF6
:10623000392002F059FC2C2002F056FC002002F01C
:1062400053FC342002F050FC022002F04DFCF720F9
:1062500002F056FC202002F047FCEA2002F050FC3D
:10626000002002F041FC002002F03EFCC02002F0C1
:1062700047FC1B2002F038FCC12002F041FC012049
:1062800002F032FCC52002F03BFC302002F02CFC76
:10629000302002F029FCC72002F032FCB72002F0C7
:1062A00023FC362002F02CFC482002F01DFC3A2092
:1062B00002F026FC552002F017FCB12002F020FC71
:1062C000002002F011FC1A2002F00EFCB62002F0B1
:1062D00017FC0A2000E0A5E002F006FCA22002F074
:1062E00003FCF22002F00CFC002002F0FDFB262053
:1062F00002F006FC012002F0F7FBE02002F000FCB7
:106300000F2002F0F1FB2A2002F0EEFB282002F021
:10631000EBFB082002F0E8FB0E2002F0E5FB082072
:1063200002F0E2FB542002F0DFFBA92002F0DCFBCC
:10633000432002F0D9FB0A2002F0D6FB0F2002F026
:10634000D3FB002002F0D0FB002002F0CDFB0020A8
:1063500002F0CAFB002002F0C7FBE12002F0D0FBF4
:10636000002002F0C1FB152002F0BEFB172002F056
:10637000BBFB072002F0B8FB112002F0B5FB0620A2
:1063800002F0B2FB2B2002F0AFFB562002F0ACFB78
:106390003C2002F0A9FB052002F0A6FB102002F031
:1063A000A3FB0F2002F0A0FB3F2002F09DFB3F204B
:1063B00002F09AFB0F2002F097FB2B2002F0A0FBCB
:1063C000002002F091FB002002F08EFB012002F081
:1063D0008BFB3F2002F088FB2A200BE0C406002440
:1063E000E04402580004025800400052780600249D
:1063F0000441005202F084FB002002F075FB0020F3
:1064000002F072FB002002F06FFBEF2002F06CFB49
:10641000112002F075FB782009F02CFA292002F0F7
:106420006FFBE4E5FE48808845F21031884240F079
:106430007C87ED2002F064FB012002F055FBFE207A
:1064400002F052FBEE2002F05BFBDE2002F04CFB80
:10645000212002F049FBF12002F052FB012002F062
:1064600043FBDF2002F04CFB102002F03DFBC42078
:1064700002F046FB8F2002F037FBC62002F040FB03
:10648000002002F031FBE22002F02EFBE22002F0BD
:106490002BFBE22002F028FBBF2002F031FBAA20F8
:1064A00002F022FBB02002F02BFB0D2002F01CFBBF
:1064B000002002F019FB0D2002F016FB002002F074
:1064C00013FB112002F010FB002002F00DFB19203D
:1064D00002F00AFB002002F007FB212002F004FB7F
:1064E000002002F001FB2D2002F0FEFA002002F055
:1064F000FBFA3D2002F0F8FA002002F0F5FA5D20E8
:1065000002F0F2FA002002F0EFFA5D2002F0ECFA5D
:10651000002002F0E9FAB12002F0F2FA802002F045
:10652000E3FA002002F0E0FA8B2002F0DDFA00200E
:1065300002F0DAFA962002F0D7FA002002F0D4FA3C
:10654000B22002F0DDFA002002F0CEFA002002F0C4
:10655000CBFA022002F0C8FA002002F0C5FA0320AC
:1065600002F0C2FA002002F0BFFAB32002F0C8FA2B
:10657000002002F0B9FA002002F0B6FA002002F082
:10658000B3FA002002F0B0FA002002F0ADFA0020C9
:1065900002F0AAFA002002F0A7FA002002F0A4FA02
:1065A000002002F0A1FA002002F09EFA002002F082
:1065B0009BFA002002F098FA002002F095FA0020E1
:1065C00002F092FA002002F08FFA002002F08CFA1A
:1065D000002002F089FA002002F086FA002002F082
:1065E00083FA002002F080FA002002F07DFA0020F9
:1065F00002F07AFA002002F077FA002002F074FA32
:10660000B42002F07DFA8B2002F06EFA002002F036
:106610006BFA962002F068FA002002F065FAA120D9
:1066200002F062FA002002F05FFAB52002F068FA88
:10663000022002F059FA002002F056FA032002F07C
:1066400053FA002002F050FA042002F04DFA002024
:1066500002F04AFAB62002F053FA002002F044FA9F
:10666000002002F041FAB72002F04AFA002002F0BE
:106670003BFA002002F038FA3F2002F035FA002001
:1066800002F032FA5E2002F02FFA002002F02CFA1B
:10669000642002F029FA002002F026FA8C2002F091
:1066A00023FA002002F020FAAC2002F01DFA0020AC
:1066B00002F01AFADC2002F017FA002002F014FAB5
:1066C000702002F011FA002002F00EFA902002F081
:1066D0000BFA002002F008FAEB2002F005FA002085
:1066E00002F002FADC2002F0FFF9002002F0FCF9CF
:1066F000B82002F005FA002002F0F6F9002002F0BE
:10670000F3F9002002F0F0F9002002F0EDF900208A
:1067100002F0EAF9002002F0E7F9002002F0E4F9C3
:10672000002002F0E1F9BA2002F0EAF9242002F098
:10673000DBF9002002F0D8F9002002F0D5F90020A2
:1067400002F0D2F9C12002F0DBF9202002F0CCF9EE
:10675000002002F0C9F9542002F0C6F9002002F02E
:10676000C3F9FF2002F0C0F9002002F0BDF9C220F9
:1067700002F0C6F90A2002F0B7F9002002F0B4F9DD
:10678000042002F0B1F9002002F0AEF9C32002F0BB
:10679000B7F93C2002F0A8F9002002F0A5F93A2050
:1067A00002F0A2F9002002F09FF9392002F09CF9D2
:1067B000002002F099F9372002F096F9002002F04B
:1067C00093F93C2002F090F9002002F08DF9362078
:1067D00002F08AF9002002F087F9322002F084F9F1
:1067E000002002F081F92F2002F07EF9002002F053
:1067F0007BF92C2002F078F9002002F075F92920AD
:1068000002F072F9002002F06FF9262002F06CF914
:10681000002002F069F9242002F066F9002001E06E
:10682000C406002402F060F9242002F05DF9002083
:1068300002F05AF9232002F057F9002002F054F92F
:106840003C2002F051F9002002F04EF9362002F00F
:106850004BF9002002F048F9322002F045F90020FF
:1068600002F042F92F2002F03FF9002002F03CF93B
:106870002C2002F039F9002002F036F9292002F02C
:1068800033F9002002F030F9262002F02DF9002023
:1068900002F02AF9242002F027F9002002F024F95E
:1068A000242002F021F9002002F01EF9232002F03A
:1068B0001BF9002002F018F9C42002F021F962202F
:1068C00002F012F9002002F00FF9052002F00CF995
:1068D000002002F009F9842002F006F9002002F0FD
:1068E00003F9F02002F000F9002002F0FDF8182072
:1068F00002F0FAF8002002F0F7F8A42002F0F4F811
:10690000002002F0F1F8182002F0EEF8002002F06A
:10691000EBF8502002F0E8F8002002F0E5F80C2037
:1069200002F0E2F8002002F0DFF8172002F0DCF8B5
:10693000002002F0D9F8952002F0D6F8002002F0ED
:10694000D3F8F32002F0D0F8002002F0CDF8E620D2
:1069500002F0CAF8002002F0C7F8C52002F0D0F813
:10696000322002F0C1F8002002F0BEF8442002F00C
:10697000BBF8002002F0B8F8652002F0B5F800205E
:1069800002F0B2F8762002F0AFF8002002F0ACF886
:10699000882002F0A9F8002002F0A6F8C62002F034
:1069A000AFF8202002F0A0F8002002F09DF8172098
:1069B00002F09AF8002002F097F8012002F094F813
:1069C000002002F091F8C72002F09AF8002002F0AF
:1069D0008BF8002002F088F8002002F085F80020F3
:1069E00002F082F8C82002F08BF8002002F07CF858
:1069F000002002F079F8002002F076F8002002F082
:106A000073F8C92002F07CF8002002F06DF8002035
:106A100002F06AF8002002F067F8002002F064F843
:106A2000002002F061F8002002F05EF8002002F081
:106A30005BF8002002F058F8002002F055F8002022
:106A400002F052F8002002F04FF8002002F04CF85B
:106A5000002002F049F8002002F046F8002002F081
:106A600043F8002002F040F8E02002F049F8162038
:106A700002F03AF8002002F037F81C2002F034F857
:106A8000002002F031F8212002F02EF8002002F060
:106A90002BF8362002F028F8002002F025F84620D6
:106AA00002F022F8002002F01FF8522002F01CF839
:106AB000002002F019F8642002F016F8002002F01D
:106AC00013F87A2002F010F8002002F00DF88B2065
:106AD00002F00AF8002002F007F8992002F004F80A
:106AE000002002F001F8A82001F0FEFF002001F0D4
:106AF000FBFFB92001F0F8FF002001F0F5FFC420F2
:106B000001F0F2FF002001F0EFFFCA2001F0ECFFDE
:106B1000002001F0E9FFD22001F0E6FF002001F0A3
:106B2000E3FFD92001F0E0FF002001F0DDFFE020CD
:106B300001F0DAFF002001F0D7FFF32001F0D4FFCD
:106B4000002001F0D1FFE12001F0DAFF162001F072
:106B5000CBFF002001F0C8FF1C2001F0C5FF002082
:106B600001F0C2FF222001F0BFFF002001F0BCFFB6
:106B7000362001F0B9FF002001F0B6FF452001F0FA
:106B8000B3FF002001F0B0FF522001F0ADFF002064
:106B900001F0AAFF642001F0A7FF002001F0A4FF8C
:106BA0007A2001F0A1FF002001F09EFF8B2001F070
:106BB0009BFF002001F098FF992001F095FF002035
:106BC00001F092FFA82001F08FFF002001F08CFF60
:106BD000B92001F089FF002001F086FFC42001F0F8
:106BE00083FF002001F080FFCA2001F07DFF00201C
:106BF00001F07AFFD22001F077FF002001F074FF4E
:106C0000D82001F071FF002001F06EFFE02001F0BC
:106C10006BFF002001F068FFF32001F065FF00200A
:106C200001F062FFE22001F06BFF052001F05CFF44
:106C3000002001F059FF0B2001F056FF002001F069
:106C400053FF1B2001F050FF002001F04DFF3420C6
:106C500001F04AFF002001F047FF442001F044FF0B
:106C6000002001F041FF4F2001F03EFF002001F025
:106C70003BFF612001F038FF002001F035FF792053
:106C800001F032FF002001F02FFF882001F02CFFDF
:106C9000002001F029FF972001F026FF002001F0DD
:106CA00023FFA62001F020FF002001F01DFFB720E8
:106CB00001F01AFF002001F017FFC22001F014FFBD
:106CC000002001F011FFC72001F00EFF002001F0AD
:106CD0000BFFD12001F008FF002001F005FFD620B6
:106CE00001F002FF002001F0FFFEDD2001F0FCFEBC
:106CF000002001F0F9FEF32001F0F6FE002001F083
:106D0000F3FEE32001F0FCFE052001F0EDFE002083
:106D100001F0EAFE0A2001F0E7FE002001F0E4FEA7
:106D20001C2001F0E1FE002001F0DEFE332001F026
:106D3000DBFE002001F0D8FE442001F0D5FE00204B
:106D400001F0D2FE502001F0CFFE002001F0CCFE79
:106D5000622001F0C9FE002001F0C6FE782001F09B
:106D6000C3FE002001F0C0FE882001F0BDFE00201F
:106D700001F0BAFE972001F0B7FE002001F0B4FE4A
:106D8000A62001F0B1FE002001F0AEFEB72001F018
:106D9000ABFE002001F0A8FEC22001F0A5FE0020FD
:106DA00001F0A2FEC72001F09FFE002001F09CFE32
:106DB000D12001F099FE002001F096FED52001F0CF
:106DC00093FE002001F090FEDD2001F08DFE0020FA
:106DD00001F08AFEF32001F087FE002001F084FE1E
:106DE000E42001F08DFE012001F07EFE002001F084
:106DF0007BFE012001F078FE002001F075FE0220EC
:106E000001F072FE002001F06FFE2A2001F06CFEFE
:106E1000002001F069FE3C2001F066FE002001F038
:106E200063FE4B2001F060FE002001F05DFE5D205E
:106E300001F05AFE002001F057FE742001F054FECC
:106E4000002001F051FE842001F04EFE002001F0F0
:106E50004BFE932001F048FE002001F045FEA220E9
:106E600001F042FE002001F03FFEB32001F03CFEA5
:106E7000002001F039FEBE2001F036FE002001F0B6
:106E800033FEC42001F030FE002001F02DFECD20A5
:106E900001F02AFE002001F027FED32001F024FE9D
:106EA000002001F021FEDD2001F01EFE002001F097
:106EB0001BFEF32001F018FE002001F015FEE52076
:106EC00001F01EFE002001F00FFE002001F00CFE7C
:106ED000002001F009FE002001F006FE022001F072
:106EE00003FE002001F000FE292001F0FDFD00203E
:106EF00001F0FAFD3C2001F0F7FD002001F0F4FD67
:106F00004B2001F0F1FD002001F0EEFD5D2001F0CD
:106F1000EBFD002001F0E8FD742001F0E5FD00200C
:106F200001F0E2FD842001F0DFFD002001F0DCFD36
:106F3000932001F0D9FD002001F0D6FDA22001F040
:106F4000D3FD002001F0D0FDB32001F0CDFD0020E5
:106F500001F0CAFDBE2001F0C7FD002001F0C4FD14
:106F6000C42001F0C1FD002001F0BEFDCD2001F0E4
:106F7000BBFD002001F0B8FDD32001F0B5FD0020DD
:106F800001F0B2FDDC2001F0AFFD002001F0ACFD0E
:106F9000F32001F0A9FD002001F0A6FDE62001F09C
:106FA000AFFD112001F0A0FD002001F09DFD342077
:106FB00001F09AFD002001F097FD562001F094FDAC
:106FC000002001F091FD762001F08EFD002001F0FF
:106FD0008BFD772001F088FD002001F085FD662003
:106FE00001F082FD002001F07FFD882001F07CFD92
:106FF000002001F079FD992001F076FD002001F0DC
:1070000073FDBB2001F070FD002001F06DFD9920A3
:1070100001F06AFD002001F067FD662001F064FDCB
:10702000002001F061FD552001F05EFD002001F01F
:107030005BFD552001F058FD002001F055FD452075
:1070400001F052FD002001F04FFD432001F04CFD06
:10705000002001F049FD442001F046FD002001F030
:1070600043FDE72001F04CFD322001F03DFD002002
:1070700001F03AFD552001F037FD002001F034FD0C
:10708000762001F031FD002001F02EFD662001F098
:107090002BFD002001F028FD672001F025FD0020D8
:1070A00001F022FD672001F01FFD002001F01CFD12
:1070B000872001F019FD002001F016FD992001F054
:1070C00013FD002001F010FDBB2001F00DFD00209C
:1070D00001F00AFD992001F007FD002001F004FDF8
:1070E000772001F001FD002001F0FEFC442001F0BA
:1070F000FBFC002001F0F8FC562001F0F5FC00201C
:1071000001F0F2FC232001F0EFFC002001F0ECFC88
:10711000332001F0E9FC002001F0E6FC452001F0FD
:10712000E3FC002001F0E0FCE82001F0E9FC002095
:1071300001F0DAFC002001F0D7FC992001F0D4FC2A
:10714000002001F0D1FC872001F0CEFC002001F0EE
:10715000CBFC882001F0C8FC002001F0C5FC7720A2
:1071600001F0C2FC002001F0BFFC662001F0BCFC75
:10717000002001F0B9FC882001F0B6FC002001F0ED
:10718000B3FCAA2001F0B0FC002001F0ADFCBB2054
:1071900001F0AAFC002001F0A7FC992001F0A4FC5A
:1071A000002001F0A1FC662001F09EFC002001F00F
:1071B0009BFC552001F098FC002001F095FC552027
:1071C00001F092FC002001F08FFC442001F08CFCC7
:1071D000002001F089FC442001F086FC002001F031
:1071E00083FC552001F080FC002001F07DFCE920AB
:1071F00001F086FCAA2001F077FC002001F074FC6D
:10720000002001F071FC002001F06EFC002001F074
:1072100077FCAA2001F068FCCF2001F071FC00206F
:1072200001F062FC002001F05FFC002001F05CFC3A
:10723000002001F059FC002001F056FC002001F074
:1072400053FC002001F050FC002001F04DFC002018
:1072500001F04AFC002001F047FC002001F044FC52
:10726000002001F041FC002001F03EFC002001F074
:107270003BFC002001F038FC002001F035FC002030
:1072800001F032FCF02001F03BFC002001F02CFC6E
:10729000502001F029FC002001F026FC002001F024
:1072A00023FC002001F020FCF32001F029FC002049
:1072B00001F01AFCF92001F023FC062001F014FC77
:1072C000102001F011FC292001F00EFC002001F03B
:1072D0000BFC3A2001F014FC552001F005FC1120B4
:1072E00001F00EFC642008F0C5FA292001F008FC2A
:1072F000352001F005FC002001F0F6FB512001F0E3
:10730000FFFBFF2001F0F0FB532001F0F9FB2C20E4
:1073100001F0EAFB552001F0F3FB822001F0E4FBD1
:107320002C2001F0EDFB01F048B8FE48808845F2C2
:10733000105188427ED155214FF4704001F0F6FB88
:10734000AA214FF2010001F0F1FB52214FF202009D
:1073500001F0ECFB08214FF2030001F0E7FB0121F3
:107360004FF2040001F0E2FB0D214FF4304001F038
:10737000DDFB0D214BF2010001F0D8FB0D214BF29A
:10738000020001F0D3FB34214FF4364001F0CEFB74
:1073900034214BF2016001F0C9FB34214BF2026051
:1073A00001F0C4FB0D214FF4314001F0BFFB0D2172
:1073B0004BF2011001F0BAFB0D214BF2021001F06B
:1073C000B5FB34214FF4374001F0B0FB34214BF2D0
:1073D000017001F0ABFB34214BF2027001F0A6FB0F
:1073E00000214FF4324001F0A1FB00214BF20120BB
:1073F00001F09CFB00214BF2022001F097FB2421BD
:107400004FF4384001F092FB24214BF6010001F0CB
:107410008DFB24214BF6020001F088FB01214FF483
:107420003F4001F083FB0F214FF4334001F07EFB1E
:107430000F2100E0FEE34BF2013001F077FB0F215A
:107440004BF2023001F072FB34214FF4394001F06D
:107450006DFB34214BF6011001F068FB34214BF633
:10746000021001F063FB08214FF4354001F05EFB90
:1074700008214BF2015001F059FB08214BF2025058
:1074800001F054FB03214FF4424001F04FFB242153
:107490004FF43A4001F04AFB24214BF6012001F061
:1074A00045FB24214BF6022001F040FB00214FF464
:1074B0003C4001F03BFB78214BF6014001F036FBEC
:1074C00000214BF6024001F031FB00214FF43D401A
:1074D00001F02CFB78214BF6015001F027FB002135
:1074E0004BF6025001F022FB00214FF43E4001F028
:1074F0001DFB64214BF6016001F018FB00214FF4E5
:10750000514001F013FB33214DF2011001F00EFB4D
:1075100000214DF2021001F009FB34214DF203105D
:1075200001F004FB00214DF2041001F0FFFA3A21B2
:107530004DF2051001F0FAFA00214DF2061001F0AB
:10754000F5FA4A214DF2071001F0F0FA00214DF250
:10755000081001F0EBFA5C214DF2091001F0E6FA97
:1075600000214DF20A1001F0E1FA81214DF20B10D9
:1075700001F0DCFA00214DF20C1001F0D7FAA6213F
:107580004DF20D1001F0D2FA00214DF20E1001F073
:10759000CDFAE5214DF20F1001F0C8FA01214DF2AC
:1075A000101001F0C3FA13214DF2111001F0BEFAD0
:1075B00001214DF2121001F0B9FA54214DF21310CD
:1075C00001F0B4FA01214DF2141001F0AFFA82215A
:1075D0004DF2151001F0AAFA01214DF2161001F03A
:1075E000A5FACA214DF2171001F0A0FA02214DF2BE
:1075F000181001F09BFA00214DF2191001F096FAD3
:1076000002214DF21A1001F091FA01214DF21B10E6
:1076100001F08CFA02214DF21C1001F087FA34219E
:107620004DF21D1001F082FA02214DF21E1001F000
:107630007DFA67214DF21F1001F078FA02214DF218
:10764000201001F073FA84214DF2211001F06EFA3E
:1076500002214DF2221001F069FAA4214DF223100B
:1076600001F064FA02214DF2241001F05FFAB72113
:107670004DF2251001F05AFA02214DF2261001F0C8
:1076800055FACF214DF2271001F050FA02214DF2A8
:10769000281001F04BFADE214DF2291001F046FAD4
:1076A00002214DF22A1001F041FAF2214DF22B1085
:1076B00001F03CFA02214DF22C1001F037FAFE21C4
:1076C0004DF22D1001F032FA03214DF22E1001F08F
:1076D0002DFA10214DF22F1001F028FA03214DF25E
:1076E000301001F023FA33214DF2311001F01EFA6F
:1076F00003214DF2321001F019FA6D214DF23310D1
:1077000001F014FA00214FF4524001F00FFA332136
:107710004DF2012001F00AFA00214DF2022001F0A1
:1077200005FA01E0C406002434214DF2032001F0E3
:10773000FDF900214DF2042001F0F8F93A214DF253
:10774000052001F0F3F900214DF2062001F0EEF9D9
:107750004A214DF2072001F0E9F900214DF20820FD
:1077600001F0E4F95C214DF2092001F0DFF900217C
:107770004DF20A2001F0DAF981214DF20B2001F0DF
:10778000D5F900214DF20C2001F0D0F9A6214DF2DF
:107790000D2001F0CBF900214DF20E2001F0C6F9C9
:1077A000E5214DF20F2001F0C1F901214DF2102029
:1077B00001F0BCF913214DF2112001F0B7F90121BC
:1077C0004DF2122001F0B2F954214DF2132001F0D4
:1077D000ADF901214DF2142001F0A8F982214DF2FA
:1077E000152001F0A3F901214DF2162001F09EF9B8
:1077F000CA214DF2172001F099F902214DF218200B
:1078000001F094F900214DF2192001F08FF90221C5
:107810004DF21A2001F08AF901214DF21B2001F0EE
:1078200085F902214DF21C2001F080F934214DF23E
:107830001D2001F07BF902214DF21E2001F076F9A6
:1078400067214DF21F2001F071F902214DF2202035
:1078500001F06CF984214DF2212001F067F9022139
:107860004DF2222001F062F9A4214DF2232001F013
:107870005DF902214DF2242001F058F9B7214DF2B3
:10788000252001F053F902214DF2262001F04EF996
:10789000CF214DF2272001F049F902214DF2282095
:1078A00001F044F9DE214DF2292001F03FF90221D7
:1078B0004DF22A2001F03AF9F2214DF22B2001F08D
:1078C00035F902214DF22C2001F030F9FE214DF264
:1078D0002D2001F02BF903214DF22E2001F026F985
:1078E00010214DF22F2001F021F903214DF230201B
:1078F00001F01CF933214DF2312001F017F9032179
:107900004DF2322001F012F96D214DF2332001F0D9
:107910000DF900214FF4534001F008F933214DF2E5
:10792000013001F003F900214DF2023001F0FEF8C0
:1079300034214DF2033001F0F9F800214DF204300A
:1079400001F0F4F83A214DF2053001F0EFF8002192
:107950004DF2063001F0EAF84A214DF2073001F00D
:10796000E5F800214DF2083001F0E0F85C214DF21D
:10797000093001F0DBF800214DF20A3001F0D6F8B1
:1079800081214DF20B3001F0D1F800214DF20C3085
:1079900001F0CCF8A6214DF20D3001F0C7F800211E
:1079A0004DF20E3001F0C2F8E5214DF20F3001F03A
:1079B000BDF801214DF2103001F0B8F813214DF25D
:1079C000113001F0B3F801214DF2123001F0AEF8A0
:1079D00054214DF2133001F0A9F801214DF2143079
:1079E00001F0A4F882214DF2153001F09FF8012139
:1079F0004DF2163001F09AF8CA214DF2173001F01D
:107A000095F802214DF2183001F090F800214DF266
:107A1000193001F08BF802214DF21A3001F086F88E
:107A200001214DF21B3001F081F802214DF21C3092
:107A300001F07CF834214DF21D3001F077F802217D
:107A40004DF21E3001F072F867214DF21F3001F047
:107A50006DF802214DF2203001F068F884214DF2DA
:107A6000213001F063F802214DF2223001F05EF87E
:107A7000A4214DF2233001F059F802214DF22430B7
:107A800001F054F8B7214DF2253001F04FF80221F2
:107A90004DF2263001F04AF8CF214DF2273001F0A7
:107AA00045F802214DF2283001F040F8DE214DF278
:107AB000293001F03BF802214DF22A3001F036F86E
:107AC000F2214DF22B3001F031F802214DF22C3031
:107AD00001F02CF8FE214DF22D3001F027F80321A2
:107AE0004DF22E3001F022F810214DF22F3001F02E
:107AF0001DF803214DF2303001F018F833214DF21A
:107B0000313001F013F803214DF2323001F00EF85C
:107B10006D214DF2333001F009F800214FF454404B
:107B200001F004F833214DF2014000F0FFFF002185
:107B30004DF2024000F0FAFF34214DF2034000F014
:107B4000F5FF00214DF2044000F0F0FF3A214DF224
:107B5000054000F0EBFF00214DF2064000F0E6FF8B
:107B60004A214DF2074000F0E1FF00214DF20840AC
:107B700000F0DCFF5C214DF2094000F0D7FF00214E
:107B80004DF20A4000F0D2FF81214DF20B4000F08F
:107B9000CDFF00214DF20C4000F0C8FFA6214DF2B0
:107BA0000D4000F0C3FF00214DF20E4000F0BEFF7B
:107BB000E5214DF20F4000F0B9FF01214DF21040D8
:107BC00000F0B4FF13214DF2114000F0AFFF01218E
:107BD0004DF2124000F0AAFF54214DF2134000F084
:107BE000A5FF01214DF2144000F0A0FF82214DF2CB
:107BF000154000F09BFF01214DF2164000F096FF6A
:107C0000CA214DF2174000F091FF02214DF21840B9
:107C100000F08CFF00214DF2194000F087FF022197
:107C20004DF21A4000F082FF01214DF21B4000F09E
:107C30007DFF00E003E302214DF21C4000F076FFDF
:107C400034214DF21D4000F071FF02214DF21E4023
:107C500000F06CFF67214DF21F4000F067FF02212A
:107C60004DF2204000F062FF84214DF2214000F0EF
:107C70005DFF02214DF2224000F058FFA4214DF299
:107C8000234000F053FF02214DF2244000F04EFF4C
:107C9000B7214DF2254000F049FF02214DF2264068
:107CA00000F044FFCF214DF2274000F03FFF0221BA
:107CB0004DF2284000F03AFFDE214DF2294000F05D
:107CC00035FF02214DF22A4000F030FFF2214DF243
:107CD0002B4000F02BFF02214DF22C4000F026FF3C
:107CE000FE214DF22D4000F021FF03214DF22E40E8
:107CF00000F01CFF10214DF22F4000F017FF032170
:107D00004DF2304000F012FF33214DF2314000F0CF
:107D10000DFF03214DF2324000F008FF6D214DF2BE
:107D2000334000F003FF00214FF4554000F0FEFE09
:107D300033214DF2015000F0F9FE00214DF20250C6
:107D400000F0F4FE34214DF2035000F0EFFE00216C
:107D50004DF2045000F0EAFE3A214DF2055000F0D9
:107D6000E5FE00214DF2065000F0E0FE4A214DF202
:107D7000075000F0DBFE00214DF2085000F0D6FE67
:107D80005C214DF2095000F0D1FE00214DF20A5065
:107D900000F0CCFE81214DF20B5000F0C7FE002117
:107DA0004DF20C5000F0C2FEA6214DF20D5000F035
:107DB000BDFE00214DF20E5000F0B8FEE5214DF25F
:107DC0000F5000F0B3FE01214DF2105000F0AEFE56
:107DD00013214DF2115000F0A9FE01214DF2125075
:107DE00000F0A4FE54214DF2135000F09FFE01213B
:107DF0004DF2145000F09AFE82214DF2155000F021
:107E000095FE01214DF2165000F090FECA214DF270
:107E1000175000F08BFE02214DF2185000F086FE44
:107E200000214DF2195000F081FE02214DF21A504E
:107E300000F07CFE01214DF21B5000F077FE022184
:107E40004DF21C5000F072FE34214DF21D5000F036
:107E50006DFE02214DF21E5000F068FE67214DF2CA
:107E60001F5000F063FE02214DF2205000F05EFE34
:107E700084214DF2215000F059FE02214DF2225092
:107E800000F054FEA4214DF2235000F04FFE0221D9
:107E90004DF2245000F04AFEB7214DF2255000F07B
:107EA00045FE02214DF2265000F040FECF214DF25A
:107EB000275000F03BFE02214DF2285000F036FE24
:107EC000DE214DF2295000F031FE02214DF22A5000
:107ED00000F02CFEF2214DF22B5000F027FE022183
:107EE0004DF22C5000F022FEFE214DF22D5000F0FC
:107EF0001DFE03214DF22E5000F018FE10214DF210
:107F00002F5000F013FE03214DF2305000F00EFE12
:107F100033214DF2315000F009FE03214DF2325071
:107F200000F004FE6D214DF2335000F0FFFD002102
:107F30004FF4564000F0FAFD33214DF2016000F09D
:107F4000F5FD00214DF2026000F0F0FD34214DF20C
:107F5000036000F0EBFD00214DF2046000F0E6FD4F
:107F60003A214DF2056000F0E1FD00214DF206607E
:107F700000F0DCFD4A214DF2076000F0D7FD002142
:107F80004DF2086000F0D2FD5C214DF2096000F076
:107F9000CDFD00214DF20A6000F0C8FD81214DF2B7
:107FA0000B6000F0C3FD00214DF20C6000F0BEFD3F
:107FB000A6214DF20D6000F0B9FD00214DF20E60DA
:107FC00000F0B4FDE5214DF20F6000F0AFFD01219E
:107FD0004DF2106000F0AAFD13214DF2116000F087
:107FE000A5FD01214DF2126000F0A0FD54214DF2DB
:107FF000136000F09BFD01214DF2146000F096FD2E
:1080000082214DF2156000F091FD01214DF21660C4
:1080100000F08CFDCA214DF2176000F087FD0221AF
:108020004DF2186000F082FD00214DF2196000F061
:108030007DFD02214DF21A6000F078FD01214DF224
:108040001B6000F073FD02214DF21C6000F06EFD1C
:1080500034214DF21D6000F069FD02214DF21E60D9
:1080600000F064FD67214DF21F6000F05FFD02210A
:108070004DF2206000F05AFD84214DF2216000F0A5
:1080800055FD02214DF2226000F050FDA4214DF279
:10809000236000F04BFD02214DF2246000F046FD0C
:1080A000B7214DF2256000F041FD02214DF226601E
:1080B00000F03CFDCF214DF2276000F037FD02219A
:1080C0004DF2286000F032FDDE214DF2296000F013
:1080D0002DFD02214DF22A6000F028FDF2214DF223
:1080E0002B6000F023FD02214DF22C6000F01EFDFC
:1080F000FE214DF22D6000F019FD03214DF22E609E
:1081000000F014FD10214DF22F6000F00FFD03214F
:108110004DF2306000F00AFD33214DF2316000F085
:1081200005FD03214DF2326000F000FD6D214DF29E
:10813000336000F0FBFC55214FF4704000F0F6FC7A
:10814000AA214FF2010000F0F1FC52214FF202008F
:1081500000F0ECFC08214FF2030000F0E7FC0021E6
:108160004FF2040000F0E2FCCC214FF4314000F06B
:10817000DDFC00214BF2011000F0D8FC05214FF48A
:10818000364000F0D3FC70214FF4374000F0CEFCB5
:1081900070214BF2017000F0C9FC01214FF438400E
:1081A00000F0C4FC03214BF6010000F0BFFC0321EA
:1081B0004BF6020000F0BAFC03214BF6030000F07E
:1081C000B5FC02214FF43C4000F0B0FC00214BF61E
:1081D000014000F0ABFC00214BF6024000F0A6FC91
:1081E000D0214FF4494000F0A1FC02214CF60110CF
:1081F00000F09CFC50214CF6021000F097FC50213E
:108200004CF6031000F092FC50214CF6041000F0E4
:108210008DFC00214FF4545000F088FC55214FF4A0
:10822000685000F083FC4FF4885000F069FC78201F
:1082300007F02CFB4FF4245000F062FCBDE07948BD
:10824000808841F663118842F8D1E22000F058FCA2
:108250001D2000F049FC022000F046FC042000F044
:1082600043FC642007F012FBE02000F049FC0120F1
:1082700000F03AFC0A2007F0FDFAE02000F040FC94
:10828000032000F031FC0C2007F0F4FA012000F08C
:1082900037FC0A2007F0EEFAE62000F031FC2F2030
:1082A00000F022FCFF2000F01FFCFF2000F01CFC6F
:1082B000B02000F025FC202000F016FC002000F08B
:1082C00013FC032000F010FC40F21F3000F00CFC07
:1082D000012000F009FC40F2DF1000F005FC002056
:1082E00000F002FCB42000F00BFC042000F0FCFBCA
:1082F00040F21F4000F0F8FB002000F0F5FB2E20BC
:1083000000F0F2FB002000F0EFFB002000F0ECFB9F
:10831000002000F0E9FB002000F0E6FBB62000F0B2
:10832000EFFB022000F0E0FB4FF4037000F0DCFBF9
:10833000002000F0D9FB172000F0D6FB152000F03C
:10834000D3FB002000F0D0FB002000F0CDFBF0209C
:1083500000F0D6FB032000F0C7FB292000F0D0FB83
:10836000D02000F0CDFB002000F0BEFBBE2000F0CE
:10837000C7FB052000F0B8FBFE2000F0B5FB012094
:1083800000F0B2FB002000F0AFFB002000F0ACFBDF
:10839000002000F0A9FBB82000F0B2FB032000F0A1
:1083A000A3FB012000F0A0FBBA2000F0A9FB0120F4
:1083B00000F09AFB642000F07DF81A48808849F2AA
:1083C0004131884211D01748808845F210318842E7
:1083D0000BD01448808845F21051884205D01148CE
:1083E000808841F66311884209D1052002900490EB
:1083F0000D49CB6A8A68486802A9F8F777F80948F6
:1084000081880AA006F0BEFF0020FDF75BFC012278
:1084100020210948F8F72CFD4FF6FF70FDF72EFCE0
:1084200015B000BDC4060024780600244C43442047
:1084300049443A25780D0A00000402581FB5F8F7A0
:1084400039FF01208DF8000003208DF8010040075E
:1084500001901B208DF8080000208DF809008DF890
:108460000A0003208DF80B0000208DF80C008DF819
:108470000D008DF80E0001208DF80F006846F8F70A
:10848000EBFE0420F8F72CFF1FBD10B502460120BB
:1084900000E050430B1EA1F10104E1B2F9D110BD7F
:1084A00008B5034800880090BDF8000008BD000032
:1084B0000000086000B50246BE2000F021FB052048
:1084C00000F012FB00EE102AB8EE400B9FED0B1BE4
:1084D00020EE010BBCEEC00B10EE101A88B200F0BB
:1084E00003FB012000F000FBFF2000F0FDFA00205C
:1084F00000F0FAFA002000F0F7FA00BD6666666642
:1085000066660440F0B50546002400279948807946
:10851000012805D19748808841F66311884208D127
:1085200094488079F0B99348808841F66311884275
:1085300018D1082D15D2DFE805F00406080A0C0E44
:10854000101206250DE007250BE0042509E005259E
:1085500007E0012505E0002503E0032501E00225F1
:1085600000BF00BF8348808849F24131884211D062
:108570008048808845F2103188420BD07D48808841
:1085800045F21051884205D07A48808841F663113F
:1085900088427DD1082D1CD2DFE805F00406090CC5
:1085A0000F12151800BF14E044F0800411E044F0ED
:1085B00040040EE044F0C0040BE044F0200408E066
:1085C00044F0600405E044F0A00402E044F0E0045C
:1085D00000BF00BF6748808845F21051884202D131
:1085E0004FF4585700E036276248808845F2103132
:1085F00088420DD05F48808845F21051884207D0EC
:108600005C48808841F66311884201D044F0080438
:108610002146384600F08AFA5648808841F66311B0
:1086200088421DD004F0200068B1524800885149AA
:108630004988884214DA4F48068840884D490880A6
:10864000084646800CE04B4800884A4949888842E1
:1086500006DD484806884088464908800846468026
:108660004448808845F21051884254D14149488994
:1086700000F046FA002000F037FA3E494989491CCB
:1086800088B200F03DFA002000F02EFA394900E0EF
:108690006FE04989891C88B200F032FA35490988AF
:1086A000491EC1F30F2000F01FFA32494989C91C45
:1086B00088B200F025FA2F490978491EC8B200F0A7
:1086C00013FA2C49888900F01BFA002000F00CFAFC
:1086D00028498989491C88B200F012FA002000F06C
:1086E00003FA24498989891C88B200F009FA2149D2
:1086F0004988491EC1F30F2000F0F6F91D49898908
:10870000C91C88B200F0FCF91A498978491EC8B220
:1087100000F0EAF92DE01749488900F0F1F900204E
:1087200000F0E2F9002000F0DFF912490988491E43
:10873000C1F30F2000F0D8F90E490978491EC8B2DC
:1087400000F0D2F90B49888900F0DAF9002000F036
:10875000CBF9002000F0C8F906494988491EC1F349
:108760000F2000F0C1F903498978491EC8B200F012
:10877000BBF9F0BDC406002410B502460C464B48B8
:10878000808849F24131884205D04848808845F2C6
:108790001031884214D14549488900F0B1F91012CE
:1087A00000F0A2F9D0B200F09FF94049888900F0AA
:1087B000A7F9201200F098F9E0B200F095F973E003
:1087C0003A48808841F66311884247D1374880791A
:1087D000A8B936480088401E801A82B233494889B9
:1087E00000F08EF9002000F07FF9002000F07CF905
:1087F000101200F079F9D0B200F076F916E02B49AA
:10880000488900F07DF9101200F06EF9D0B200F046
:108810006BF926490988491EC1F30F2000F064F95D
:1088200022490978491EC8B200F05EF91F498889BB
:1088300000F066F9201200F057F9E0B200F054F9A8
:108840001A494988491EC1F30F2000F04DF9174914
:108850008978491EC8B200F047F925E0134880889E
:1088600045F2105188421FD11049488900F048F95B
:10887000101200F039F90D494989491C88B200F0FD
:108880003FF9D0B200F030F90849888900F038F992
:10889000201200F029F905498989491C88B200F0A5
:1088A0002FF9E0B200F020F910BD0000C40600244A
:1088B0002DE9F84F80460F4616461C46BB4620461B
:1088C000E31704EB5373DB1021464FEAE47C04EB1F
:1088D0005C7C4FEAEC0CA4EBCC0CBCF1000F02D09A
:1088E0004FF0010C01E04FF0000C6344224604EB12
:1088F000D27C4FEA6C0C03FB0CF3DBB20093A6F1C5
:108900002000C6B200255EE00C2C07D106EB460025
:108910002F4901EB800010F805901BE0102C05D1C9
:108920002C4800EB061010F8059013E0182C07D126
:1089300006EBC600284901EB800010F8059009E01D
:10894000202C05D1254800EBC61010F8059001E059
:10895000BDE8F88F4FF0000A2FE009F0800030B139
:108960001F48394602684046FDF76CFA07E00A984E
:1089700028B91C48394602684046FDF763FA4FEAB9
:1089800049604FEA1069781C87B217484088B8429E
:1089900000DCDDE7A7EB0B00A0420AD15F4608F13F
:1089A00001001FFA80F810480088404500DCCFE73E
:1089B00006E00AF1010000F0FF0ABAF1080FCCDB73
:1089C00000BF681CC5B2009885429DDB00BFBFE7B1
:1089D0002411010898150108881B0108E4280108E2
:1089E0002000002424000024C40600242DE9FF4FA9
:1089F00081B0074691461E460E9D4FF0000A0024A6
:108A000039E0301B401EC1B20A20FFF73EFDB9FB22
:108A1000F0F00A21B0FBF1F201FB1208BAF1000FED
:108A200016D1701EA04213DDB8F1000F0ED1002048
:108A3000AB4605EBDB71491001FB0471009088B275
:108A40002B4620220299FFF733FF12E04FF0010A74
:108A50000020AB4605EBDB71491001FB047100906F
:108A600088B208F13001CAB22B460299FFF720FF05
:108A700000BF601CC4B2B442C3DB05B0BDE8F08FD8
:108A80002DE9F84F04460D4690469946DDE90A6700
:108A900004F0FF0A08EB04001FFA80F809EB050058
:108AA0001FFA80F916E0444502DB5446A81985B246
:108AB0004D4500DB14E0002000903A78334629460B
:108AC0002046FFF7F5FE304606EBD07104EB61015E
:108AD0008CB27F1C38787E2802DC38782028E2DAD5
:108AE00000BFBDE8F88F000001B5BDF800000090A0
:108AF000BDF800000149088008BD000000000860C2
:108B000001B5BDF800000090BDF8000001490880E3
:108B100008BD0000FEFF0760024800890249088086
:108B200070470000C4060024FEFF0760024A108060
:108B3000921C118070470000FEFF076000B587B0EF
:108B400000BF1248006840F0020010490860084663
:108B5000006800F00200019000BF00BF03200290F7
:108B60000120039004900320059002A90848F8F71B
:108B70004DF8012211460648F8F77AF90122022140
:108B80000348F8F775F907B000BD0000E04402584B
:108B90000004025818B5044606480094008B401E95
:108BA00083B20448C08A401E82B20021084600F009
:108BB00059F818BDDC07002470B5B0B004460E4665
:108BC00015464FF0005001900A940B9602210C912B
:108BD0000D910E9501A8F9F787FE10B9002030B06D
:108BE00070BD0120FBE700000949487530B989884C
:108BF000074AD18211460988118308E0012806D16D
:108C000003490988024AD182114689881183704735
:108C1000DC07002470B5114B5B7D6BB10F4BDB693A
:108C20000E4D2D6805FB01056B430C4D2D7D0C4E43
:108C300056F82550EA520FE0084B1D685B681B1A76
:108C40005B1E05FB0313054DED696B43034D2D7D45
:108C5000034E56F82550EA5270BD0000DC07002490
:108C6000280000242DE9F04F04460D4616464FF02B
:108C7000000CDFF8289199F81590B9F1000F04D095
:108C80002046294632461F4611E02846DFF80C915F
:108C9000D9F80490A9EB0609A9F101011A46DFF8F9
:108CA000FC90D9F80490A9EB0409A9F10107DFF8B9
:108CB000EC90B9F80090A2EB000A0AF1010AA9EBC6
:108CC0000A091FFA89F8DFF8D49099F81490DFF8B0
:108CD000D0A05AF82990DFF8C4A0DAF81CA0DFF879
:108CE000BCB0DBF800B00BFB010B0AFB0B9EDFF8FE
:108CF000B490D9F8009049F40009DFF8A8A0CAF8A8
:108D000000904FF44039DFF8A0A0CAF800904FF06F
:108D10000209CAF83490D146C9F84080D9F80090C9
:108D200029F00109CAF80090D146C9F83CE0A7EB48
:108D3000010909F10109A2EB000A0AF1010A49EA55
:108D40000A49DFF864A0CAF84490DDF82490CAF814
:108D50003890D146D9F8009049F00109CAF800903E
:108D600005E00CF1010CBCF5001F00D308E0DFF8B2
:108D70003890D9F8049009F00209B9F1000FF0D049
:108D800000BFDFF82490D9F8089049F00209DFF815
:108D900018A0CAF80890BDE8F08F0000DC07002496
:108DA00028000024D8440258001000521FB50024A7
:108DB00000F050FA044644F24230844217D14FF496
:108DC000F070F24908604FF4887048600120088113
:108DD0004881282088810820C88105200882082031
:108DE00048825822A0210520FFF7E6FE2FE147F236
:108DF0008400844217D14FF44870E44908604FF46E
:108E0000F07048600120088148812E208881172059
:108E1000C881D2200882162048821822A02105206D
:108E2000FFF7CAFE13E147F21600844218D14FF44F
:108E30008060D64908604FF416704860142008819D
:108E4000032048818C2088811420C881A0200882BA
:108E50000C2048821222A0210520FFF7ADFEF6E08B
:108E600047F21800844207D14FF4A060C749086058
:108E70004FF448704860EAE048F21600844206D198
:108E80004011C24908604FF416704860DFE041F2BB
:108E90001800844215D14FF4A060BC4908604FF41B
:108EA000487048608C2088810A2008820881C88127
:108EB0004882032048811022A0210520FFF77CFE74
:108EC000C5E04AF20100844218D140F25650AF4941
:108ED00008604FF4407048608F2008814620088267
:108EE000D5208881032048811820C881032048822A
:108EF0001C22A0210520FFF75FFEA8E04AF2020035
:108F0000844217D14011A14908604FF4487048606D
:108F10002020088130200882502088810620488146
:108F20000E20C881032048821622A0210520FFF7C9
:108F300043FE8CE04AF20300844217D1401193496A
:108F400008604FF4407048602020088150208881DC
:108F500030200882072048810C20C88103204882E5
:108F60001722A0210520FFF727FE70E04AF2040037
:108F7000844218D14FF48060844908604FF44070F7
:108F800048608820088118200882A0208881062057
:108F900048811D20C881032048821222A02105207B
:108FA000FFF70AFE53E04AF20500844217D14FF45E
:108FB0005470764908604FF4F07048607020088162
:108FC000888110200882082048811720C881062047
:108FD00048822F22A0210520FFF7EEFD37E04AF25C
:108FE0000600844218D14FF44870684908604FF475
:108FF00016704860802008815820888128200882C7
:10900000042048811720C881012048822822A021FD
:109010000520FFF7D1FD1AE04AF20700844216D17D
:1090200080115A4908604FF4F07048606020088150
:109030000820088238208881022048812920C881A0
:10904000022048823E22A0210520FFF7B5FD4F48AF
:1090500000884F4908804D488088488002204B494D
:10906000C8614C484C4908604C484D490860002094
:10907000486000214A488160C160016141F21800E6
:10908000844203D14FF08051454801613F48008937
:10909000401E434948613D484089401E88613B4825
:1090A00000893A4989890844401E3D49C8613748CA
:1090B00040893649C9890844401E39490862334805
:1090C0000089324989890844304909680844401EAA
:1090D000334948622D4840892C49C98908442B49A5
:1090E00049680844401E2E4988622848008927495B
:1090F000898908442549096808442449098A08449B
:10910000401E2749C862214840892049C98908442E
:109110001E49496808441D49498A0844401E20499F
:10912000086300211E4880F8361080F8351080F85A
:109130003410F7F719FF002007210622CDE90002BD
:10914000CDE902101448FF2302220168002000F03C
:109150002BF80E48808880B200900C48008883B2BB
:1091600000221146104600F05DF80020FFF73CFD9C
:10917000002000F0D7F8012220210A48F7F778FEF6
:109180004FF0FF30FFF706FD1FBD0000DC07002495
:10919000C4060024000000C0280000240010005075
:1091A000D4060024000402582DE9F04F8DB0054686
:1091B0000E4617469846DDE917ABDDF85890199C26
:1091C0000020009002901548006801901348406804
:1091D00003900497CDF81480CDF818904FEA0A2038
:1091E00007904FEA0B20089009960C4800680A90F7
:1091F0000A4840680B90002001148DF832100112CB
:109200008DF83110E0B28DF830002A4669460448E6
:10921000F7F77AFE0DB0BDE8F08F0000DC07002400
:10922000D40600242DE9F04104460E4617461D469B
:10923000DDF8188023463A4631460548F7F7A0FF87
:109240002346424629460248F7F7D0FFBDE8F081A1
:10925000D406002410B586B0002400BF2E48006854
:1092600040F400702C4908600846006800F4007063
:10927000009000BF00BF00BF0846006840F4806057
:1092800008600846006800F48060009000BF00BFDE
:1092900040200190002002900320049001A91F4863
:1092A000F7F7B4FC4420019001A91D48F7F7AEFC84
:1092B00040211A48F7F7D0FD044604211848F7F773
:1092C000CBFD44EA4000C4B240211548F7F7C4FD85
:1092D00044EA8000C4B21CB944F2423006B010BD6A
:1092E000012C02D147F28400F8E7022C02D147F2A8
:1092F0001600F3E7032C02D147F21800EEE7042C26
:1093000002D148F21600E9E7052C02D141F218001B
:10931000E4E70020E2E70000E0440258002402589D
:10932000002802580149087570470000DC07002436
:10933000F0B50023002400258E880768FF68C7F376
:109340000B473E44330406688436802707FB0266D9
:10935000766806F47047066884364FF0800C0CFB84
:10936000026677600E680768FF68C7F30B473E44E4
:10937000761C1E43076884370CFB02777E608E895B
:109380000768FF68C7F30A073E443304066884365B
:10939000802707FB0266B66806F4704706688436C5
:1093A0000CFB0266B7608E680768FF68C7F30A07A0
:1093B0003E44761C1E43076884370CFB0277BE6070
:1093C00006688436802707FB0266366926F00707A1
:1093D000066884360CFB026637610F6906688436BE
:1093E0000CFB026637613126765C33023226765CEE
:1093F00034040E7E350606688436802707FB026635
:10940000B6690027066884360CFB0266B76191F8DE
:1094100030601E4326432E43076884370CFB0277D7
:10942000BE6106688436802707FB0266766926F0EF
:10943000FF07066884360CFB026677614F69066891
:1094400084360CFB0266776106688436802707FB4A
:109450000266F76940F20776B743066884360CFB6C
:109460000266F761D1E907673E43076884370CFB62
:109470000277FE6106688436802707FB0266B66ABB
:109480000027066884360CFB0266B7624F6A0668DE
:1094900084360CFB0266B7620E690EB9042313E032
:1094A0000E69012E01D103230EE00E69042E08D0AF
:1094B0000E69022E05D00E69032E02D00E69072E0A
:1094C00001D1022300E0012306688436802707FBD0
:1094D0000266F66A06F0E027066884364FF0800CD4
:1094E0000CFB0266F762D1E90076F61B5E43F71DBE
:1094F0000E8D5E4347EA0647066884360CFB02661B
:10950000F76206688436802707FB0266366BF70A27
:10951000FF02066884360CFB02663763CF6A066872
:1095200084360CFB0266376306688436D701F65929
:1095300046F00107066884364FEAC21C46F80C70F4
:10954000F0BD0EB500200121009103230A46CDE9AC
:1095500001101221480600F00CF801200022CDE98C
:1095600000200323022219210290980700F001F83D
:109570000EBD2DE9FF4704460D4616461F46DDE9A0
:109580000D9ADDF83080F7F795FE01208DF8000088
:10959000F0B28DF801000194E8B28DF808000020C7
:1095A0008DF809008DF80A008DF80B708DF80C000D
:1095B0008DF80D808DF80E908DF80FA06846F7F7A6
:1095C0004BFE0420F7F78CFE002004B0BDE8F087C6
:1095D00070B50546D5F8184248F20C002044007BCF
:1095E00050B948F20C002044806828B1607A18B95C
:1095F0000121284604F0E7FA8121284604F0E3FA25
:10960000607A022807D11F2348F20C00221801219A
:10961000284604F043FA70BD70B50546D5F81842E7
:1096200048F20C002044406848F22C012144486074
:1096300048F20C002044806848F22C0121448860E4
:109640000121284604F0BCF91F2817D148F20C006C
:1096500000592B49884211D148F20C002044407B2C
:1096600001280BDC48F20C002044807B012805DB3C
:1096700048F20C002044807B10280EDD48F20C00DC
:109680002044417B20230522284601F048FB02208C
:1096900060722846FFF79CFF31E048F20C0020443E
:1096A000417B48F20C0022180F32284601F09CF84A
:1096B00000280BDA207A052804D10121284600F081
:1096C000C1F81CE02846FFF783FF18E0207A022843
:1096D00015D0207A012812D0207A03280FD0608973
:1096E000002806DD628904F10C01284600F0CAF862
:1096F00005E0608918B90021284600F0A3F870BD84
:109700005553424370B506460D46D6F81842607A66
:10971000022806D18121304604F055FA00206072FB
:109720000AE005F08000802806D1607A012803D085
:109730000121304600F086F870BD70B505460E4632
:10974000D5F81842207A022804D0032815D004281E
:1097500018D111E048F20C002044417B48F20C0083
:1097600022180F32284601F03FF8002803DA0121C1
:10977000284600F067F806E000BF0021284600F008
:1097800061F800E000BF00BF70BD70B505460E4631
:10979000D5F81842207A10B1012816D103E02846E6
:1097A000FFF73AFF12E048F20C002044417B48F2F8
:1097B0000C0022180F32284601F016F8002803DAB0
:1097C0000121284600F03EF800E000BF00BF70BD58
:1097D000D0F8181200220A72704770B50546D5F805
:1097E0001842002020726072002148F25D0001558D
:1097F000401E0155D5F81C02016800208847012150
:10980000284604F0D3F88121284604F0CFF81F231E
:1098100048F20C0022180121284604F03FF970BDDF
:1098200070B50546D5F818420020207201206072FC
:109830001F2348F20C0022180121284604F02EF9BB
:1098400070BD000070B505460E46D5F818420C49AB
:1098500048F22C00015120440673002020720D2391
:1098600048F22C0022188121284604F0C8F91F2351
:1098700048F20C0022180121284604F00FF970BDAF
:10988000555342532DE9F04106460F461546D6F88A
:10989000184248F20C0020448068A84204D248F2E2
:1098A0000C002044806800E0284685B248F22C0075
:1098B00020448068401B48F22C012144886000202D
:1098C00048F22C0121440873042020722B463A46AA
:1098D0008121304604F093F9BDE8F08100BFFEE736
:1098E00001B502E00098401E009000980028F9D1D0
:1098F00008BD00002DE9F74F82B00546164600204E
:109900000190002481460120039900F055F8074694
:109910000020039900F050F882463146012000F003
:109920004BF880463146002000F046F8834687EA2F
:109930000A0080EA080080EA0B00019040F6FF71FF
:109940000198884219D187EA080421460FA005F042
:1099500019FD2046E11704EB51714FEAE109E117C7
:1099600004EB5171C910A4EBC1020121914015F81B
:109970000920514005F8091006E008A005F002FD95
:10998000012005B0BDE8F08F0020FAE76572726F24
:1099900072706F733A25640D0A00000032626974B8
:1099A00020656363206572726F72206F72206D6F25
:1099B00072650D0A0000000030B502460B4600201B
:1099C000002113E00C4601EBD4756D10A1EB4505A9
:1099D000954209D123FA01F404F0010424B14D1099
:1099E0000124AC400444A0B24C1CE1B21829E9DBCC
:1099F00030BD000010B50446114800691149884285
:109A000001D1E40105E00E4800690F49884200D108
:109A1000A40160200D4908700D490C70200A0870DF
:109A2000200C0870D02009490870042005F022FF9E
:109A300000F0A4FA402801D0012010BD0020FCE76E
:109A4000CC0B002489260048569590DC000001804C
:109A50000000028000B589B000F070F82E482F4950
:109A600008604FF48070486000212C488160C1601C
:109A700001614FF4003141610A218161C1610A2015
:109A80000590069007900890019002900390049032
:109A900001AA05A92148F7F745FC00F05DFA64200A
:109AA00005F0E8FE00F092F81D49086108460169DA
:109AB0001CA005F067FC042000F068F81848006955
:109AC0001C4988420FD14FF48750154908804FF444
:109AD00080504880E02088808020887100010881C3
:109AE0004000488116E00E480069134988420ED1B3
:109AF0004FF404600A4908804FF400604880402019
:109B000088808871400108814000488102E001207E
:109B100009B000BD0020FBE7804000528C0B002400
:109B2000CC0B00244E414E442049443A2523780D65
:109B30000A00000089260048569590DC1FB5F7F70B
:109B4000B9FB01208DF8000004208DF801004007CA
:109B500001901B208DF8080000208DF809008DF879
:109B60000A0003208DF80B0001208DF80C00002066
:109B70008DF80D008DF80E008DF80F006846F7F790
:109B80006BFB0420F7F7ACFB1FBD000010B50446CB
:109B9000EF200C49087001200B4908702320FFF7C3
:109BA0009FFE4FF00040047000204FF0004108700D
:109BB0000870087000F0E2F9402801D1002010BDC3
:109BC0000120FCE700000180000002801CB590200D
:109BD0001C49087000201C4908701E20FFF780FEF9
:109BE0004FF0004000788DF800004FF00040007802
:109BF0008DF801004FF0004000788DF802004FF022
:109C0000004000788DF803004FF0004000788DF898
:109C100004009DF8010000069DF8021040EA014092
:109C20009DF8031040EA01209DF8041040EA010469
:109C300000F0A4F9402801D120461CBD4FF0FF30B0
:109C4000FBE7000000000180000002802DE9FC5FBE
:109C500081460F4616461D460020019080468246EA
:109C6000002400908D4908708D490F7038120870DB
:109C700081F800904FEA192008704FEA19400870E7
:109C8000302086490870002000F094F98046B8F131
:109C9000000F02D00220BDE8FC9F012000F08AF9ED
:109CA0008046B8F1000F01D00220F4E7E91705EB78
:109CB000D1514912A5EB412189B10020019009E061
:109CC0004FF00040007806F8010BBDF80400401C7E
:109CD00080B20190BDF80400A842F1DBD5E028462F
:109CE000E91705EBD151C1F3472A3846F91707EBBD
:109CF000D151C1F34724B3464FF0000839E000F0DA
:109D000039FC6848006840F0400066498039C1F875
:109D100080000020019009E04FF00040007806F834
:109D2000010BBDF80400401C80B20190BDF8040096
:109D3000B0F5007FF0DB00BF5A48001D006800F05E
:109D400040000028F8D000F015FC56481430016897
:109D500008EB0402544840F8221052488038D0F8EA
:109D6000800020F040004F49086008F1010000F039
:109D7000FF08D045C3DB4C481C384088103000EB4E
:109D8000840080B201903220FFF7AAFD05204349EC
:109D90000870BDF8040042490870BDF804000012C4
:109DA0000870E0203D4908701E20FFF799FD3E48ED
:109DB000203000EB840600F0DDFB0020019009E07C
:109DC0004FF00040007806F8010BBDF80400401C7D
:109DD00080B201904FEA8A00BDF804108842EFDC9F
:109DE000002001904DE0BDF8040001192E482030FC
:109DF00050F82110BDF8040002192B4850F8220039
:109E0000814239D0BDF8040003192748203050F8AA
:109E10002320BDF804000319234850F8231023A081
:109E200005F0B0FA2246514626A005F0ABFA3A46B4
:109E300049462AA005F0A6FABDF8043003EB040C4D
:109E4000194B53F82C20BDF8043003EB040C164BCF
:109E5000203353F82C10BDF804304FF4007C0CFB79
:109E600003B0FFF747FD8046B8F1000F02D0042091
:109E7000009001E003200090BDF80400401C80B277
:109E80000190BDF804005045ADDB00F077F84028A4
:109E900001D0012000900098FDE600000000018044
:109EA0000000028080400052E80B0024657272209E
:109EB00068642C72643A307825782C307825780DD7
:109EC0000A0000006563636E756D2C6563637374CF
:109ED0006172743A25642C25640D0A00506167652F
:109EE0004E756D2C436F6C4E756D3A25642C256450
:109EF0000D0A00002DE9F04707460C4690461D4626
:109F00004FF0000900260A480079001BC6B2B5428E
:109F100000DD354606484088204481B22B46424643
:109F20003846FFF793FE81464846BDE8F0870000BB
:109F3000CC0B002408B50020009070200549087063
:109F40001E20FFF7CDFC4FF00040007800909DF8F8
:109F5000000008BD0000018010B5FF200649087010
:109F6000032005F087FC00F009F8402801D100200B
:109F700010BD0120FCE700000000018008B50022B0
:109F8000002000900FE0FFF7D5FF024602F04000EE
:109F900000B109E00098401C0090054900988842F3
:109FA00001D3022008BDEEE700BF4020FAE7000021
:109FB000FFFF010001B582B000200190009018E081
:109FC0000198401C019040210D48F6F745FF9DF88F
:109FD0000810884205D19DF80000401CC0B20090D6
:109FE00001E0002000909DF80000022801DD002023
:109FF0000EBD6FF07E4101988842E1D30120F7E762
:10A00000000C02582DE9F84F80460E4615461C46B6
:10A010000020009000278246814680205A4908701F
:10A020005A490E703012087081F800804FEA1820EB
:10A0300008704FEA184008702320FFF751FCE11721
:10A0400004EBD1514912A4EB412189B100200090C9
:10A0500009E015F8010B4FF000410870BDF8000051
:10A06000401C80B20090BDF80000A042F1DB7AE015
:10A070002046E11704EBD151C1F3472A3046F117CE
:10A0800006EBD151C1F34729002737E000F072FAFF
:10A090003F48006840F040003D498039C1F88000E9
:10A0A0000020009009E015F8010B4FF00041087006
:10A0B000BDF80000401C80B20090BDF80000B0F573
:10A0C000007FF0DB00BF3248001D006800F0400058
:10A0D0000028F8D000F04EFA2D481430016807EB44
:10A0E00009022C4840F8221029488038D0F8800016
:10A0F00020F0400026490860781CC7B25745C5DBF0
:10A1000024481C384088103000EB890080B2009051
:10A110002320FFF7E5FB85201B490870BDF80000F0
:10A120001A490870BDF80000001208702320FFF7DC
:10A13000D7FB184800EB8905002000900FE00027AE
:10A1400006E015F8010B4FF000410870781CC7B20B
:10A15000042FF6DBBDF80000401C80B20090BDF873
:10A1600000005045EBDB1020074908704FF4AF703A
:10A1700005F08CFBFFF702FF402802D00120BDE86C
:10A18000F88F0020FBE70000000001800000028043
:10A1900080400052E80B00242DE9F04707460C46AA
:10A1A00090461D464FF0000900260A480079001B22
:10A1B000C6B2B54200DD354606484088204481B22B
:10A1C0002B4642463846FFF71DFF81464846BDE80C
:10A1D000F0870000CC0B00247047000010B5024847
:10A1E000F7F7BCFB10BD0000006F03242DE9F84F0A
:10A1F00007460E46D7F8008000240025A146A24657
:10A20000C6EBC60107F1380000EB8104D4E9050173
:10A21000451AA068A84200D2A568E81CC11700EB47
:10A2200091714FEAA1091AE0D4E90501451AA06825
:10A23000A84200D2A568E81CC11700EB91714FEA53
:10A24000A109387CABB2F2B200904046E16804F05C
:10A250009DFEE0682844E060A0692844A06108F5FC
:10A26000106000EB4610806980B2484506D9D4E9F9
:10A270000510884202D260690028D5D1002D0CDC7F
:10A28000012000FA06FA40F6340050F8080020EAEF
:10A290000A0040F6340141F808000020BDE8F88FBC
:10A2A00010B50024FBF7EEFB4120FBF7ADFBFBF7FD
:10A2B0003DFC0020FBF772FB0446FBF70DFC20463B
:10A2C00010BD70B504460E46FFF7EAFF05461EB9FD
:10A2D0000120A040854303E00120A0402843C5B2EF
:10A2E000284600F001F870BD10B50446FBF7CAFB24
:10A2F0004020FBF789FBFBF719FC2046FBF784FBAA
:10A30000FBF714FCFBF7E8FB0A2005F0B3FA10BDDD
:10A31000704700002DE9F04104460E4600274848EA
:10A32000006800F00300032802D10120BDE8F0819D
:10A3300043482838006820F0806041492839086087
:10A34000F6F79CFD054606E0F6F798FD401B02284F
:10A3500001D90320EAE73A4828380068C0F3C06012
:10A360000028F1D100BF3648006820F47C30216815
:10A3700040EA013032490860A088401EC0F308005E
:10A38000A168491E4FF47E4202EA41210843A18997
:10A39000491ED20102EA01410843217C491E1202F2
:10A3A00002EA0161084326491031086000BF2448D1
:10A3B000001D006820F0C000616908432049091DA4
:10A3C00008600846006820F02000A16908431C4985
:10A3D000091D08602EB90846006840F40020086096
:10A3E00012E0012E08D11648001D006840F48010CC
:10A3F0001349091D086007E01148001D006840F47A
:10A4000000100F49091D08600D482838006840F009
:10A4100080600B4928390860F6F730FD054606E0F4
:10A42000F6F72CFD401B022801D903207EE70448E3
:10A4300028380068C0F3C0600028F1D0384675E7BE
:10A44000284402582DE9F04104460E4600274848AA
:10A45000006800F00300032802D10120BDE8F0816C
:10A4600043482838006820F0805041492839086066
:10A47000F6F704FD054606E0F6F700FD401B02284E
:10A4800001D90320EAE73A4828380068C0F3407051
:10A490000028F1D100BF3648006820F07C70218888
:10A4A00040EA015032490860A088401EC0F308000D
:10A4B000A168491E4FF47E4202EA41210843A18966
:10A4C000491ED20102EA01410843217C491E1202C1
:10A4D00002EA0161084326491831086000BF244898
:10A4E000001D006820F44060616908432049091D8F
:10A4F00008600846006820F40070A16908431C4900
:10A50000091D08602EB90846006840F48000086004
:10A5100012E0012E08D11648001D006840F400002A
:10A520001349091D086007E01148001D006840F04C
:10A5300080700F49091D08600D482838006840F0F8
:10A5400080500B4928390860F6F798FC054606E06C
:10A55000F6F794FC401B022801D903207EE704484B
:10A5600028380068C0F340700028F1D0384675E7FD
:10A570002844025810B500231B4C236000BF00BFC5
:10A5800000BFBFF34F8F00BF00BF00BF231F18687D
:10A59000C0F34E3100BFC0F3C90200BF43F6E07301
:10A5A00003EA41134FF0404404EA827423430F4C02
:10A5B000236000BF00BF131EA2F10102EED10B1EEB
:10A5C000A1F10101E7D100BF00BF00BFBFF34F8F72
:10A5D00000BF00BF00BF00BF00BF00BFBFF36F8F51
:10A5E00000BF00BF00BF10BD84ED00E074EF00E0CD
:10A5F00010B50023234C236000BF00BF00BFBFF392
:10A600004F8F00BF00BF00BF231F1868C0F34E313B
:10A6100000BFC0F3C90200BF43F6E07303EA411371
:10A620004FF0404404EA82742343174C236000BF78
:10A6300000BF131EA2F10102EED10B1EA1F1010118
:10A64000E7D100BF00BF00BFBFF34F8F00BF00BF07
:10A6500000BF0C4B703B1B6843F48033094C703CCB
:10A66000236000BF00BF00BFBFF34F8F00BF00BF1C
:10A6700000BF00BF00BF00BFBFF36F8F00BF00BFB0
:10A6800000BF10BD84ED00E060EF00E000BF00BF40
:10A6900000BFBFF34F8F00BF00BF00BF00BF00BFB0
:10A6A00000BFBFF36F8F00BF00BF00BF0020144981
:10A6B000086000BF00BF00BFBFF34F8F00BF00BFE7
:10A6C00000BF00BF00BF00BFBFF36F8F00BF00BF60
:10A6D00000BF0C48006840F400300A49086000BF21
:10A6E00000BF00BFBFF34F8F00BF00BF00BF00BF60
:10A6F00000BF00BFBFF36F8F00BF00BF00BF704738
:10A7000050EF00E014ED00E02DE9F04104460F4663
:10A7100015461E46D4F81882A91948F2600050F870
:10A720000800814209D9212305223946204600F03C
:10A73000F6FA4FF0FF30BDE8F0810020FBE70000A3
:10A74000F0B504460D46D4F81862507800F00100C8
:10A7500010B10E4B07210CE0D4F81C02C06905EBC8
:10A76000C50700EB87031879411D1079884200DC8A
:10A770001179718105E0481E81B25F5C06F10C0021
:10A7800047540029F7D10020F0BD0000B858010857
:10A7900070B503460C4615460821D3F8182251819E
:10A7A00006E0481E81B20448465C02F10C004654A3
:10A7B0000029F6D1002070BDC758010870B50346C6
:10A7C0000C461546D3F818220821518106E0481E90
:10A7D00081B20448465C02F10C0046540029F6D1CF
:10A7E000002070BDBF58010870B505460E461446DE
:10A7F0002078232845D00DDC1A2836D005DCB0B1EE
:10A8000003281AD012285AD11DE01B2821D01E2857
:10A8100055D124E02A2846D004DC252837D0282822
:10A820004DD13AE02F2844D05A2848D123E022467F
:10A830003146284600F0A1FA70BD2246314628462E
:10A8400000F01EFAF8E7224631462846FFF778FF67
:10A85000F2E722463146284600F087FAECE7224626
:10A860003146284600F081FAE6E72246314628467E
:10A87000FFF7A4FFE0E7224631462846FFF788FFAE
:10A88000DAE722463146284600F0B5F9D4E72246F9
:10A890003146284600F065F9CEE722463146284683
:10A8A00000F0DDF8C8E722463146284600F0BCFA41
:10A8B000C2E722463146284600F08CFABCE7202346
:10A8C00005223146284600F02AFA4FF0FF30B3E760
:10A8D0002DE9F04706460F46D6F8184248F26800C0
:10A8E0000059B0F5004F03D248F26800005901E06A
:10A8F0004FF40040054648F25E00005BB5FBF0F007
:10A900001FFA80F848F264000159801F005BB1FB18
:10A91000F0F9D6F81C0243464A4604F10C01D0F87F
:10A9200010C03846E047002809DA112304223946CE
:10A93000304600F0F4F94FF0FF30BDE8F087ABB2DD
:10A9400004F10C028121304603F059F948F2640009
:10A950000059411948F264000151001D0059411B82
:10A9600048F26800015148F22C0020448068401BE6
:10A9700048F22C012144886048F26800005908B967
:10A98000032020720020D8E72DE9F04706460F4645
:10A99000D6F8184248F268000059B0F5004F03D2CB
:10A9A00048F26800005901E04FF40040054648F2C3
:10A9B0005E00005BB5FBF0F01FFA80F848F264001F
:10A9C0000159801F005BB1FBF0F9D6F81C02434629
:10A9D0004A4604F10C01D0F814C03846E04700287C
:10A9E00009DA032304223946304600F098F94FF083
:10A9F000FF30BDE8F08748F264000059411948F281
:10AA000064000151001D0059411B48F268000151CA
:10AA100048F22C0020448068401B48F22C0121445D
:10AA2000886048F26800005920B900213046FEF7DE
:10AA300009FF12E048F268000059B0F5004F03D258
:10AA400048F26800005901E04FF4004083B204F17D
:10AA50000C020121304603F021F80020C9E72DE95E
:10AA6000F04106460F461546D6F81842207A0028CF
:10AA70006FD148F20C002044007B00F08000802859
:10AA80000CD048F20C002044417B202305223046A4
:10AA900000F045F94FF0FF30BDE8F081D6F81C0218
:10AAA00081683846884740B13A2302223946304609
:10AAB00000F035F94FF0FF30EEE7A8780006E978AE
:10AAC00040EA0140297940EA01206979084348F2C7
:10AAD00064010851287AE97940EA012148F26800C6
:10AAE0000151005B83B248F2640002593946304696
:10AAF000FFF70AFE002802DA4FF0FF30CCE7022011
:10AB0000207248F26400005948F25E01095B484334
:10AB100048F264010851081D0059891F095B484328
:10AB200048F26801085148F20C002044816848F25C
:10AB30006800005981420CD048F20C002044417B4F
:10AB400020230522304600F0EAF84FF0FF30A3E75B
:10AB5000FFE74FF40040608139463046FFF7B8FE0A
:10AB60009AE72DE9F04105460E461746D5F81842FA
:10AB7000D5F81C02436848F25E002218801C211898
:10AB80003046984748B13A2302223146284600F021
:10AB9000C6F84FF0FF30BDE8F08148F26000005980
:10ABA000401E000E207348F260000059401E010C48
:10ABB000617348F26000005B401E010AA17348F215
:10ABC0006000005D401EE07348F25E00005B01160D
:10ABD000217448F25E00005B0114617448F25E006B
:10ABE000005B0112A17448F25E00015DE17408206F
:10ABF00060810020CFE72DE9FC4105460F469046D5
:10AC0000D5F81842002605E0002104F10C0081551A
:10AC1000701C86B20C2EF7DBD5F81C0201AA69461F
:10AC200043683846984748B13A23022239462846B5
:10AC300000F075F84FF0FF30BDE8FC810821E173AA
:10AC40000098401E010E21740098401E010C617492
:10AC50000098401E010AA1740098401EE074022171
:10AC60002175BDF8040001146175BDF804000112DE
:10AC7000A175BDF80400E0750C2060810020DBE7C1
:10AC800070B504460D46D4F81812002305E00026DE
:10AC900001F10C00C654581CC3B2122BF7DB702014
:10ACA00008730C26CE7448F25C00465C401C405C85
:10ACB00086422BD048F25C00405C48F23C060E44D1
:10ACC00016F830608E7348F25C00405C48F23C0637
:10ACD0000E4406EBC00046790E7648F25C00405CFC
:10ACE00048F23C060E4406EBC00006794E7648F268
:10ACF0005C00405C401CC6B248F25C004654405CBC
:10AD0000042803D1002648F25C00465412204881F2
:10AD10001079122801DC10794881002070BDF0B54F
:10AD20000446D4F8180248F25D052D5C48F23C0652
:10AD3000064406F835201E0248F25D052D5C48F2F7
:10AD40003C07074407EBC5056E6048F25D052D5CC6
:10AD50006D1CEEB248F25D052E542D5C042D03D11E
:10AD6000002648F25D052E54F0BD10B503460C4692
:10AD7000D3F818120020488110BD2DE9F041054696
:10AD80000E461746D5F8184248F20C002044806859
:10AD900060B148F20C002044417B20230522284664
:10ADA000FFF7BDFF4FF0FF30BDE8F081D5F81C0282
:10ADB00081683046884748B13A2302223146284606
:10ADC000FFF7ADFF05202072801FEDE700206081B6
:10ADD00000BFE9E72DE9F04105460F461646D5F8D4
:10ADE0001842707800F00200022809D124230522BD
:10ADF00039462846FFF793FF4FF0FF30BDE8F0815A
:10AE000048F26800005B83B248F264000259394698
:10AE10002846FFF779FC002802DA4FF0FF30EDE713
:10AE20000020608100BFE9E72DE9F04106460F46AA
:10AE30001546D6F81842207A00287BD148F20C003B
:10AE40002044007B00F0800080280CD148F20C00E8
:10AE50002044417B202305223046FFF760FF4FF05E
:10AE6000FF30BDE8F081D6F81C028168384688477B
:10AE700040B13A23022239463046FFF750FF4FF0E7
:10AE8000FF30EEE7D6F81C02C1683846884740B16B
:10AE90002723022239463046FFF741FF4FF0FF30AB
:10AEA000DFE7A8780006E97840EA0140297940EA1E
:10AEB00001206979084348F264010851287AE97948
:10AEC00040EA012148F268000151005B83B248F278
:10AED0006400025939463046FFF716FC002802DAB2
:10AEE0004FF0FF30BDE748F26400005948F25E01C0
:10AEF000095B484348F264010851081D0059891F45
:10AF0000095B484348F26801085148F20C002044AC
:10AF1000816848F26800005981420CD048F20C0068
:10AF20002044417B202305223046FFF7F8FE4FF0F6
:10AF3000FF3096E715E00120207248F268000059C2
:10AF4000B0F5004F03D248F26800005901E04FF419
:10AF5000004083B204F10C020121304602F09EFD54
:10AF600004E039463046FFF70FFD7AE7002078E726
:10AF700070B586B005460C460194372002904FF418
:10AF800080700390002004904FF48050059001A938
:10AF9000284600F039FC41F288323721284600F07B
:10AFA00041FA0646304606B070BD70B586B005461B
:10AFB0000C460194292002904FF4807003900020E9
:10AFC00004904FF48050059001A9284600F01CFC25
:10AFD000284600F02BFB0646304606B070BD70B523
:10AFE00086B005460C4601941020029000010390A3
:10AFF000002004904FF48050059001A9284600F0ED
:10B0000003FC41F288321021284600F00BFA064674
:10B01000304606B070BD70B586B005460C4601944A
:10B02000062002904FF480700390002004904FF4AB
:10B030008050059001A9284600F0E6FB41F28832D5
:10B040000621284600F0EEF90646304606B070BDEF
:10B0500030B585B004460020009001900290039026
:10B060004FF4805004906946204600F0CDFB204606
:10B0700000F0B6F90546284605B030BD30B585B0BC
:10B0800004464FF4D57000900820019040010290D2
:10B09000002003904FF4805004906946204600F051
:10B0A000B3FB204600F044FB0546284605B030BD02
:10B0B00070B586B005460C460194122002904FF4FC
:10B0C00080700390002004904FF48050059001A9F7
:10B0D000284600F099FB41F288321221284600F000
:10B0E000A1F90646304606B070BD70B586B005467B
:10B0F0000C460194112002904FF4807003900020C0
:10B1000004904FF48050059001A9284600F07CFB84
:10B1100041F288321121284600F084F90646304673
:10B1200006B070BDF0B585B0064614461D460094C5
:10B13000072001904FF480700290002003904FF49C
:10B14000805004906946304600F05EFB41F2883240
:10B150000721304600F066F90746384605B0F0BDD5
:10B1600030B585B0044600200090022001904FF4D5
:10B1700040700290002003904FF480500490694684
:10B18000204600F041FB204600F020FA0546284604
:10B1900005B030BD70B586B005460C460194092057
:10B1A00002904FF440700390002004904FF48050C0
:10B1B000059001A9284600F027FB284600F006FA72
:10B1C0000646304606B070BD30B585B00446002056
:10B1D0000090332001904FF4807002900020039083
:10B1E0004FF4805004906946204600F00DFB41F278
:10B1F00088323321204600F015F90546284605B06F
:10B2000030BD70B586B005460C4601940D20029005
:10B210004FF480700390002004904FF4805005900C
:10B2200001A9284600F0F0FA41F288320D212846A3
:10B2300000F0F8F80646304606B070BD70B586B02E
:10B2400005460C4600200190032002904FF48070C8
:10B250000390002004904FF48050059001A92846E7
:10B2600000F0D2FA22460321284600F007FA0646EB
:10B27000304606B070BD30B585B004460020009061
:10B280000D2001904FF480700290002003904FF445
:10B29000805004906946204600F0B6FA41F28832A8
:10B2A0000D21204600F0BEF80546284605B030BD09
:10B2B00030B585B00446002000900C2001904FF47A
:10B2C00080700290002003904FF480500490E0685A
:10B2D00040F08000E060E06820F04000E0606946F7
:10B2E000204600F091FA064A0C21204600F09AF818
:10B2F0000546E06820F08000E060284605B030BDDB
:10B3000000E1F50570B586B005460C4601940620AF
:10B3100002904FF480700390002004904FF480500E
:10B32000059001A9284600F06FFA41F28832062103
:10B33000284600F077F80646304606B070BD70B576
:10B3400086B005460C460194192002904FF4807097
:10B350000390002004904FF48050059001A92846E6
:10B3600000F052FA41F288321921284600F05AF8CA
:10B370000646304606B070BD70B586B005460C4630
:10B380000194182002904FF48070039000200490E4
:10B390004FF48050059001A9284600F035FA41F29B
:10B3A00088321821284600F03DF80646304606B09F
:10B3B00070BD10B50246002308685062486890626C
:10B3C000D1E9020420430C6920434C692043034324
:10B3D000D06A20F0FF001843D062002010BD0000AA
:10B3E00001460E480068C0084FF47A73B0FBF3F0D2
:10B3F00041F2883300FB03F200BF101EA2F10102EC
:10B4000002D14FF000407047486B00F080000028E8
:10B41000F3D0034888630020F5E700000000002413
:10B42000C50020002DE9F04105460E461746644848
:10B430000068C0084FF47A71B0FBF1F000FB07F828
:10B4400000BFB8F10000A8F1010803D14FF000409F
:10B45000BDE8F081686B5B4908400028F1D0686B5B
:10B4600000F0040010B10420A863F1E7686B00F05D
:10B47000010010B10120A863EAE752488030A863B8
:10B48000284600F087F9B04201D00120E0E7002112
:10B49000284600F088F904464B48204008B90020AF
:10B4A000D6E704F00040B0F1004F02D14FF0007039
:10B4B000CEE704F08040B0F1804F01D14020C7E7D3
:10B4C00004F00050B0F1005F01D18020C0E704F02B
:10B4D0008050B0F1805F02D14FF48070B8E704F083
:10B4E0000060B0F1006F02D14FF40070B0E704F0DB
:10B4F0008060B0F1806F02D14FF48060A8E704F063
:10B500008070B0F1807F02D14FF40060A0E704F4B6
:10B510000000B0F5000F02D14FF4805098E704F41A
:10B520008000B0F5800F02D14FF4005090E704F492
:10B530000010B0F5001F02D14FF4804088E704F4FA
:10B540008010B0F5801F02D14FF4004080E704F472
:10B550008020B0F5802F02D14FF4003078E704F45A
:10B560000030B0F5003F02D14FF4802070E704F4C2
:10B570008030B0F5803F02D14FF4002068E704F43A
:10B580000040B0F5004F02D14FF4801060E704F4A2
:10B590008040B0F5804F02D14FF4001058E704F41A
:10B5A0000050B0F5005F02D14FF4800050E704F086
:10B5B0000800082801D100054AE74FF4803047E72A
:10B5C000000000244500200008E0FFFD014615486A
:10B5D0000068C0084FF47A73B0FBF3F041F288338F
:10B5E00000FB03F200BF101EA2F1010202D14FF0D6
:10B5F00000407047486B00F045000028F3D0486BCE
:10B6000000F0040010B104208863F2E7486B00F0FA
:10B61000010010B101208863EBE703488863002034
:10B62000E7E7000000000024C500200001461148A3
:10B630000068C0084FF47A73B0FBF3F041F288332E
:10B6400000FB03F200BF101EA2F1010202D14FF075
:10B6500000407047486B00F045000028F3D0486B6D
:10B6600000F0040010B104208863F2E70248886308
:10B670000020EEE700000024C50020002DE9F04185
:10B6800004460E46174628480068C0084FF47A71F1
:10B69000B0FBF1F041F2883100FB01F800BFB8F1D6
:10B6A0000000A8F1010803D14FF00040BDE8F0818F
:10B6B000606B00F045000028F1D0606B00F00400E2
:10B6C00010B10420A063F1E7606B00F0010010B13D
:10B6D0000120A063EAE7204600F05CF8B04201D008
:10B6E0000120E3E71148A0630021204600F05BF849
:10B6F000054605F4604018B9280C38800020D5E7CD
:10B7000005F48040B0F5804F02D14FF40050CDE7F2
:10B7100005F40040B0F5004F02D14FF48050C5E76A
:10B720004FF48030C2E7000000000024C500200074
:10B73000014617480068C0084FF47A73B0FBF3F075
:10B7400041F2883300FB03F200BF101EA2F1010298
:10B7500002D14FF000407047486B00F045000028D0
:10B76000F3D0486B00F0040010B104208863F2E7C6
:10B77000486B00F0010010B101208863EBE7486BD3
:10B7800000F0400008B1402088630020E3E700009B
:10B790000000002401460869C0B2704701460868ED
:10B7A00000F003007047024602F1140043181868C5
:10B7B000704700000FB410B504460021DDE9030214
:10B7C0001043059A1043069A1043079A1043014309
:10B7D0006068044A104008436060002010BC5DF8B7
:10B7E00014FB0000002CFCFF10B50446206840F05C
:10B7F000030020600220F5F7EBF9002010BD0146A0
:10B80000D1F880007047000010B502460023086898
:10B810009060D1E901042043CC6820430C692043A7
:10B820000343D068024C20401843D060002010BD74
:10B83000C0E0FEFF02460868C2F8800000207047A2
:10B8400000B587B0164817490860002048600121FC
:10B85000144881600821C1602021016140214161BB
:10B86000890081610021C1614FF4006101624900DA
:10B870004162002181620220009008200190062090
:10B8800002900390022004900590069069460548B6
:10B89000F8F7BAFB034800F007F807B000BD000056
:10B8A000404100524406002470B5054600240023A0
:10B8B00001221146184600F021F84FF4FA7003F007
:10B8C000E5FF002301220221184600F017F80023AB
:10B8D00008220321184600F011F840F222242346E2
:10B8E00001220421002000F009F840F2A5210248BD
:10B8F000F8F77CFC70BD0000440600242DE9FF41F0
:10B9000004460D4616461F464FF0000814B94FF086
:10B91000100803E0012C01D14FF008080095CDF884
:10B920000480029603974FF6FF7269460448F8F7C1
:10B9300071FC18B9002004B0BDE8F0810120FAE7DD
:10B94000440600242DE9F04389B004460F46F5F77C
:10B9500095FA81464FF000080020019002903E4683
:10B9600008212068FFF73BFB05461DB1284609B0BA
:10B97000BDE8F0834422125B11042068FFF7F8FA57
:10B9800005460DB12846F2E74FF0FF30039008203E
:10B99000049030200590022006900020079001209E
:10B9A000089003A92068FFF704FD2068FFF70CFC4E
:10B9B00005460DB12846DAE71AE02068406B00F42E
:10B9C000002060B9B8F1000F09D12068FFF717FF18
:10B9D00001902068FFF713FF029008F10108F5F7C6
:10B9E0004DFAA0EB0900401C10B94FF00040BEE733
:10B9F0002068406B40F22A5108400028DDD02068C2
:10BA0000406B00F0080018B1082021688863AEE799
:10BA10002068406B00F0020018B1022021688863A2
:10BA2000A5E72068406B00F0200018B120202168B5
:10BA300088639CE71248216888630298000602998F
:10BA400001F47F4140EA0120029901F47F0140EABC
:10BA50001120029940EA11603060361D01980006FD
:10BA6000019901F47F4140EA0120019901F47F012D
:10BA700040EA1120019940EA11603060002076E729
:10BA80003A0F001810B50448F8F73FFD042801D01C
:10BA9000012010BD0020FCE7FC0700242DE9F04147
:10BAA00096B00446002540216846F4F763FC002761
:10BAB000F5F7E4F98046A06D20B94FF0806016B02C
:10BAC000BDE8F081A06DB0F5807F7DD100202168B8
:10BAD000C86240212068FFF782FA05460DB128466A
:10BAE000EDE74FF0FF301090402011906020129051
:10BAF00002201390002014900120159010A92068B6
:10BB0000FFF757FC10B14FF48030D8E72F49206879
:10BB1000FFF7F8FB05460DB12846D0E720E0206886
:10BB2000406B00F4004068B1002608E02068FFF791
:10BB300066FE082101FB07614DF82100761C082EE6
:10BB4000F4D37F1CF5F79AF9A0EB0800401C38B934
:10BB50004FF000406063012084F83000C007AEE77A
:10BB60002068406B40F22A5108400028D7D0206856
:10BB7000406B00F0080028B1082021688863002588
:10BB800028469CE72068406B00F0020028B10220A4
:10BB9000216888630225284691E72068406B00F001
:10BBA000200030B12020216888632025284686E7C0
:10BBB0000AE00748216888639DF80D0000F0020044
:10BBC000022801D04FF08055284678E701FFFF801A
:10BBD000FF0FE01F10B50D480D49086000204860B8
:10BBE00000210B4881604FF48041C1600021016158
:10BBF00004214161F8F7FAFC04460CB1012010BDA4
:10BC000004490348F8F76EFC0020F8E70070005282
:10BC1000FC0700247808002430B58DB004460120CC
:10BC200001902068FFF7BAFD18B94FF080600DB0A1
:10BC300030BDA06B03281AD02068FFF791FA0546A3
:10BC40000DB12846F3E700212068FFF7ACFDE06660
:10BC500004212068FFF7A7FD206708212068FFF76F
:10BC6000A2FD60670C212068FFF79DFDA067A06B17
:10BC7000032807D001A92068FFF7E0FA05460DB1B7
:10BC80002846D4E7A06B032820D0BDF804106164D7
:10BC90004422125B11042068FFF77CFA05460DB1BF
:10BCA0002846C4E700212068FFF77DFDE0650421F8
:10BCB0002068FFF778FD206608212068FFF773FDF4
:10BCC00060660C212068FFF76EFDA06604212068E5
:10BCD000FFF769FD010D216402A92046F8F71EFB5C
:10BCE00010B14FF08050A2E74420005B01040A46E7
:10BCF00000232068FFF716FA05460DB1284696E79F
:10BD0000002094E7F8B504460020009000260027A4
:10BD10002068FFF79DF905460DB12846F8BD20685B
:10BD2000FFF7ACF9054615B10021E16301E00121FF
:10BD3000E16300212068FFF71BF9054615B14FF0BC
:10BD40008050EBE71DE000212068FFF711F9054660
:10BD50000DB12846E2E717492068FFF726F90546A6
:10BD600015B14FF08050D9E700212068FFF71BFD87
:10BD70000646012080EAD67080F001070098401C3A
:10BD800000904FF6FF710098884201D2002FDAD060
:10BD90004FF6FF710098884202D34FF08070BDE7E4
:10BDA00006F08040B0F1804F01D10120A063002057
:10BDB000B4E70000000010C12DE9F84605460C4626
:10BDC00016464FF00009DFF840A02746F4F76FFA57
:10BDD000504633463A46294600900C48F8F7F8FC9E
:10BDE000814607E0BAF10000AAF1010A02D14FF042
:10BDF000010903E0FFF746FE0028F3D100BFF4F786
:10BE000058FA4846BDE8F88600E1F505FC0700242D
:10BE10002DE9F04387B004460F46F5F72FF880462A
:10BE20003E4600212068FFF7BEFC00F00070B0F134
:10BE3000007F04D14FF4006007B0BDE8F0834021DB
:10BE40002068FFF7CCF805461DB1606B606328469B
:10BE5000F2E74422125B11042068FFF789F80546D7
:10BE60001DB1606B60632846E6E74FF0FF3001903C
:10BE70004020029060200390022004900020059052
:10BE80000120069001A92068FFF793FA2068FFF7C8
:10BE9000F2F905461DB1606B60632846CCE71AE0F5
:10BEA0002068406B00F4004060B14FF0000906E0EC
:10BEB0002068FFF7A4FC3060361D09F10109B9F1D3
:10BEC000080FF5D3F4F7DAFFA0EB0800401C10B917
:10BED0004FF00040B0E72068406B00F495700028F8
:10BEE000DED02068406B00F0080008B10820A3E70E
:10BEF0002068406B00F0020008B102209CE7206837
:10BF0000406B00F0200008B1202095E70DE020688C
:10BF1000FFF775FC3060361DF4F7B0FFA0EB0800AA
:10BF2000401C10B94FF0004086E72068406B00F4D9
:10BF300000500028EBD102482168886300207BE78D
:10BF40003A0F001870B504460D4615B94FF0006061
:10BF500070BD4422125B11042068FFF752F90646B7
:10BF60000EB13046F4E700212068FFF71CFC286082
:10BF70000020EDE77CB504460020009001900021F0
:10BF80002068FFF710FC00F00070B0F1007F02D1D4
:10BF90004FF400607CBD69462046FFF7D3FC0546A0
:10BFA0000DB12846F6E7019800F4803098B144229C
:10BFB000125B11042068FEF7DBFF05460DB1284631
:10BFC000E8E700212068FFF726F805460DB128466E
:10BFD000E0E70020DEE74FF08060DBE77CB5044659
:10BFE00000200090019000212068FFF7DCFB00F0AA
:10BFF0000070B0F1007F02D14FF400607CBD694653
:10C000002046FFF79FFC05460DB12846F6E701984C
:10C0100000F4802098B14422125B11042068FEF7DE
:10C02000A7FF05460DB12846E8E702212068FEF784
:10C03000F2FF05460DB12846E0E70020DEE74FF0AD
:10C040008060DBE72DE9F84605460C4616464FF0C2
:10C050000009DFF840A02746F4F729F95046334697
:10C060003A46294600900C48F8F7C8FC814607E09C
:10C07000BAF10000AAF1010A02D14FF0010903E070
:10C08000FFF700FD0028F3D100BFF4F712F948468E
:10C09000BDE8F88600E1F505FC07002410B5174857
:10C0A000174908604FF480004860002114488160FF
:10C0B0000721C1604FF000710161491041618900A1
:10C0C0008161002141634FF0004141654FF0E04143
:10C0D000C16100210162416281620721C162F8F7FA
:10C0E000A9FD07480068006840F00100044909689C
:10C0F0000860FF2000F006F810BD00000038004086
:10C10000280C002401B582B04FF47A70012301AAF3
:10C1100002A900900248F8F7FDFE9DF804000EBD4C
:10C12000280C00240F490968096821F001010D4A13
:10C13000126811600B490968896821F0E041094AD9
:10C14000126891600749096889680143054A1268C5
:10C15000916004490968096841F00101014A1268C7
:10C1600011607047280C00240268516902689269C6
:10C1700042F0080203689A610268926942F0100274
:10C1800003689A610268126822F0010203681A606B
:10C190000268126940F26B339A4303681A610268BD
:10C1A000926822F4404203689A6090F88120042A41
:10C1B0000ED001F020025AB1D0F8842042F0800263
:10C1C000C0F884200268926942F0200203689A61F4
:10C1D00090F88120032A21D001F040025AB1D0F812
:10C1E000842042F00402C0F884200268926942F080
:10C1F000400203689A61826AB2F5800F0ED101F0A5
:10C2000080025AB1D0F8842042F00202C0F88420A3
:10C210000268926942F0800203689A6101F4007238
:10C220005AB1D0F8842042F00102C0F8842002689C
:10C23000926942F4007203689A6101F480725AB103
:10C24000D0F8842042F00802C0F884200268926985
:10C2500042F4807203689A610022A0F86220A0F87C
:10C260006A20704710B501460124C86B04EB5013D7
:10C27000C868421CD01DC20802FB03F010BD2DE9A6
:10C28000F04106460C4617469846069D0BE0681C92
:10C2900048B12DB1F4F7F2FDA0EB0800A84202D995
:10C2A0000320BDE8F081306840692040A04201D100
:10C2B000012000E00020B842E9D00020F1E70000B2
:10C2C000F0B589B006460C4615464FF0FF3716B15B
:10C2D000012E11D106E04FF4007028804FF4484041
:10C2E000206009E069460648F8F7FCF80698401E09
:10C2F00020600798288000BF00BF002009B0F0BD73
:10C30000FC07002400B589B069460548F8F7EAF84B
:10C31000069810B1012009B000BD0020FBE7000025
:10C32000FC07002470B50446002514B1012C07D188
:10C3300002E002F07BFE03E0FFF74CFC054600BF85
:10C3400000BF68B270BD000001460020034A1278A9
:10C3500042F01002014B1A70704700006C0200247A
:10C3600001460020704700002DE9F04106460F46C7
:10C3700015461C464FF000081348007840F00200B4
:10C380001149087016B1012E11D108E04FF6FF7067
:10C3900000EA44226902384602F096FE07E022468F
:10C3A00029463846FFF708FD4FFA80F800BF00BF66
:10C3B000B8F1000F05D00448007840F008000249A9
:10C3C00008704046BDE8F0816C0200242DE9F04180
:10C3D00006460F4615461C464FF0000813480078E5
:10C3E00040F001001149087016B1012E11D108E08A
:10C3F0004FF6FF7000EA44226902384602F0F6FE6A
:10C4000007E0224629463846FFF71CFE4FFA80F81F
:10C4100000BF00BFB8F1000F05D00448007840F01D
:10C420000400024908704046BDE8F0816C02002417
:10C43000704700002DE9F0419CB080460C4615463F
:10C440001E4600273948006820F00400374908607C
:10C4500000BF0020009035480C30006840F4404098
:10C4600032490C3108600846006800F440400090F2
:10C4700000BF00BF00BF2D480C30006800F4005022
:10C48000B0F5005FF7D1212001904FF48030029089
:10C490000120079000200490089002200A900221B9
:10C4A0000B91CDF834800C940E950F9600211291CB
:10C4B000082111910021139101A8F7F743FA0746CB
:10C4C0000FB100BFFEE73F2014900320159000201D
:10C4D0001690082017904020199000011A904020D3
:10C4E000189050201B90022114A8F6F799FF0746D8
:10C4F0000FB100BFFEE70E48006840F080000C4915
:10C50000086000BF0A48F430006840F002000849A3
:10C51000F43108600846006800F00200009000BF97
:10C5200000BFF4F769FB1CB0BDE8F0810C4802586D
:10C530000044025810B5F4F7A7FC10BD204800686D
:10C5400040F470001E4908601E48006840F0010079
:10C550001C49086000201B49103108601948006818
:10C560001949084017490860002016491831086029
:10C57000091D0860091D0860124928310860091D5D
:10C580000860091D0860091D0860091D0860091D73
:10C590000860091D0860091D08600A48006820F449
:10C5A00080200849086000200649603108600120A9
:10C5B00006490860C00602498039086070470000DB
:10C5C00088ED00E0004402587FEDF6EA0881005152
:10C5D00010B50E480068C06800F0010078B10C4941
:10C5E00008698047002009490968486200BF642043
:10C5F00006490968C86264210448C16000BF6FF041
:10C60000010002490968086110BD0000B01C002447
:10C610006000002410B500220288294B98420ED0F9
:10C62000B0F1804F0BD0274B984208D0264B984250
:10C6300005D0264B984202D0254B984203D122F0D8
:10C6400070024B681A431E4B984217D0B0F1804FCE
:10C6500014D01C4B984211D01B4B98420ED01B4B50
:10C6600098420BD01A4B984208D01A4B984205D0EA
:10C67000194B984202D0194B984203D122F44072D0
:10C68000CB681A4322F080034C6943EA040202801B
:10C690008B68C3620B880385094B98420BD00C4B07
:10C6A000984208D00B4B984205D00B4B984202D0D1
:10C6B0000A4B984201D10B8A03860123436110BDC6
:10C6C000000001400004004000080040000C004051
:10C6D0000004014000400140004401400048014086
:10C6E00038B504460D4600BF1148006840F004000C
:10C6F0000F4908600846006800F00400009000BF81
:10C7000000BF032211461E20F4F7BEFE1E20F4F7E0
:10C71000ABFE084808490860084645600021816072
:10C72000C4600161F8F792FE0348F8F7AAFE38BD2D
:10C73000E844025800080040B01C002490F834106F
:10C7400001F0010139B10168496821F40031826BBF
:10C7500011430268516090F8341001F0020139B1C0
:10C760000168496821F48031C26B1143026851604D
:10C7700090F8341001F0040139B10168496821F4DE
:10C780008021026C11430268516090F8341001F06E
:10C79000080139B10168496821F40041426C114334
:10C7A0000268516090F8341001F0100139B101684D
:10C7B000896821F48051826C11430268916090F87D
:10C7C000341001F0200139B10168896821F4005169
:10C7D000C26C11430268916090F8341001F040017E
:10C7E00099B10168496821F48011026D1143026812
:10C7F0005160016DB1F5801F07D10168496821F4CE
:10C80000C001426D11430268516090F8341001F08C
:10C81000800139B10168496821F40021826D11431A
:10C8200002685160704738B5044600250020E06773
:10C83000F4F724FB05462068006800F0080008288B
:10C840000CD16FF07E402B4600224FF40011009077
:10C85000204600F0A6FD08B1032038BD206800681E
:10C8600000F0040004280CD16FF07E402B4600221B
:10C870004FF480010090204600F093FD08B10320A2
:10C88000EBE7202084F8790084F87A0000BF0020CC
:10C8900084F8780000BF00BFDFE770B50546AC6BD9
:10C8A0000020A4F86A00A4F862002046F8F7F9FD19
:10C8B00070BD0168096821F4907102681160016817
:10C8C000896821F0010102689160202180F87A10C6
:10C8D000704710B504462068006820F040002168C9
:10C8E0000860202084F879002046F8F7FFFF002038
:10C8F00010BD2DE9F0410446B4F86C7094F87A004C
:10C90000222833D12068858CA068B0F5805F09D1DA
:10C91000206938B9666E05EA07003080606E801CB9
:10C92000606605E0F8B22840626E511C61661070C6
:10C93000B4F86A00401E80B2A4F86A00A0B920686A
:10C94000006820F49070216808602068806820F0FA
:10C95000010021688860202084F87A002046F8F7DA
:10C9600081FF0020BDE8F0810020FBE72068008BFC
:10C9700040F00800216808830220F3E72DE9F04F1A
:10C9800089B0044600254FF08008A946AA46002039
:10C990000890FA492068884201D1012000E0002077
:10C9A00000B100E000BFA06AB0F1005F00D100BF9D
:10C9B0002169A068084361690843E16940EA01050B
:10C9C000A06A054320680068ED49084028432168B3
:10C9D00008602068406820F44050E16808432168FE
:10C9E0004860A569E5492068884201D1012000E03E
:10C9F000002008B9206A0543A06AB0F1005F03D1A6
:10CA0000D4E90B010843054320688068DD490840EC
:10CA10002843216888602068C06A20F00F00616A9E
:10CA200008432168C86200BFD7492068884224D1E2
:10CA3000D648006800F03800182814D005DC48B14A
:10CA400008280AD0102817D10AE020280ED028285C
:10CA500012D10EE04FF001080EE04FF004080BE099
:10CA60004FF0400808E04FF0080805E04FF01008CC
:10CA700002E04FF0200800BF17E1C5492068884256
:10CA80001DD1C248006800F00700062816D2DFE872
:10CA900000F00306090C0F124FF000080EE04FF0F3
:10CAA00004080BE04FF0400808E04FF0080805E0EC
:10CAB0004FF0100802E04FF0200800BFF5E0B54944
:10CAC000206888421DD1B148006800F007000628A0
:10CAD00016D2DFE800F00306090C0F124FF0000831
:10CAE0000EE04FF004080BE04FF0400808E04FF074
:10CAF000080805E04FF0100802E04FF0200800BFE2
:10CB0000D3E0A549206888421DD1A048006800F004
:10CB10000700062816D2DFE800F00306090C0F1202
:10CB20004FF000080EE04FF004080BE04FF0400813
:10CB300008E04FF0080805E04FF0100802E04FF061
:10CB4000200800BFB1E09549206888421DD18F4878
:10CB5000006800F00700062816D2DFE800F00306A0
:10CB6000090C0F124FF000080EE04FF004080BE024
:10CB70004FF0400808E04FF0080805E04FF01008BB
:10CB800002E04FF0200800BF8FE08549206888420E
:10CB900024D17E48006800F03800182814D005DC45
:10CBA00048B108280AD0102817D10AE020280ED052
:10CBB000282812D10EE04FF001080EE04FF00408D3
:10CBC0000BE04FF0400808E04FF0080805E04FF098
:10CBD000100802E04FF0200800BF66E071492068AD
:10CBE00088421DD16948006800F00700062816D267
:10CBF000DFE800F00306090C0F124FF000080EE00A
:10CC00004FF004080BE04FF0400808E04FF0080830
:10CC100005E04FF0100802E04FF0200800BF44E0AC
:10CC20006149206888421DD15848006800F007001B
:10CC3000062816D2DFE800F00306090C0F124FF0A9
:10CC400000080EE04FF004080BE04FF0400808E049
:10CC50004FF0080805E04FF0100802E04FF0200800
:10CC600000BF22E04549206888421ED14748001D88
:10CC7000006800F00700062816D2DFE800F003067F
:10CC8000090C0F124FF002080EE04FF004080BE001
:10CC90004FF0400808E04FF0080805E04FF010089A
:10CCA00002E04FF0200800BF00BF00BF33492068FA
:10CCB000884201D1012000E0002000285DD000253D
:10CCC000B8F1100F33D009DCB8F1020F10D0B8F171
:10CCD000040F11D0B8F1080F2ED117E0B8F1200FD2
:10CCE00027D0B8F1400F0CD0B8F1800F24D124E048
:10CCF000F5F7B8FB054623E005A8F5F7C9FB069D47
:10CD00001EE002A8F5F7DAFC039D19E01F4854382D
:10CD10000068C0F3401040B11C4854380068C0F3AC
:10CD2000C101224820FA01F500E0204D08E0204D25
:10CD300006E04FF4004503E000BF0120089000BF6B
:10CD400000BF002D0AD0606800EB4000A84203D865
:10CD500060680003A84202D201200890D4E2B8F132
:10CD6000100F7CD026DCB8F1020F2DD0B8F1040FE3
:10CD700052D0B8F1080F73D19EE03FE1000C00588B
:10CD8000F369FFCFFFF4FF11001001405444025833
:10CD90000044004000480040004C0040005000406B
:10CDA0000014014000780040007C00400090D00357
:10CDB00000093D00B8F1200F7DD0B8F1400F54D0EC
:10CDC000B8F1800FD7D109E1F5F74CFB00270646F3
:10CDD000FB49606A31F810C062463B46304639462E
:10CDE000F3F77EFA4FF4807600220346A3FB060792
:10CDF00001FB067103FB02136168490806467118BE
:10CE00005A41CDE90012666832460023084601996E
:10CE1000F3F766FA0546E4E005A8F5F739FBDDF817
:10CE200018C0E749606A31F810B05A4600236046DE
:10CE30001946F3F755FA4FF4807C0022A0FB0C3B17
:10CE400001FB0CB100FB0210616849085E1840EB61
:10CE50000201D4F804C062460023304601E079E0C4
:10CE6000BBE0F3F73DFA0546BBE002A8F5F726FC68
:10CE7000DDF80CC0D249606A31F810B05A46002380
:10CE800060461946F3F72CFA4FF4807C0022A0FB91
:10CE90000C3B01FB0CB100FB0210616849085E18F5
:10CEA00040EB0201D4F804C0624600233046F3F799
:10CEB00017FA054695E06EE0C2480068C0F34010DE
:10CEC00038B3C0480068C0F3C101BF4820FA01FC74
:10CED000BB49606A31F810B05A46002360461946D3
:10CEE000F3F7FEF94FF4807C0022A0FB0C3B01FB22
:10CEF0000CB100FB0210616849085E1840EB0201AA
:10CF0000D4F804C0624600233046F3F7E9F9054639
:10CF10001FE0AB49606A31F810C062460023AA489E
:10CF20001946F3F7DDF94FF4807C0022A0FB0C3B9F
:10CF300001FB0CB100FB0210616849085E1840EB70
:10CF40000201D4F804C0624600233046F3F7C8F962
:10CF5000054646E09A49606A31F810C062460023EF
:10CF60009A481946F3F7BCF94FF4807C0022A0FBE5
:10CF70000C3B01FB0CB100FB0210616849085E1814
:10CF800040EB0201D4F804C0624600233046F3F7B8
:10CF9000A7F9054625E08A49606A31F810C0624663
:10CFA00000234FF400401946F3F79AF94FF4807CC0
:10CFB0000022A0FB0C3B01FB0CB100FB02106168DE
:10CFC00049085E1840EB0201D4F804C06246002311
:10CFD0003046F3F785F9054603E000BF01200890CD
:10CFE00000BF00BFB5F5407F05D3B5F5801F02D265
:10CFF0002068C56088E10120089085E1E069B0F50E
:10D00000004F7CD1B8F1100F7AD00CDCB8F1000FD2
:10D0100013D0B8F1010F21D0B8F1040F2FD0B8F11F
:10D02000080F6ED151E0B8F1200F6BD0B8F1400F6E
:10D0300038D0B8F1800F64D197E0F6F735FB604A3D
:10D04000616A32F81110B0FBF1F04000616800EB4A
:10D050005100B0FBF1F01FFA80FA89E0F6F73AFBD5
:10D06000574A616A32F81110B0FBF1F04000616874
:10D0700000EB5100B0FBF1F01FFA80FA78E005A850
:10D08000F5F706FA06994E4A606A32F81000B1FBCD
:10D09000F0F04000616800EB5100B0FBF1F01FFAC6
:10D0A00080FA65E002A8F5F709FB0399444A606A33
:10D0B00032F81000B1FBF0F04000616800EB510065
:10D0C000B0FBF1F01FFA80FA52E03E480068C0F36E
:10D0D0004010C0B13B480068C0F3C1013A48C840A5
:10D0E000374A616A32F81110B0FBF1F04000616814
:10D0F00000EB5100B0FBF1F01FFA80FA12E044E0BF
:10D1000011E031E01FE02E49606A31F810002E492D
:10D11000B1FBF0F04000616800EB5100B0FBF1F0B2
:10D120001FFA80FA24E02649606A31F81000274986
:10D13000B1FBF0F04000616800EB5100B0FBF1F092
:10D140001FFA80FA14E01E49606A31F810004FF4AB
:10D150000041B1FBF0F04000616800EB5100B0FB12
:10D16000F1F01FFA80FA03E000BF0120089000BF31
:10D1700000BF4FF6F0700AEA0009CAF3420049EA1C
:10D1800000092068C0F80C90BEE0B8F1100F7CD008
:10D190000CDCB8F1000F1BD0B8F1010F29D0B8F1A9
:10D1A000040F37D0B8F1080F70D159E0B8F1200F53
:10D1B0006DD0B8F1400F40D0B8F1800F66D19FE03C
:10D1C000F4100108004402580090D00300093D000B
:10D1D000F6F76AFA4E4A616A32F81110B0FBF1F0C4
:10D1E000616800EB5100B0FBF1F080B22168C860CB
:10D1F00089E0F6F76FFA464A616A32F81110B0FB1F
:10D20000F1F0616800EB5100B0FBF1F080B22168F1
:10D21000C86078E005A8F5F73BF906993C4A606AD2
:10D2200032F81000B1FBF0F0616800EB5100B0FB88
:10D23000F1F080B22168C86065E002A8F5F73EFA17
:10D240000399334A606A32F81000B1FBF0F061686C
:10D2500000EB5100B0FBF1F080B22168C86052E0F1
:10D260002C480068C0F34010C0B12A480068C0F3E1
:10D27000C1012948C840264A616A32F81110B0FB42
:10D28000F1F0616800EB510002E017E037E025E0C3
:10D29000B0FBF1F080B22168C8600EE01C49606A02
:10D2A00031F810001C49B1FBF0F0616800EB51004F
:10D2B000B0FBF1F080B22168C86024E01449606AD4
:10D2C00031F810001549B1FBF0F0616800EB510036
:10D2D000B0FBF1F080B22168C86014E00C49606ACC
:10D2E00031F810004FF40041B1FBF0F0616800EB41
:10D2F0005100B0FBF1F080B22168C86003E000BFCC
:10D300000120089000BF00BF089809B0BDE8F08F69
:10D31000F4100108004402580090D00300093D00B9
:10D32000014691F87900212839D1B1F86200C8B9D5
:10D330000868006800F0005030B10868806820F488
:10D3400000000B68986005E00868006820F0800025
:10D350000B6818600868006840F040000B681860AF
:10D36000002070478868B0F5805F0BD1086948B924
:10D37000CA6D1088C0F308000B681885C86D801C42
:10D38000C86505E0CB6D581CC86518780B68188512
:10D39000B1F86200401EA1F862000020E1E702201F
:10D3A000DFE72DE9F04104460D4617469846069EF4
:10D3B00021E0701CF8B12EB1F3F760FDA0EB08007E
:10D3C000B04218D92068006820F4D0702168086045
:10D3D0002068806820F0010021688860202084F89F
:10D3E000790084F87A0000BF002084F8780000BF3C
:10D3F0000320BDE8F0812068C0692840A84201D11F
:10D40000012000E00020B842D3D00020F1E7000066
:10D4100070B500240F4D1048F8F74EF800BF03E038
:10D42000641CAC4200D904E00B48F8F73BF8202814
:10D43000F6D100BF002403E0641CAC4200D906E032
:10D44000012206490448F8F79DF90028F4D100BFED
:10D4500070BD0000FFFF0100C4050024120000247D
:10D4600070B504460D46D4F8140229464268204699
:10D470009047002070BD70B504460D4694F8FC013D
:10D48000022802D0032811D100E000BF68880128DB
:10D490000BD10020C4F80402D4F814022946826893
:10D4A00020469047204600F04AF804E029462046EE
:10D4B00000F01BF800BF00BF70BD70B506460C46FB
:10D4C00015462B4622460021304600F0E7FA0020A0
:10D4D00070BD70B506460C4615462B462246002107
:10D4E000304600F08CFB002070BD70B504460D4640
:10D4F0008021204600F067FB0021204600F063FBFE
:10D5000070BD10B504460520C4F8F40100231A4686
:10D510001946204600F0C2FA002010BD70B504463E
:10D520000E4615460220C4F8F401A561E5612B46BC
:10D5300032460021204600F062FB002070BD10B58D
:10D5400004460420C4F8F40100231A461946204674
:10D5500000F055FB002010BD70B504460D46E8886C
:10D56000012804D029462046FFF7BFFF1BE094F8AE
:10D57000FC01022802D003280FD108E00020A0609F
:10D58000012204F108012046FFF7C8FF0AE001224A
:10D59000211D2046FFF7C2FF04E029462046FFF781
:10D5A000A4FF00BF00BF70BDF8B504460E467088EA
:10D5B000001208287FD2DFE800F07E040C207E7E77
:10D5C0005F6D207CD4F810120A68694690470546C2
:10D5D00076E0207C40B9D4F81402816A6846884716
:10D5E00005460221697007E0D4F81402C16A684652
:10D5F000884705460221697062E0B078062834D277
:10D60000DFE800F0030B131B232B207CD4F810124F
:10D610004A686946904705462CE0207CD4F81012F1
:10D620008A6869469047054624E0207CD4F81012A9
:10D63000CA686946904705461CE0207CD4F8101261
:10D640000A6969469047054614E0207CD4F8101218
:10D650004A696946904705460CE0207CD4F81012D0
:10D660008A6969469047054604E031462046FFF73F
:10D670003CFFF8BD00BF23E0207C30B9D4F8140291
:10D68000416B6846884705461AE031462046FFF759
:10D690002CFFEEE7207C48B9D4F81402016B6846F1
:10D6A00088470546072169700AE004E031462046B4
:10D6B000FFF71BFFDDE731462046FFF716FFD8E7EF
:10D6C00000BFBDF8000088B1F08878B1F088BDF8DF
:10D6D0000010884202DDBDF8000000E0F0880090F4
:10D6E000BDF8002029462046FFF718FF00BFC0E71D
:10D6F0000146002002E0421CD0B2491C0A78002AF0
:10D70000F9D1704770B504460D4694F8FC01022823
:10D7100002D0032811D100E000BF0120E060D4F85E
:10D72000040218B1E06840F00200E060022204F157
:10D730000C012046FFF7F2FE04E029462046FFF7E1
:10D74000D4FE00BF00BF70BD2DE9F04104460D4678
:10D7500017460026FCB12046FFF7CAFF022101EB65
:10D76000400038803A783046711CCEB22A540322E9
:10D770003046711CCEB22A540AE014F8012B304610
:10D78000711CCEB22A5400223046711CCEB22A54EB
:10D7900020780028F1D1BDE8F081000070B5044682
:10D7A0000D46164654B90EA001F0ECFD0EA001F096
:10D7B000E9FD13A001F0E6FD022070BDD4F81402CB
:10D7C00010B10020C4F814020DB1C4F810520120A9
:10D7D00084F8FC012670204600F0FCF80020ECE7FD
:10D7E0004552524F523A2000496E76616C6964206E
:10D7F0004465766963652068616E646C650000004D
:10D800000D0A000070B504460D462946D4F82002E2
:10D81000F3F760FF002070BD70B504460D46294641
:10D82000D4F82002F3F720FF002070BD2DE9F0416D
:10D8300004460E461746002E54D104F11405D4F8C0
:10D84000F401022843D1D5E90201884210D9D5E973
:10D850000201401AA860288982B239462046FFF7A3
:10D8600038FE00231A461946204600F017F92EE02C
:10D87000E9686868B0FBF1F201FB1200B8B9E96829
:10D880006868884213D36868D4F8F81188420ED2C9
:10D89000002211462046FFF71CFE0020C4F8F801C4
:10D8A00000231A461946204600F0F8F80FE0D4F895
:10D8B0001402C06840B194F8FC01032804D1D4F8E4
:10D8C0001402C168204688472046FFF71AFE94F8E4
:10D8D0000002012814D1204600F08EFB002084F8BD
:10D8E00000020DE0D4F81402406948B194F8FC013C
:10D8F000032805D1D4F814023146426920469047E6
:10D900000020BDE8F0812DE9F04105460E4617469E
:10D910005EBB05F58274D5F8F401032833D1D4E950
:10D920000201884210D9D4E90201401AA060D4E96A
:10D930000201884201D2A06800E0E06882B2394664
:10D940002846FFF7BAFD1EE0D5F81402006940B181
:10D9500095F8FC01032804D1D5F814020169284682
:10D9600088472846FFF7EBFD0DE0D5F814028069E3
:10D9700048B195F8FC01032805D1D5F814023146C9
:10D980008269284690470020BDE8F08101460020CA
:10D99000704710B50446012084F8FC012179D4F8C1
:10D9A0001402426820469047002010BD70B504461E
:10D9B0000D462946D4F82002F3F7C1FE002070BDC1
:10D9C00070B504460D462946D4F82002F3F7D9FE77
:10D9D00070BD000010B504461548164908600820BF
:10D9E0004860002113480163402141610021016228
:10D9F000022181610021C1610221C1600021C16257
:10DA00008162C0F8FC43C4F82002F4F751FB802186
:10DA10000848F3F7B0FD402200210648F3F7B0FDB7
:10DA2000802201210348F3F7ABFD002010BD000068
:10DA300000000840006F032410B50246D2F82032DF
:10DA400001F08000802809D101F07F00C0EBC00404
:10DA500003F1380000EB8400807810BD01F07F00F6
:10DA6000C0EBC00403F5FC7000EB84008078F4E7A1
:10DA70000246002070470246002070472DE9F04121
:10DA800004460F4615461E462B4632463946D4F804
:10DA90002002F3F782FE0020BDE8F0812DE9F0417D
:10DAA00004460D4616461F463B4632462946D4F8E4
:10DAB0002002F3F7B9FE0020BDE8F08110B504465E
:10DAC0004023002211462046FFF7D8FF40214FF4A3
:10DAD000887001514023002280212046FFF7CEFFAD
:10DAE00040212162012084F8FC01D4F8180228B1F9
:10DAF0002179D4F81402426820469047002010BDD6
:10DB0000014691F8FD0181F8FC010020704710B535
:10DB1000044694F8FC01032808D1D4F81402C06923
:10DB200020B1D4F81402C16920468847002010BDF6
:10DB3000024611740020704770B504460D4601205E
:10DB4000044908702946D4F82002F4F71AFC002092
:10DB500070BD00001B02002470B504460D46294626
:10DB600004F5027000F00DFA0120C4F8F40140F24F
:10DB70000E20005BC4F8F80194F8080200F01F00C2
:10DB800020B1012808D0022812D10BE004F502715F
:10DB9000204600F0F8FA13E004F50271204600F088
:10DBA000D6FB0DE004F50271204600F025FB07E0EE
:10DBB00094F8080200F08001204600F004F800BF4D
:10DBC00000BF002070BD70B504460D462946D4F84C
:10DBD0002002F3F756FE002070BD10B50446D4F8BD
:10DBE0002002F4F7F0FB002010BD014691F8FC0183
:10DBF00081F8FD01042081F8FC01002070472DE927
:10DC0000F04104460D4616461F463B46324629461D
:10DC1000D4F82002F3F773FE0020BDE8F081000085
:10DC200070B505460C462DB92246064906A0FFF7F9
:10DC30008BFD04E02246034903A0FFF785FD014860
:10DC400070BD0000007303244D534320436F6E6684
:10DC50006967000070B504460D4629462046FBF76B
:10DC60006CFD002070BD70B504460D462946204667
:10DC7000FBF78BFD002070BD70B504460D460121F9
:10DC80002046FFF7C9FD81212046FFF7C5FD20464C
:10DC9000FBF79EFDD4F8180238B10020D4F8181212
:10DCA00002F01AF90020C4F81802002070BD00002C
:10DCB0000246122008800148704700003802002404
:10DCC00001460A2008800148704700001002002425
:10DCD000014620200880014870470000D001002440
:10DCE000014620200880014870470000B001002450
:10DCF000014620200880014870470000F001002400
:10DD000070B504460E460025207C70B94FF40073B0
:10DD1000022201212046FFF7B1FE4FF400730222D8
:10DD200081212046FFF7AAFE0BE0402302220121B9
:10DD30002046FFF7A3FE4023022281212046FFF761
:10DD40009DFE48F26C01002002F0D8F8C4F81802D9
:10DD5000D4F8180208B9012503E02046FBF73DFD81
:10DD60000025E8B270BD000070B505460C462DB91F
:10DD70002246064906A0FFF7E7FC04E022460349D5
:10DD800003A0FFF7E1FC014870BD0000007303240D
:10DD90004D534320496E74657266616365000000EF
:10DDA0000246042008800148704700004C0200240D
:10DDB00070B505460C462246024903A0FFF7C4FC95
:10DDC000004870BD0073032453544D6963726F653E
:10DDD0006C656374726F6E696373000070B505469D
:10DDE0000C462DB92246064906A0FFF7ADFC04E01B
:10DDF0002246034909A0FFF7A7FC014870BD0000B7
:10DE0000007303244D6173732053746F72616765EF
:10DE100020696E204853204D6F6465004D61737317
:10DE20002053746F7261676520696E204653204DE0
:10DE30006F646500024609B1C2F81C1200207047E9
:10DE400070B505460C461A202080F2F72DFE0148D9
:10DE500070BD00005002002470B505460C46D5F890
:10DE60001862207800F0600000283FD0202876D18A
:10DE70006078FE2802D0FF2830D11BE0608890B97E
:10DE8000E08801280FD1207800F0800080280AD196
:10DE9000D5F81C1288698047306001223146284637
:10DEA000FFF73CFB05E021462846FFF71EFB02205A
:10DEB00070BD19E0608850B9E08840B9207800F062
:10DEC0008000802803D02846FBF7AAFC05E0214605
:10DED0002846FFF70AFB0220EAE705E0214628462C
:10DEE000FFF703FB0220E3E700BF47E0607801286B
:10DEF0000DD00A2802D00B283DD105E00122311DAA
:10DF00002846FFF70BFB36E0A078706033E02179FC
:10DF10002846FFF74BFD21792846FFF77DFC207945
:10DF200000F08000802810D1287C38B94FF40073AD
:10DF3000022281212846FFF7A1FD17E0402302229B
:10DF400081212846FFF79AFD10E0287C40B94FF464
:10DF50000073022201212846FFF790FD06E00CE045
:10DF60004023022201212846FFF788FD2179284617
:10DF7000FBF7C8FB00BF00BF00E000BF00BF0020F0
:10DF800096E70A7802704A7842708B78CA7803EB79
:10DF9000022242800B794A7903EB022282808B793C
:10DFA000CA7903EB0222C2807047000070B50546B3
:10DFB0000C46002614B1C5F8144209E005A001F092
:10DFC000E1F906A001F0DEF90AA001F0DBF9022672
:10DFD000304670BD4552524F523A2000496E76612C
:10DFE0006C696420436C6173732068616E646C6556
:10DFF000000000000D0A000001460020704770B5C7
:10E0000004460D46A888F8B9E888E8B9A87800F071
:10E010007F0694F8FC01032804D129462046FFF727
:10E0200064FA15E084F8FE6131462046FFF784FD6E
:10E030002046FFF784FA1EB1022084F8FC0107E0B5
:10E04000012084F8FC0103E029462046FFF74DFA41
:10E0500070BD70B504460D460226D4F8140238B1DE
:10E06000D4F81402294602682046904700B90026D9
:10E07000304670BD70B504460D46A8783449087026
:10E0800008460078012804DD29462046FFF72DFACE
:10E090005BE094F8FC01022802D003284FD11CE079
:10E0A0002B480078A8B12A4800786060032084F8E3
:10E0B000FC01274801782046FFF7CBFF022804D156
:10E0C00029462046FFF711FA70BD2046FFF737FAC0
:10E0D00002E02046FFF733FA36E01D48007870B9B9
:10E0E000022084F8FC011A48007860601848017822
:10E0F0002046FFF7B5F92046FFF721FA1EE0144944
:10E1000009786068884216D021792046FFF7A8F97F
:10E110000F48007860600E4801782046FFF799FFAD
:10E12000022804D129462046FFF7DFF9CCE7204634
:10E13000FFF705FA02E02046FFF701FA04E029465E
:10E140002046FFF7D2F900BF00BF00BFBCE70000C8
:10E150001A02002470B504460D46688801280AD1C9
:10E16000C4F80402D4F81402294682682046904775
:10E170002046FFF7E4F970BD10B504462046FFF7CE
:10E180002CFD002010BD70B505460C4600266078B9
:10E190000A2829D2DFE800F01923281E280A0528BA
:10E1A000140F21462846FFF7FFF922E021462846B2
:10E1B000FFF725FF1DE021462846FFF75BFF18E02B
:10E1C00021462846FFF7C8F913E021462846FFF705
:10E1D00099FA0EE021462846FFF7BCFF09E02146E8
:10E1E0002846FFF748F904E021462846FFF77DF965
:10E1F00000BF00BF304670BD2DE9F04105460E4618
:10E200004FF000083479307800F06000202808D101
:10E21000D5F8140231468268284690470020BDE8B0
:10E22000F0817078002855D001282AD003287AD1AF
:10E2300095F8FC01022802D003281BD107E02CB17D
:10E24000802C03D021462846FFF7BDFC17E07088DC
:10E2500030B92CB1802C03D021462846FFF7B3FCFF
:10E26000D5F8140231468268284690472846FFF7C1
:10E2700066F904E031462846FFF737F900BF00BFD2
:10E2800062E095F8FC01022802D003281BD107E0C8
:10E290002CB1802C03D021462846FFF794FC17E0D0
:10E2A000708878B904F07F0048B121462846FFF70E
:10E2B000A9FAD5F8140231468268284690472846C4
:10E2C000FFF73DF904E031462846FFF70EF900BF9D
:10E2D00000BF39E095F8FC01022802D003282BD1B9
:10E2E00007E004F07F0018B121462846FFF76BFCD9
:10E2F00027E004F08000802806D104F07F0105F1BA
:10E30000140000EB011005E004F07F0105F58270B8
:10E3100000EB0110074621462846FFF78DFB18B198
:10E320000120386002E00EE0002038600222394609
:10E330002846FFF7F3F804E031462846FFF7D5F802
:10E3400000BF00BF00E000BF00BF404667E770B5F8
:10E3500004460D46002694F8FC01032814D12879C0
:10E3600001280CDCD4F81402294682682046904724
:10E37000E88840B93EB92046FFF7E1F803E02946B6
:10E380002046FFF7B2F804E029462046FFF7ADF833
:10E3900000BF00BF002070BD10B5024648780128BC
:10E3A0002BD140F61C0080580C780123A3409BB26F
:10E3B000184340F61C039850087802F5106303EBED
:10E3C0004010006800F40040F0BB0889C0F30A0068
:10E3D000CB7840EA83400B7840EA835040F080508D
:10E3E00040F4004002F5106404EB43131B6818432B
:10E3F0000B7804EB431318602CE040F61C008058A7
:10E400000C780123A340144C04EA0343184340F65C
:10E410001C039850087802F5306303EB4010006845
:10E4200000F4004080B90889C0F30A00CB7840EAC4
:10E43000834040F0805040F400400B7802F5306497
:10E4400004EB43131B6800E004E018430B7804EB73
:10E4500043131860002010BD0000FFFF01464FF479
:10E4600010604058C20AD2024FF41060425040F689
:10E470000800405800F00600042807D14FF410604F
:10E48000405840F003024FF41060425040F6040040
:10E49000405840F4807240F604004250002070471B
:10E4A0000FB410B504460898012816D1A06B20F4CB
:10E4B0008030A063E06815490840E060E06820F41F
:10E4C0004010E0600F98012803D1E06840F480100C
:10E4D000E060204600F01CF809E0E06840F04000F1
:10E4E000E060204600F014F84FF48030A0630698F6
:10E4F000012807D1A06840F00C00A060A06840F09F
:10E500002000A060002010BC5DF814FBBFFFBDFF21
:10E510000146002200BF501C02460F4B984201D911
:10E5200003207047086900F000400028F3D0002263
:10E53000086940F00100086100BF501C0246064B0C
:10E54000984201D90320ECE7086900F00100002897
:10E55000F3D100BFE5E70000400D030010B502460F
:10E560004878012822D140F63C0080580C780123DD
:10E57000A3409BB2984340F63C03985040F61C00E1
:10E5800080580C780123A3409BB2984340F61C03AB
:10E590009850087802F5106303EB4010006820F4EF
:10E5A0000044087803EB4010046026E040F63C008D
:10E5B00080580C780123A340114C04EA034398438C
:10E5C00040F63C03985040F61C0083580C7801201C
:10E5D000A0400B4C04EA004023EA000040F61C0374
:10E5E0009850087802F5306303EB4010006820F47F
:10E5F0000044087803EB40100460002010BD0000C8
:10E600000000FFFF10B5044640F60400005920F05A
:10E61000020140F6040001510320F2F7D9FA00206C
:10E6200010BD10B5044640F60400005940F0020148
:10E6300040F6040001510320F2F7CAFA002010BD91
:10E640000FB430B504460025A06B40F40010A06361
:10E650000E9858B9A06B20F40010A063206840F019
:10E6600040002060206840F0800020600020C4F856
:10E67000000ED4F80008C4F80008099801280BD14E
:10E68000069820B90021204600F078FC08E001211E
:10E69000204600F073FC03E00321204600F06EFCEE
:10E6A0001021204600F0B4FB204600F09BFB002127
:10E6B0004FF401600151001D0151491E001D01511F
:10E6C0000021001D0151002524E004F5106000EB3D
:10E6D0004510006800F00040B0F1004F07D14FF046
:10E6E000904104F5106000EB4510016005E0002149
:10E6F00004F5106000EB45100160002104F5106086
:10E7000000EB45100161FF2104F5106000EB45109E
:10E7100081606D1C0498A842D7D8002524E004F538
:10E72000306000EB4510006800F00040B0F1004F91
:10E7300007D14FF0904104F5306000EB45100160C7
:10E7400005E0002104F5306000EB45100160002178
:10E7500004F5306000EB45100161FF2104F53060E5
:10E7600000EB451081606D1C0498A842D7D84FF487
:10E770000160005920F480714FF401600151079845
:10E7800001280BD115494FF4036001510059144978
:10E7900008434FF403610851084605590020A06161
:10E7A0006FF080406061079818B9A06940F01000D0
:10E7B000A061A0690B490843A0610A9818B1A0693B
:10E7C00040F00800A0610E98012803D1A069064915
:10E7D0000843A061002030BC5DF814FB0004000277
:10E7E0000300010800383C800400004001468868AE
:10E7F00020F00100886000207047000030B503461B
:10E80000487801287DD1486918BB087803F5106461
:10E8100004EB40100069644C20400C7803F510654F
:10E8200005EB4414206108782C4604EB4010006985
:10E8300040F40025087804EB40100561087804EBEB
:10E8400040100069C50CED04087804EB4010056128
:10E8500037E0087803F5106404EB40100069C50C3C
:10E86000ED04087804EB40100561087804EB4010D3
:10E8700004694D480440087803F5106505EB401025
:10E8800004618C684869A04201D9886848610878A9
:10E8900003F5106404EB4010006940F4002508788B
:10E8A00004EB40100561087804EB401004694869E6
:10E8B000C0F312000443087803F5106505EB40101F
:10E8C0000461012A07D1087803F5106404EB4010B5
:10E8D0000D6945610BE0486948B140F63400C05805
:10E8E0000D780124AC40204340F63404E050087811
:10E8F00003F5106404EB4010006840F0044508780C
:10E9000000E003E004EB401005604AE0087803F5FE
:10E91000306404EB40100069C50CED04087804EB8A
:10E9200040100561087804EB401000691E4C20403F
:10E930000C7803F5306505EB44142061486908B193
:10E9400088684861087803F5306404EB401000697A
:10E9500040F40025087804EB40100561087804EBCA
:10E96000401000698C68C4F3120420430C7803F54E
:10E97000306505EB44142061012A06D1087803F5BF
:10E98000306404EB4010CD684561087803F53064CD
:10E9900004EB4010006840F00445087804EB401098
:10E9A0000560002030BD0000FFFF07E010B5034602
:10E9B0000024C3F8104BD3F8100B40F40024C3F824
:10E9C000104BD3F8100B40F01804C3F8104BD3F8D9
:10E9D000100B40F0C044C3F8104B012906D1C3F816
:10E9E000142B4FF080244FF43060C450002010BD31
:10E9F00010B50246487801281ED1087802F5106348
:10EA000003EB4010006820F40014087803EB40107A
:10EA10000460C878032802D0C87802282AD1087870
:10EA200002F5106303EB4010006840F08054087852
:10EA300003EB401004601DE0087802F5306303EB3F
:10EA40004010006820F40014087803EB40100460C4
:10EA5000C878032802D0C87802280BD1087802F5BC
:10EA6000306303EB4010006840F08054087803EBFB
:10EA700040100460002010BD10B5024648780128FF
:10EA80001FD1087802F5106303EB4010006800F016
:10EA9000004048B9087803EB4010006820F080443B
:10EAA000087803EB40100460087802F5106303EB6C
:10EAB0004010006840F40014087803EB4010046034
:10EAC0001EE0087802F5306303EB4010006800F0A8
:10EAD000004048B9087803EB4010006820F08044FB
:10EAE000087803EB40100460087802F5306303EB0C
:10EAF0004010006840F40014087803EB40100460F4
:10EB0000002010BDF8B505460C4616460027607873
:10EB100001287DD1606918BB207805F5106101EBF3
:10EB200040100069AA490840217805F5106202EBFF
:10EB3000411108612078114601EB4010006940F452
:10EB40000022207801EB40100261207801EB401098
:10EB50000069C20CD204207801EB401002614FE042
:10EB6000207805F5106101EB40100069C20CD20459
:10EB7000207801EB40100261207801EB4010006921
:10EB800093490840217805F5106202EB41110861B4
:10EB9000A16860690844401EB0FBF1F08C49C9438C
:10EBA00001EAC040217802EB41110969084321784C
:10EBB00002EB411108612078114601EB4010016918
:10EBC0006069C0F312000143207802EB401001613C
:10EBD000E078012814D12078114601EB401000693B
:10EBE00020F0C042207801EB40100261207801EB58
:10EBF0004010006940F00052207801EB40100261A3
:10EC0000012E09D1207805F5106101EB401000E0DC
:10EC10004BE0226942610EE0E07801280BD0606988
:10EC200048B140F634004059227801219140084310
:10EC300040F634014851E07801281ED140F6080022
:10EC4000405900F4807060B9207805F5106101EB3F
:10EC50004010006840F00052207801EB4010026044
:10EC60000BE0207805F5106101EB4010006840F0E2
:10EC70008052207801EB40100260207805F5106189
:10EC800001EB4010006840F00442207801EB401096
:10EC90000260E078012807D10096A08A83B222782A
:10ECA0002846E16800F072F98FE0207805F53061C0
:10ECB00001EB40100069C20CD204207801EB401037
:10ECC0000261207801EB4010016941480140207841
:10ECD00005F5306202EB401001616069C0B920782F
:10ECE000114601EB40100069A168C1F3120108430D
:10ECF000217802EB411108612078114601EB4010A8
:10ED0000006940F40022207801EB4010026125E008
:10ED1000A16860690844401EB0FBF1F087B220781A
:10ED200005F5306101EB401000692949C94301EA4A
:10ED3000C7410843217805F5306202EB41110861B3
:10ED40002078114601EB40100169A0687843C0F3B8
:10ED500012000843217802EB41110861012E06D10F
:10ED6000207805F5306101EB4010E2684261E078FF
:10ED700001281ED140F60800405900F4807060B9A7
:10ED8000207805F5306101EB4010006840F000523A
:10ED9000207801EB401002600BE0207805F530612F
:10EDA00001EB4010006840F08052207801EB4010E9
:10EDB0000260207805F5306101EB4010006840F0FA
:10EDC0000442207801EB401002600020F8BD0000F2
:10EDD000FFFF07E00146886840F0010088600020DE
:10EDE00070470000014600221020086100BF501C3F
:10EDF0000246064B984201D903207047086900F08B
:10EE000010001028F3D00020F7E70000400D0300A9
:10EE100010B502460023202040EA8110106100BF97
:10EE2000581C0346054CA04201D9032010BD1069AF
:10EE300000F020002028F3D00020F7E7400D030069
:10EE40000146002040F60802525802F0060202B9BC
:10EE500017E040F60802525802F00602022A06D0D5
:10EE600040F60802525802F00602062A01D1032099
:10EE700007E040F60802525802F00602042A00D1C8
:10EE8000022070470146486900F0010070470146C2
:10EE900040F618004258001D4058024090B270479A
:10EEA000014640F618004258001D40580240100C20
:10EEB000704730B502464FF40165AB5840F6340553
:10EEC000AC5824FA01F505F0010543EAC51302F533
:10EED000106505EB4115AD6805EA030030BD02463B
:10EEE00002F5306303EB4113986840F614039B5816
:10EEF000184070470146002048698A6910407047F1
:10EF000070B503460024D01CC61700EB9676B510EA
:10EF100000BF05E04FF48050C0580860091D641C14
:10EF2000AC42F7D3084670BD70B504460D46E068A4
:10EF300020F0C040E060012D04D1E06840F00050B6
:10EF4000E06004E01DB9E06840F08040E0603220FD
:10EF5000F1F73EFE002070BD0246D2F8000820F412
:10EF6000FE60C2F80008D2F800084FF4FE6303EA1E
:10EF700001131843C2F80008002070470246D2F877
:10EF800000080843C2F8000800207047F0B50446A6
:10EF9000059E00270025A6B9D81C4FEAE07C00EBAF
:10EFA0009C7C4FEAAC0700BF09E0D1F800C004F533
:10EFB000805000EB0230C0F800C0091D6D1CBD423E
:10EFC000F3D30020F0BD00BFFEE7000010B50446FB
:10EFD000240300F067F900F0FFF800224FF480618D
:10EFE0001048F1F745FF2020FDF78CF80E48008807
:10EFF0004EF61871884202D1200EFDF783F8C4F353
:10F000000740FDF77FF8C4F30720FDF77BF8E0B277
:10F01000FDF778F8012291020248F1F729FF00F08C
:10F02000DBF810BD001402583000002410B586B083
:10F0300000BF2248006840F02000204908600846D0
:10F04000006800F02000009000BF00BF4FF4806017
:10F0500001900120029003900320049001A9184818
:10F06000F1F7D4FD012291021548F1F701FFFDF7F8
:10F0700015F84FF00050FDF755F800F05DF8114914
:10F080000880084600884EF61871884214D1032083
:10F0900000F078F8044604F0010068B900224FF44B
:10F0A00080610748F1F7E4FEB720FDF72BF8012255
:10F0B00091020348F1F7DCFE06B010BDE0440258AF
:10F0C00000140258300000242DE9F04106460C4699
:10F0D000174600224FF480611548F1F7C9FE03205E
:10F0E000FDF710F8134800884EF61871884202D1D7
:10F0F000200EFDF707F8C4F30740FDF703F8C4F34B
:10F100000720FCF7FFFFE0B2FCF7FCFF002505E05D
:10F11000FF20FCF7F7FF7055681C85B2BD42F7DB96
:10F12000012291020248F1F7A3FEBDE8F081000040
:10F13000001402583000002410B5002400224FF4BF
:10F1400080610F48F1F794FE9020FCF7DBFF002070
:10F15000FCF7D8FF0020FCF7D5FF0020FCF7D2FF1A
:10F16000FF20FCF7CFFF44EA0024FF20FCF7CAFF92
:10F170000443012291020248F1F77AFE204610BDB5
:10F180000014025870B5044600250026012C04D056
:10F19000022C04D0032C06D103E0052605E0352619
:10F1A00003E0152601E0052600BF00BF00224FF452
:10F1B00080610848F1F75CFE3046FCF7A3FFFF20B2
:10F1C000FCF7A0FF0546012291020248F1F750FE2C
:10F1D000284670BD0014025810B500BF0120FFF78B
:10F1E000D1FF00F001000028F8D110BD2DE9F05F3B
:10F1F00081460F461646DFF8A8B04FEA1738C7F326
:10F200000B0ACAF58054A64200DC344644E04FEABB
:10F2100008314FF480525846FFF756FF002508E0AA
:10F220000AEB05001BF80000FF2800D003E0681C73
:10F2300085B2A542F4DB00BFA54216DA4046FFF7CF
:10F24000C5FE002507E019F8050005EB0A010BF8DB
:10F250000100681C85B2A542F5DB4FEA08314FF486
:10F260008052584600F030F804E0224639464846BD
:10F2700000F02AF8A64200D10FE008F101084FF093
:10F28000000AA1442744301B86B2B6F5805F02DD38
:10F290004FF4805400E03446B9E700BFBDE8F09F6A
:10F2A000B00C002410B500224FF480610548F1F73E
:10F2B000DFFD0620FCF726FF012291020148F1F74D
:10F2C000D7FD10BD001402582DE9F04107460E4647
:10F2D0001446F0B2C0F58075AC4200DC254612E061
:10F2E0002A463146384600F013F8AC4200D10BE014
:10F2F0002F442E44601B84B2B4F5807F02DD4FF4AE
:10F30000807500E02546EBE700BFBDE8F081000016
:10F310002DE9F04106460C461746FFF7C3FF0022D1
:10F320004FF480611548F1F7A3FD0220FCF7EAFED7
:10F33000134800884EF61871884202D1200EFCF75F
:10F34000E1FEC4F30740FCF7DDFEC4F30720FCF741
:10F35000D9FEE0B2FCF7D6FE002504E0705DFCF7B4
:10F36000D1FE681C85B2BD42F8DB01229102034840
:10F37000F1F77EFDFFF730FFBDE8F0810014025881
:10F38000300000240FB4054B10B503A9044A0298BD
:10F3900000F034F810BC5DF814FB0000D5F800084C
:10F3A0000C00002402480068C0F3022070470000EF
:10F3B0000CED00E010B5002804DB0A07130E054A27
:10F3C000135406E00A07140E034A00F00F031B1F34
:10F3D000D45410BD00E400E018ED00E002E008C8DD
:10F3E000121F08C1002AFAD170477047002001E0BF
:10F3F00001C1121F002AFBD1704700002DE9FF4F09
:10F400008DB00F460546002606E025280BD0DDE925
:10F410000F1290476D1C761C28780028F5D111B08A
:10F420003046BDE8F08F0024A246A1460122EC49F7
:10F4300000E0044315F8013F203B02FA03F00842C4
:10F44000F7D128782A2810D06FF02F022878A0F161
:10F450003001092914D80AEB8A0102EB410144F07A
:10F46000020400EB010A6D1CF0E701CF5FEA000A1D
:10F4700003D544F40054CAF1000A44F002046D1CA0
:10F4800028782E2817D115F8010F44F004042A28F3
:10F490000ED06FF02F022878A0F1300109290AD888
:10F4A00009EB890102EB410100EB01096D1CF2E758
:10F4B00057F8049B6D1C28786C280FD006DC4C286C
:10F4C00017D068280DD06A2814D104E0742810D011
:10F4D0007A280FD10DE044F400140AE044F48014BB
:10F4E00001E044F440146978814202D104F58014AB
:10F4F0006D1C6D1C2A786E2A1FD00CDC632A31D05B
:10F5000004DC002A8BD0582A11D1A3E0642A68D0E9
:10F51000692A0CD165E0732A2ED004DC6F2A73D0DF
:10F52000702A04D19BE0752A6FD0782A6ED01046DD
:10F53000DDE90F129047761C50E1C4F30250022817
:10F5400006D0032809D0042801CF09D0066045E180
:10F5500001CFF117C0E9006140E101CF06803DE134
:10F5600006703BE117F8040B8DF8000000208DF8C1
:10F570000100EB46012003E057F804BB4FF0FF30D9
:10F5800061074FF0000102D40DE008F10101884647
:10F5900049450FDA8045F8DB1BF808100029F4D143
:10F5A00008E008F1010188468142FADB1BF80810E7
:10F5B0000029F6D1DDE90F23AAEB08008146214698
:10F5C00000F036F9304400EB080604E0DDE90F12E4
:10F5D0001BF8010B9047B8F10108F7D221464846C5
:10F5E000F7E00A21C4F302534FF0000B0891022BFD
:10F5F00004D001CFC117032B09D00AE0FF1D27F06B
:10F600000707F7E8020108E032E01FE020E000B25F
:10F61000C117042B01D140B2C117031E71F10003C1
:10F6200007DA4FF0000CD0EB0C006CEB01012D233E
:10F6300002E0230504D52B238DF82430012303E0B9
:10F64000E30701D02023F7E7984658E00A2110E0AD
:10F6500010210EE010204FF0000B08900CE010215C
:10F660004FF0000B44F004044FF00809089103E048
:10F6700008214FF0000B0891C4F30253022B04D071
:10F6800001CF0021032B06D006E0FF1D27F007075E
:10F69000F7E8020103E080B2042B00D1C0B24FF0C2
:10F6A000000823072BD5702A07D0DDF820C08CF086
:10F6B000100C5CEA0B0C05D00EE040238DF82430D2
:10F6C000012308E050EA010306D030238DF82430EE
:10F6D0008DF8252002239846DDF820C08CF0080C18
:10F6E0005CEA0B0C0BD150EA010301D1630706D58C
:10F6F00030238DF824304FF00108A9F10109582A70
:10F7000004D038A20B9208AA0A920BE03AA2F9E7B9
:10F710005B46089AF0F7E4FD0B9B9B5C0A9A521E2D
:10F720000A92137050EA0102F2D10A98ADEB000080
:10F7300000F1200B600702D524F4803401E04FF083
:10F740000109D94502DDA9EB0B0000E0002000EB28
:10F750000B0141440890AAEB010AE00306D4DDE95D
:10F760000F232146504600F063F806444FF000098D
:10F7700008E009A911F80900DDE90F12904709F125
:10F780000109761CC145F4DBE0030CD5DDE90F234C
:10F790002146504600F04CF8064404E0DDE90F1223
:10F7A00030209047761C0899481E08900029F5DC07
:10F7B00008E00A980A990078491C0A91DDE90F12BD
:10F7C0009047761CBBF10001ABF1010BF1DC214647
:10F7D0005046DDE90F2300F019F806446D1C1BE6C6
:10F7E0000928010030313233343536373839616217
:10F7F00063646566000000003031323334353637DB
:10F800003839414243444546000000002DE9F041AB
:10F81000044600251E461746880404D405E03946F0
:10F820002020B0476D1C641EF9D52846BDE8F08144
:10F830002DE9F041044600251E469046C80301D537
:10F84000302700E02027880404D505E041463846EB
:10F85000B0476D1C641EF9D52846BDE8F081000054
:10F8600010B504460420F5F7C3FD0148046010BD3F
:10F870000800002430B50446002504E04FF47A70F7
:10F8800000F004F86D1CA542F8D330BD70B50346F6
:10F8900000224FF0E02675690D4E366803FB06F432
:10F8A0004FF0E026B16910E04FF0E026B0698842E1
:10F8B0000BD0884202D20E1A324402E02E1A0E44B5
:10F8C00032440146A24200D300E0EDE700BF70BD24
:10F8D0000800002400BF054AD26902F04002002A55
:10F8E000F9D0C2B2014B1A857047000000100140E8
:10F8F0001CB500260027F0F7A7FD042302220521EE
:10F90000A020FCF797FDF1F7CBFA4FF4C870FFF792
:10F91000A7FF4FF4E13000F013FBBC484168C8205A
:10F920008847F9F70BF9F6F755F9F9F70AFEFBF7EF
:10F9300087FFF6F751FBFFF779FB002000F042FA52
:10F94000012000F03FFA022000F03CFA4FF478402A
:10F95000AF490860AFA010210B46C822CDE90010C6
:10F9600032211E20F9F78CF8AFA010210B46C822D7
:10F97000CDE9001046211E20F9F782F8B0A0102131
:10F980000B46C822CDE900105A211E20F9F778F85D
:10F99000AFA010210B46C822CDE900106E211E2019
:10F9A000F9F76EF8FCF716F950B1ACA010210B4630
:10F9B000C822CDE9001082211E20F9F761F819E074
:10F9C000AAA010210B46C822CDE9001082211E20DA
:10F9D000F9F756F8AB488069AA49C969A0FB014507
:10F9E00010200090200D40EA053205238221862058
:10F9F000F8F7FCFFFFF7A0FB4EF6187188420AD01B
:10FA0000A1A010210B46C822CDE9001082211E20A2
:10FA1000F9F736F809E0A0A010210B46C822CDE97D
:10FA2000001096211E20F9F72BF8F0F7BDFF50B11A
:10FA30009EA010210B46C822CDE90010AA211E204D
:10FA4000F9F71EF819E09CA010210B46C822CDE959
:10FA50000010AA211E20F9F713F8102000909C48EE
:10FA6000C0899B4989794843994949884843021587
:10FA70000423AA219E20F8F7B9FF00229549964851
:10FA8000FDF78CFE95499448FEF790FA9449924808
:10FA9000FEF7D0F99048FEF76FFBF2F7BDFC4FF48C
:10FAA000E160FFF7E7FEAFE00120FFF7E3FE8D48DE
:10FAB0000078804566D04FF6FF70E223F022D22115
:10FAC00000901E20F6F750FA8648007800F00100FA
:10FAD00070B1002201218448F1F7CAF983A01021F6
:10FAE0000B46C822CDE90010D2211E20F8F7C8FF2E
:10FAF0007C48007800F0020070B1002201217A48B1
:10FB0000F1F7B6F97DA010210B46C822CDE900100F
:10FB1000D2211E20F8F7B4FF7248007800F00400EC
:10FB200050B17AA010210B46C822CDE90010E62181
:10FB30001E20F8F7A5FF08E04FF6FF70F623F0222D
:10FB4000E62100901E20F6F70FFA6648007800F0D4
:10FB5000080050B171A010210B46C822CDE9001059
:10FB6000FA211E20F8F78CFF09E04FF6FF704FF4E2
:10FB70008573F022FA2100901E20F6F7F5F9594816
:10FB800090F800806948007881451BD0674800786C
:10FB900001280AD166A010210B46C822CDE9001029
:10FBA000BE211E20F8F76CFF09E066A010210B466D
:10FBB000C822CDE90010BE211E20F8F761FF5B4886
:10FBC00090F80090781CC7B2C82F1DD100270122E1
:10FBD00011464548F1F74CF902214348F1F744F941
:10FBE0004048007800F0100020B1002601204F4965
:10FBF000087006E0701CC6B20A2E02DD00204B49D8
:10FC000008700020374908704EE7000060000024AB
:10FC100020000024504F4C41524953204837353082
:10FC20002F4637353000000055534220436172643F
:10FC300020526561646572205445535400000000F1
:10FC400041544F4D40414C49454E54454B000000F6
:10FC5000323031392F352F313700000053442043E3
:10FC6000617264204572726F722100005344204318
:10FC70006172642053697A653A20202020204D4229
:10FC80000000000078080024573235513235362004
:10FC90004572726F7221000053504920464C415307
:10FCA000482053697A653A32354D42004E414E4400
:10FCB000204572726F7221004E414E4420466C61A5
:10FCC00073682053697A653A202020204D42000055
:10FCD000CC0B00241C020024D8020024780100244C
:10FCE000B80200246C02002400040258555342203C
:10FCF00057726974696E672E2E2E0000555342208C
:10FD000052656164696E672E2E2E000055534220A5
:10FD10005772697465204572722000005553422065
:10FD20005265616420204572722000001B0200248D
:10FD300055534220436F6E6E6563746564202020C6
:10FD40002000000055534220446973436F6E6E6576
:10FD500063746564200000002DE9F04104460E46FE
:10FD60001548005D38B91448203801682046884796
:10FD70000120BDE8F081114850F82400B04219D9A3
:10FD80000F4850F82400B6FBF0F10B480C3850F83F
:10FD9000240050F82120002508E0002306480C38F4
:10FDA00050F824004F1940F827306D1C9542F4DBC1
:10FDB0000020DEE70220DCE77401002494580108EB
:10FDC0008858010810B50446074951F824108A00E4
:10FDD000064951F82400002100F0A4F8012103484D
:10FDE0000C30015510BD00007C580108680100244A
:10FDF0002DE9F04704460F460025A9462348005D3B
:10FE000020B9224820380168204688471FB94FF0A2
:10FE1000FF30BDE8F0871E4850F82400B7FBF0F62D
:10FE20001B4850F82400B7FBF0F100FB117000B143
:10FE3000761C184850F82400451E22E013480C3860
:10FE400050F8240050F8250010B909F1010901E02B
:10FE50004FF00009B14513D14FF0000809E00B48FD
:10FE60000C3850F8240005EB080140F8216008F137
:10FE70000108B045F3D3064850F824006843C8E7AA
:10FE80006D1E002DDADA4FF0FF30C2E77401002456
:10FE9000885801087C58010810B50146002300224B
:10FEA00007E00B4850F8210050F8220000B15B1C1D
:10FEB000521C084850F821009042F2D84FF47A7052
:10FEC0005843044C54F82140B0FBF4F080B210BD0C
:10FED000680100247C58010870B505460C4604B939
:10FEE00070BD054850F82500261A31462846FFF710
:10FEF00033FF00BFF4E700005C01002470B5044646
:10FF00000E4631462046FFF773FF0546681C08B9C8
:10FF1000002070BD024850F824002844F9E7000092
:10FF20005C01002430B5034601E003F8011B141EF8
:10FF3000A2F10102F9D130BD014608687047000006
:10FF400010B5044609480A49086008464460002183
:10FF50008160C160016181610C214161F5F78AFB1B
:10FF6000012204490248F5F70DFC10BD00100140C4
:10FF7000C40500241200002430B595B0054613AB2B
:10FF800012AA09A9284600F03FFA044614B12046F7
:10FF900015B030BD0020149026E0224909689DF874
:10FFA000502001EBC20113AB11AA486801A900F06F
:10FFB0002BFA04460CB12046EAE709A901A800F093
:10FFC000E1FC60B99DF844009DF84810884201DDCD
:10FFD0000220DDE79DF85000124988750AE09DF87F
:10FFE0005000401CC0B214900E48007D9DF8501087
:10FFF0008842D2DC00BF0B48007D9DF8501088423B
:020000040801F1
:1000000001D10420C4E714A9284600F0DDFA044613
:100010000CB12046BCE79DF850000249487500200D
:10002000B6E70000600000242DE9F0419AB09C483A
:10003000847D007DA04202DC1AB0BDE8F0819849C1
:10004000096801EBC40106AB07AA486808A900F0DB
:10005000DBF908A993A0FFF795F9002644E0904842
:10006000008B0121B1400840D8B122218FA0FFF7B9
:1000700089F9304600F02EFB89492431471839466A
:100080008BA0FFF77FF9222188A0FFF77BF930468C
:1000900000F020FB82492431084410A941F82600D1
:1000A00018E0304600F016FB7D492431085810A9AD
:1000B00041F826007A48C07D30B910A850F82610C3
:1000C0007CA0FFF75FF905E010A850F826107AA091
:1000D000FFF758F99DF81C00401EB04202D078A0EE
:1000E000FFF750F9701CC6B29DF81C008642B6DBC3
:1000F00074A0FFF747F900F03FFB6948407D0B28EB
:100100000DD2DFE800F0060D151E27323F4E5F725C
:1001100087006349096851F834008047054690E03C
:100120005F4A126852F8341010988847054688E0F4
:100130005B4B1B6853F83420DDE9100190470546FE
:100140007FE0574F3F6857F8343010A807C89847EA
:10015000054676E0DFF848C1DCF800C05CF8347092
:1001600010A80FC8B84705466BE01498DFF830C1F7
:100170000090DCF800C05CF8347010A80FC8B847D5
:1001800005465EE0DDE91401DFF814C1CDE90001A8
:10019000DCF800C05CF8347010A80FC8B8470546FA
:1001A0004FE0DDE914121698DFF8F4C0CDE9001233
:1001B0000290DCF800C05CF8347010A80FC8B84793
:1001C00005463EE0DDE91423DDE91610DFF8D0C076
:1001D000CDE90023CDE90210DCF800C05CF83470F2
:1001E00010A80FC8B84705462BE0DDE91523DDE967
:1001F0001710CDE90123CDE903101498DFF8A0C052
:100200000090DCF800C05CF8347010A80FC8B84744
:10021000054616E0DDE91623DDE91810CDE90223D5
:10022000CDE90410DDE91401DFF874C0CDE9000167
:10023000DCF800C05CF8347010A80FC8B847054659
:1002400000BF00BF00F056FA9DF8180001280CD13D
:100250001348C07D20B929461BA0FFF793F807E09B
:1002600029461BA0FFF78EF802E018A0FFF78AF8D6
:100270000B4890F8EC0088B10948D0F8F0000A214A
:10028000B0FBF1F201FB12070548D0F8F000B0FB1B
:10029000F1F83A46414611A0FFF774F800BFCBE6EB
:1002A000600000240D0A257328000000256300006B
:1002B00025730000256C64003058255800000000AC
:1002C0002C000000290000003D256C753B0D0A0044
:1002D0003D305825583B0D0A0000000046756E63FE
:1002E00074696F6E2052756E2054696D653A25648D
:1002F0002E2531646D730D0A00000000F0B5034631
:10030000154600200022002600245BE01F782C2FD9
:1003100001D104B901221F78292F01D01F780FB90C
:1003200004B950E0002E3AD11F78302F02DB1F783D
:10033000392F17DD1F782D2F14D01F782B2F11D0B8
:100340001F78612F02DB1F78662F0BDD1F78412F8E
:1003500002DB1F78462F05DD1F78582F02D01F784B
:10036000782F0CD102B12EE01F78612F03DB1F78AC
:10037000203F0F7001E01F780F70491C1FE01F78AD
:10038000222F04D102B11EE00126012417E01F78BC
:10039000202F14D01F782C2F11D0FF2613E01F78A8
:1003A000222F00D1002402B10DE044B11F785C2F50
:1003B00002D15B1C471CF8B21F780F70491C471C08
:1003C000F8B25B1CA2E700BF00270F702E70F0BDD3
:1003D00010B50446002010700BE020780870641CF3
:1003E000491C1078401C10701078984201DB0120E5
:1003F00010BD2078202802D020780028EDD10020E0
:10040000087000BFF4E700002DE9FF4F85B080467B
:1004100089460027002004900390012002904FF0AD
:10042000000B002544461DE02078202816D005F05A
:100430007F00052812DA0DB945F0800505F07F0030
:10044000042803D120782A2800D00EE0207805F077
:100450007F010DF80100681CC5B202E0852D00D1B6
:1004600003E0641C20780028DED100BF8DB100209D
:1004700005F07F010DF8010051A1684600F082FAF5
:1004800018B900210898017002E001210898017054
:1004900000254FF0000A444614E0641C0AF10100F4
:1004A00000F0FF0A2078202802D020782A2809D1DD
:1004B000204600F0D9F90646282E03D02A2E01D076
:1004C000CDF810A02078282802D020780028E4D188
:1004D0004446049810B10498401C04444FF0000AAC
:1004E000002654E0207810B94FF0010A50E020783F
:1004F000282803D116B9781CC7B213E02078292820
:1005000008D13EB917B1781EC7B201E04FF0010A19
:1005100047B93DE02078222804D10EB9012000E03F
:100520000020064647B9207820282FD0207889F867
:10053000000009F1010929E020782C2804D10120CC
:100540000290681CC5B214E02078202811D02078D1
:1005500028280ED04DB9BBF1050F06DA20780DF82A
:100560000B000BF1010000F0FF0B0298401CC0B221
:100570000290012F0AD10298022807D10298401C4C
:10058000C0B202900398401CC0B20390641CA9E75B
:1005900000BF0398012809D100200DF80B0008A125
:1005A000684600F0EFF908B9002003900799039816
:1005B0000870002089F80000504609B0BDE8F08FAF
:1005C000766F6964000000002DE9F043B5B0054680
:1005D0000F460024002604E000213D488155701C90
:1005E000C6B20A2EF8DB06E06D1C287818B9012087
:1005F00035B0BDE8F08328782828F5D16D1C61E07E
:1006000034AA69462846FFF779FE064635449DF828
:10061000D00020B1012827D0FF284CD149E09DF817
:10062000000000B333A9684600F029F906460EB170
:100630000220DDE7204600F04DF825490A31339AC3
:100640000A50A1F12400008B0121A14088432049D8
:100650001A39088304211E480155601CC4B20A2CB3
:1006600001DD0320C4E726E0684600F0A7F9401C3E
:1006700000F0FF08204600F02DF815490A3100EB84
:1006800001094946684600F08EF911481A38018B75
:100690000120A040014388B20D491A3908830C4853
:1006A00000F80480601CC4B20A2C01DD03209FE71F
:1006B00001E002209CE700BF2878292801D0287893
:1006C00000B900E09CE700BF3C70002090E700000C
:1006D0007A00002402460020002105E0044B5B5C08
:1006E0000344D8B24B1CD9B29142F7DB70470000EB
:1006F0007A0000240E480068006900F0010040B153
:100700000C48D0F8F0004FF6FF7108440949C1F8D1
:10071000F0000848D0F8F00005490968496A084423
:100720000449C1F8F0000846D0F8F0007047000016
:10073000B01C00246000002410B5044604EBC40083
:1007400000EB04100122C2EB800081B24FF47A70FA
:10075000FBF7C6FF01200149C87510BD60000024E9
:1007600010B50246012000E050430B1EA1F1010428
:10077000E1B2F9D110BD00006FF00100094909682C
:10078000086100BF000C07490968C86201460548B6
:10079000C16000BF00200349096848620249C1F8EE
:1007A000F0007047B01C00246000002470B51D48A4
:1007B000008800F40040002833D01A480578002053
:1007C00019494855194881681748884704461CB993
:1007D0001649C868804721E0134800F0FBF8054639
:1007E000012D00D02C46CCB1012C06D0022C08D013
:1007F000032C0AD0042C10D10BE00DA0FEF7C2FD93
:100800000BE00EA0FEF7BEFD07E00FA0FEF7BAFD5D
:1008100003E010A0FEF7B6FD00BF00BF00200149B5
:10082000088070BD10000024FC0400246000002437
:10083000BAAFCAFDB4EDCEF3210D0A00B2CECAFDA7
:10084000B4EDCEF3210D0A00B2CECAFDCCABB6E0BA
:10085000210D0A00CEB4D5D2B5BDC6A5C5E4B5C438
:10086000BAAFCAFD210D0A000146491C00E0491C2F
:100870000878202801D10029F9D1087870472DE99E
:10088000F04F05460F4600264FF00A09B3462C46A6
:100890000020386034E02078392802DC20783028C5
:1008A00011DA28782D2802D028782B2800D156B1CB
:1008B0002078462802DC2078412804DA207858285D
:1008C00017D1012E15D12078412801DB4FF01009F6
:1008D00028782D2803D14FF0020B6D1C0FE02878EB
:1008E0002B2803D14FF0010B6D1C08E0701CC6B221
:1008F00005E0207800B904E00120BDE8F08F641C19
:10090000C9E700BF2C46B9F1100F0FD1032E01DA51
:100910000220F2E72078302806D16078582803D1E9
:10092000A41CB01EC6B204E00320E6E70EB9042002
:10093000E3E71BE00EB1701EC6B22078392806DC52
:100940002078302803DB2078A0F1300A02E02078FC
:10095000A0F1370A31464846FFF702FF39680AFB23
:1009600000103860641C207800B900E0E2E700BFA6
:10097000BBF1020F04D13868C0F10008C7F800804D
:100980000020BAE702460AE010780B78984201D0BE
:1009900001207047107800B902E0521C491CF3E7AF
:1009A00000BF0020F5E706E002780A70027802B97D
:1009B00002E0401C491CF7E700BF704701460020D9
:1009C00005E00A7802B903E0421CD0B2491CF8E7FE
:1009D00000BF704710B58CB004461E230BAA03A9B4
:1009E0002046FFF7F5FC0090009810B101200CB0F4
:1009F00010BD9DF82C00044400200B900EE04048F0
:100A00009DF82C2050F8221003A8FFF7BBFF00B977
:100A100008E09DF82C00401CC0B20B909DF82C0003
:100A20000728ECD300BF9DF82C00072863D2DFE82D
:100A300000F004053C5E6564630000BF31A0FEF772
:100A4000A1FC31A0FEF79EFC3FA0FEF79BFC4EA050
:100A5000FEF798FC5CA0FEF795FC6BA0FEF792FCFD
:100A600079A0FEF78FFC87A0FEF78CFC8CA0FEF728
:100A700089FC94A0FEF786FC98A0FEF783FC9DA05D
:100A8000FEF780FCA2A0FEF77DFCA8A0FEF77AFC92
:100A9000B4A0FEF777FCC1A0FEF774FCCCA0FEF773
:100AA00071FCD8A0FEF76EFCA2E216A0FEF76AFC6D
:100AB000E4A0FEF767FC00200B900EE0F148006810
:100AC0009DF82C2000EBC2004168EFA0FEF75AFC15
:100AD0009DF82C00401CC0B20B90EA48007D9DF8A8
:100AE0002C108842EADC07A0FEF74CFC80E205A04F
:100AF000FEF748FCCCE179E24DE221E2F4E10000AE
:100B0000340000240D0A00002D2D2D2D2D2D2D2D0E
:100B10002D2D2D2D2D2D2D2D2D2D2D2D2D2D2D2D05
:100B200055534D4152542056332E332D2D2D2D2DFE
:100B30002D2D2D2D2D2D2D2D2D2D2D2D2D2D2D2DE5
:100B40002D2D2D200D0A00002020202055534D4131
:100B50005254CAC7D3C9414C49454E54454BBFAA0C
:100B6000B7A2B5C4D2BBB8F6C1E9C7C9B5C4B4AE63
:100B7000BFDAB5F7CAD4BBA5BDBBD7E9BCFE2CCD47
:100B8000A8B9FD200D0A0000CBFC2CC4E3BFC9D2DC
:100B9000D4CDA8B9FDB4AEBFDAD6FACAD6B5F7D36C
:100BA000C3B3CCD0F2C0EFC3E6B5C4C8CEBACEBA98
:100BB000AFCAFD2CB2A2D6B4D0D02ED2F2B4CB2C78
:100BC000C4E3BFC90D0A0000D2D4CBE6D2E2B8FC20
:100BD000B8C4BAAFCAFDB5C4CAE4C8EBB2CECAFD48
:100BE00028D6A7B3D6CAFDD7D62831302F3136BD87
:100BF000F8D6C62CD6A7B3D6B8BACAFD29A1A2D7B3
:100C0000D6B7FBB4AE0D0A00A1A2BAAFCAFDC8EBBD
:100C1000BFDAB5D8D6B7B5C8D7F7CEAAB2CECAFD17
:100C2000292CB5A5B8F6BAAFCAFDD7EEB6E0D6A75F
:100C3000B3D63130B8F6CAE4C8EBB2CECAFD2CB296
:100C4000A2D6A7B3D60D0A00BAAFCAFDB7B5BBD8B6
:100C5000D6B5CFD4CABE2ED6A7B3D6B2CECAFDCF94
:100C6000D4CABEBDF8D6C6C9E8D6C3B9A6C4DC2C62
:100C7000D6A7B3D6BDF8D6C6D7AABBBBB9A6C4DC27
:100C80002E0D0A00BCBCCAF5D6A7B3D63A77777743
:100C90002E6F70656E6564762E636F6D0D0A0000B1
:100CA00055534D415254D3D037B8F6CFB5CDB3C319
:100CB000FCC1EE28B1D8D0EBD0A1D0B4293A0D0AAE
:100CC000000000003F3A202020202020BBF1C8A1D6
:100CD000B0EFD6FAD0C5CFA20D0A000068656C70DF
:100CE0003A202020BBF1C8A1B0EFD6FAD0C5CFA2E0
:100CF0000D0A00006C6973743A202020BFC9D3C369
:100D0000B5C4BAAFCAFDC1D0B1ED0D0A0A000000EA
:100D100069643A2020202020BFC9D3C3BAAFCAFDDE
:100D2000B5C44944C1D0B1ED0D0A0A006865783AEE
:100D300020202020B2CECAFD3136BDF8D6C6CFD491
:100D4000CABE2CBAF3B8FABFD5B8F12BCAFDD7D6B4
:100D5000BCB4D6B4D0D0BDF8D6C6D7AABBBB0D0A9A
:100D60000A0000006465633A20202020B2CECAFD4C
:100D70003130BDF8D6C6CFD4CABE2CBAF3B8FABF4C
:100D8000D5B8F12BCAFDD7D6BCB4D6B4D0D0BDF8F7
:100D9000D6C6D7AABBBB0D0A0A00000072756E74D6
:100DA000696D653A312CBFAAC6F4BAAFCAFDD4CB7F
:100DB000D0D0BCC6CAB13B302CB9D8B1D5BAAFCAB5
:100DC000FDD4CBD0D0BCC6CAB13B0D0A0A0000008E
:100DD000C7EBB0B4D5D5B3CCD0F2B1E0D0B4B8F154
:100DE000CABDCAE4C8EBBAAFCAFDC3FBBCB0B2CE41
:100DF000CAFDB2A2D2D4BBD8B3B5BCFCBDE1CAF81F
:100E00002E0D0A002D2D2D2D2D2D2D2D2D2D2D2D81
:100E10002D2D2D2D2D2D2D2D2D2D2D2D2D2D414CCF
:100E200049454E54454B2D2D2D2D2D2D2D2D2D2D40
:100E30002D2D2D2D2D2D2D2D2D2D2D2D2D2D2D20EF
:100E40000D0A00002D2D2D2D2D2D2D2D2D2D2D2D6F
:100E50002D2D2D2D2D2D2D2D2D2D2D2D2DBAAFCA16
:100E6000FDC7E5B5A52D2D2D2D2D2D2D2D2D2D2D90
:100E70002D2D2D2D2D2D2D2D2D2D2D2D2D2D2D2DA2
:100E8000200D0A006000002425730D0A00000000F8
:100E900059A0FEF777FA00200B901AE0664909681E
:100EA0009DF82C2001EBC20101AB02AA486803A9FE
:100EB000FFF7AAFA604800689DF82C1050F831201E
:100EC00003A95EA0FEF75EFA9DF82C00401CC0B29C
:100ED0000B905948007D9DF82C108842DEDCAFF263
:100EE000DC30FEF74FFA83E0AFF2E830FEF74AFA63
:100EF0000BAA03A92046FFF701FA9DF82C00C8B9F8
:100F0000694603A8FFF7BBFC0B909DF82C0020B9A5
:100F10004FA00099FEF736FA0EE09DF82C00042849
:100F200001D0022063E54DA0FEF72CFA01204249D2
:100F3000C87501E002205AE547A0FEF723FA57E002
:100F400045A0FEF71FFA0BAA03A92046FFF7D6F922
:100F50009DF82C00C8B9694603A8FFF790FC0B90D8
:100F60009DF82C0020B942A00099FEF70BFA0EE084
:100F70009DF82C00042801D0022038E53FA0FEF7A0
:100F800001FA00202C49C87501E002202FE532A0AB
:100F9000FEF7F8F92CE030A0FEF7F4F90BAA03A94C
:100FA0002046FFF7ABF99DF82C00C8B9694603A8A5
:100FB000FFF765FC0B909DF82C0078B91E4900984E
:100FC00081F8EC00084690F8EC0018B130A0FEF76C
:100FD000D9F907E035A0FEF7D5F903E0022006E5D0
:100FE000022004E51CA0FEF7CDF901E00120FEE49B
:100FF00000BF0020FBE400002D2D2D2D2D2D2D2DCB
:101000002D2D2D2D2D2D2D2D2D2D2D2D2D2D2D2D10
:101010002DBAAFCAFD204944202D2D2D2D2D2D2D6B
:101020002D2D2D2D2D2D2D2D2D2D2D2D2D2D2D2DF0
:101030002D2D2D2D200D0A00600000242573206920
:10104000642069733A0D0A3058253038580D0A006B
:101050004845583A305825580D0A00003136BDF839
:10106000D6C6B2CECAFDCFD4CABE210D0A0000003A
:101070004445433A256C750D0A0000003130BDF837
:10108000D6C6B2CECAFDCFD4CABE210D0A0000001A
:1010900052756E2054696D652043616C63756C6197
:1010A00074696F6E204F4E0D0A00000052756E205D
:1010B00054696D652043616C63756C6174696F6E12
:1010C000204F46460D0A00000160704701000200F3
:1010D0000400060008000A000C0010002000400078
:1010E000800000010000000001020304010203046B
:1010F00006070809010002000400060008000A00B3
:101100000C001000200040008000000101000200DF
:101110000400060008000A000C0010002000400037
:10112000800000010000000000000000000000003E
:10113000000000003F400000000000000000300000
:10114000400030004000000009000BC03D000BC013
:101150003D00090018C024407FE02240318000009B
:10116000180024C01B000D803240018003801C4009
:1011700027401C8007400040100060000000000075
:10118000000000000000000000001F802040402000
:101190000000402020401F800000000009000600E1
:1011A0001F80060009000000040004003F800400C6
:1011B00004000000001000600000000000000000BB
:1011C00004000400040004000400000000000040CB
:1011D0000000000000000000002001C006003800F0
:1011E000400000001F802040204020401F80000061
:1011F000000010403FC000400000000018C0214027
:101200002240244018400000108020402440244008
:101210001B80000002000D0011003FC001400000D3
:101220003C80244024402440238000001F80244030
:1012300024403440038000003000200027C03800E4
:10124000200000001B802440244024401B8000001C
:101250001C0022C0224022401F800000000000002D
:1012600008400000000000000000000004600000D2
:1012700000000000000004000A001100208040402F
:1012800009000900090009000900000000004040B1
:10129000208011000A0004001800200023402400D0
:1012A000180000001F802040274029401F400000F8
:1012B000004007C039000F0001C0004020403FC07F
:1012C000244024401B8000001F80204020402040FC
:1012D0003080000020403FC0204020401F800000A0
:1012E00020403FC024402E4030C0000020403FC07E
:1012F00024402E00300000000F00108020402240CB
:101300003380020020403FC0040004003FC0204062
:10131000204020403FC020402040000000602020AE
:1013200020203FC02000200020403FC024400B0070
:1013300030C0204020403FC020400040004000C05E
:101340003FC03C0003C03C003FC0000020403FC005
:101350000C4023003FC020001F8020402040204040
:101360001F80000020403FC02440240018000000DF
:101370001F802140214020E01FA0000020403FC0EE
:101380002440260019C0004018C0244024402240B8
:1013900031800000300020403FC02040300000007D
:1013A00020003F80004000403F80200020003E00A1
:1013B00001C0070038002000380007C03C0007C00B
:1013C00038000000204039C0060039C0204000002D
:1013D0002000384007C0384020000000304021C0C5
:1013E0002640384020C00000000000007FE0402080
:1013F00040200000000070000C000380004000004E
:101400000000402040207FE000000000000020009D
:10141000400020000000000000100010001000102C
:10142000001000100000000040000000000000005C
:10143000000002800540054003C0004020003FC07E
:101440000440044003800000000003800440044086
:101450000640000000000380044024403FC00040DC
:1014600000000380054005400340000000000440E8
:101470001FC0244024402000000002E00550055019
:101480000650042020403FC00440040003C0004038
:101490000000044027C000400000000000100010C1
:1014A000041027E00000000020403FC0014007007A
:1014B00004C00440204020403FC0004000400000E5
:1014C00007C0040007C0040003C00000044007C0B8
:1014D0000440040003C000400000038004400440B6
:1014E00003800000041007F0045004400380000053
:1014F000000003800440045007F00010044007C0BF
:1015000002400400040000000000064005400540C1
:1015100004C00000000004001F80044000400000E0
:10152000040007800040044007C00040040007009A
:1015300004C0018006000400060001C0070001C0CD
:1015400006000000044006C0010006C00440000080
:101550000410071004E001800600040000000440AD
:1015600005C00640044000000000000004007BE0CD
:1015700040200000000000000000FFF0000000001C
:10158000000040207BE004000000000040008000DC
:10159000400020002000400000000000000000008B
:1015A00000000000000000000000000000001FCC50
:1015B000000C000000000000000008003000600087
:1015C0000800300060000000022003FC1E20022002
:1015D00003FC1E200220000000000E1811043FFF33
:1015E00010840C78000000000F0010840F3800C039
:1015F000077818840078000000780F8410C4112444
:101600000E9800E4008400080800680070000000E4
:10161000000000000000000000000000000007E0E3
:10162000181820044002000000004002200418188E
:1016300007E00000000000000240024001800FF0BF
:1016400001800240024000000080008000800FF80E
:1016500000800080008000000001000D000E0000EE
:1016600000000000000000000000008000800080FA
:1016700000800080008000800000000C000C000052
:1016800000000000000000000000000600180060DC
:101690000180060018002000000007F00808100470
:1016A0001004080807F000000000080408041FFCEC
:1016B000000400040000000000000E0C10141024B0
:1016C000104411840E0C000000000C1810041104CA
:1016D000110412880C700000000000E003200424B4
:1016E00008241FFC0024000000001F98108411042F
:1016F0001104108810700000000007F00888110421
:10170000110418880070000000001C00100010FC7C
:1017100013001C001000000000000E38114410845B
:10172000108411440E38000000000700088C10449B
:101730001044088807F00000000000000000030CBF
:10174000030C000000000000000000000001010682
:1017500000000000000000000000008001400220A6
:1017600004100808100400000220022002200220B9
:1017700002200220022000000000100408080410CB
:10178000022001400080000000000E001200100C3A
:10179000106C10800F00000003E00C1813E41424F8
:1017A00017C4082807D000000004003C03C41C40F4
:1017B000074000E4001C000410041FFC1104110485
:1017C00011040E880070000003E00C1810041004CF
:1017D000100410081C10000010041FFC100410045A
:1017E0001004080807F0000010041FFC1104110485
:1017F00017C410040818000010041FFC1104110085
:1018000017C010000800000003E00C1810041004BA
:1018100010441C780040000010041FFC108400805D
:10182000008010841FFC10040000100410041FFC32
:10183000100410040000000000030001100110015A
:101840001FFE10001000000010041FFC1104038094
:101850001464181C1004000010041FFC1004000481
:1018600000040004000C000010041FFC1F0000FC1A
:101870001F001FFC1004000010041FFC0C040300D8
:1018800000E010181FFC100007F0080810041004F6
:101890001004080807F0000010041FFC10841080DA
:1018A000108010800F00000007F00818102410248A
:1018B000101C080A07F2000010041FFC110411009C
:1018C00011C011300E0C000400000E1C1104108415
:1018D000108410441C3800001800100010041FFC75
:1018E000100410001800000010001FF8100400047D
:1018F000000410041FF8100010001E0011E0001C6E
:10190000007013801C0010001FC0103C00E01F007E
:1019100000E0103C1FC000001004180C163401C079
:1019200001C01634180C100410001C00130400FC35
:1019300013041C00100000000804101C1064108424
:1019400013041C04101800000000000000007FFEBB
:101950004002400240020000000030000C00038002
:101960000060001C00030000000040024002400232
:101970007FFE00000000000000000000200040008A
:1019800040004000200000000001000100010001B3
:1019900000010001000100010000400040002000A3
:1019A0000000000000000000000000980124014435
:1019B0000144014400FC000410001FFC00880104E5
:1019C000010400880070000000000070008801041D
:1019D0000104010400880000000000700088010478
:1019E000010411081FFC0004000000F80144014438
:1019F0000144014400C800000000010401040FFC80
:101A00001104110411001800000000D60129012959
:101A1000012901C90106000010041FFC0084010017
:101A20000100010400FC000400000104190419FC79
:101A30000004000400000000000000030001010198
:101A4000190119FE0000000010041FFC00240040D2
:101A500001B4010C010400000000100410041FFC7C
:101A60000004000400000000010401FC0104010066
:101A700001FC0104010000FC010401FC00840100E0
:101A80000100010400FC0004000000F8010401044E
:101A90000104010400F80000010101FF00850104B8
:101AA000010400880070000000000070008801043C
:101AB0000104010501FF00010104010401FC00848F
:101AC0000104010001800000000000CC0124012479
:101AD000012401240198000000000100010007F822
:101AE0000104010400000000010001F800040004EA
:101AF0000004010801FC0004010001800170000CD9
:101B0000001001600180010001F0010C003001C0F3
:101B10000030010C01F0010000000104018C007490
:101B20000170018C01040000010101810171000EAE
:101B3000001801600180010000000184010C0134E3
:101B400001440184010C00000000000000000000BE
:101B500001003EFC400240020000000000000000C6
:101B6000FFFF0000000000000000400240023EFCB9
:101B70000100000000000000000060008000800004
:101B80004000400020002000000000000000000095
:101B90000000000000000000000000000000000045
:101BA0000000000000000000000000000000000035
:101BB00000000000000000000000000F80380FFE51
:101BC000380F803800000000000000000000000016
:101BD0000000000000000100000600000C000038BA
:101BE00000003100000600000C000038000030004A
:101BF000000000000000000061800067F807F98025
